:020000040800F2
:1000000000000520F902000845600008496000086A
:100010004D600008516000085560000800000000B5
:100020000000000000000000000000000D040008B7
:100030005960000800000000150400088151000804
:1000400029040008290400082904000829040008DC
:1000500029040008290400082904000829040008CC
:1000600029040008290400082904000829040008BC
:1000700029040008290400082904000829040008AC
:10008000290400082904000829040008290400089C
:10009000290400082904000829040008290400088C
:1000A000290400082904000829040008290400087C
:1000B0002904000849560008595600082904000878
:1000C000290400082904000829040008290400085C
:1000D000290400082904000829040008290400084C
:1000E000290400082904000829040008290400083C
:1000F000290400082904000829040008290400082C
:10010000290400082904000829040008290400081B
:10011000290400082904000829040008290400080B
:100120002904000829040008290400083956000899
:1001300029040008290400082904000829040008EB
:1001400029040008290400082904000829040008DB
:1001500029040008290400082904000829040008CB
:1001600029040008290400082904000829040008BB
:1001700029040008290400082904000800000000E0
:10018000290400082904000829040008290400089B
:10019000290400082904000829040008290400088B
:1001A000290400082904000829040008290400087B
:1001B000290400082904000829040008290400086B
:1001C000290400082904000800B583B003F054FC9A
:1001D000384B394A1360394A136039490CE00A68D0
:1001E0004B6801F10C04886803E01168196004335E
:1001F00004329842F9D82146324B9942EFD32E4B24
:100200001A68314B9A4204D12C4B1A682F4B9A42F0
:1002100000D0FEE7274B2E4A13602E4A13602E4B68
:100220000AE0194651F8082B5B6802E000201060D4
:1002300004329A42FAD30B46284A9342F1D3244B14
:100240001B6813B9234B1B6803B1FEE704F00CF9DC
:1002500001A8694603F08CFB214C224B1C1BA41007
:10026000002504E01E4B53F8253098470135AC4279
:10027000F8DC1D4C1D4B1C1BA410002504E01A4B80
:1002800053F8253098470135AC42F8DC01980099C5
:1002900005F040FA0546164C164B1C1BA41004E052
:1002A000013C134B53F824309847002CF8DC2846C7
:1002B00003F030FBBABADECA00000020441D002063
:1002C0002C040008440400087856341232547698FE
:1002D000481D0020605E002044040008540400080B
:1002E000540400085404000854040008540400088E
:1002F000540400085404000808B5FFF765FF00BF68
:1003000000BEFEE71EF0040F0CBFEFF30880EFF312
:1003100009807146414A10472DE9F04182B00446F8
:100320008846134B5E6B9D6B9F6A1B6B13F0020F2D
:100330000DD00F4BDB6A002B09DA4BF6AB6103F0F3
:1003400025FC20B14FF00042094BDA620CE009486D
:1003500003F022FBCDF800802046394632462B467A
:1003600003F09CFB00BEFEE702B0BDE8F08100BFD9
:1003700000ED00E0D885000800BEFEE71EF0040F87
:100380000CBFEFF30880EFF309807146244A104751
:100390002DE9F04182B007468846084B5D6B9C6BA7
:1003A0009E6A074803F0F8FACDF8008038463146D7
:1003B0002A46234603F072FB00BEFEE700ED00E094
:1003C000E88500081EF0040F0CBFEFF30880EFF380
:1003D00009807146134A10472DE9F04182B0074663
:1003E0008846084B5D6B9C6B9E6A074803F0D4FA05
:1003F000CDF80080384631462A46234603F04EFBAE
:1004000000BEFEE700ED00E0F485000800BEFEE758
:1004100000BEFEE700BEFEE77047000019030008BB
:0C04200091030008D903000800BEFEE7AD
:10042C00E40E010800000020481D0020E40E010825
:10043C000000001000000010481D0020645E002029
:08044C00000000100000001088
:1004580010B5044602F018F8064BA3FB00308009DB
:1004680000F092F94FF0FF302146002200F038F9F1
:10047800002010BDD34D621008B5032000F012F91A
:100488000020FFF7E5FF05F0D7FD002008BD00BFFD
:10049800024A136801331360704700BF4C1D0020E7
:1004A800014B1868704700BF4C1D002010B582B082
:1004B8000446002301938369012B04D942484FF471
:1004C800DD7103F059FAE36A002B18BFB3F1805FBE
:1004D8000AD0B3F1005F07D0B3F1405F04D03A48C7
:1004E80040F2BB1103F048FA94F83C30012B5FD07E
:1004F800012384F83C3023689A6812F0010F13D165
:100508009A6842F001029A60304B1B68304AA2FB9D
:1005180003239B0C03EB4303019302E0019B013B84
:100528000193019B002BF9D12268936813F0010F06
:1005380040D0216C274B0B4043F4807323645368ED
:1005480013F4806F05D0236C23F4405343F4805395
:100558002364236C13F4805F04D0636C23F00603D8
:10056800636401E000236364002384F83C306FF087
:1005780002031360184B5B6813F01F0F0AD123683E
:100588009A6812F0405F17D19A6842F080429A60E8
:10059800002016E02368114A93420FD19A6812F09E
:1005A800405F0DD19A6842F080429A60002008E0CE
:1005B800022006E0002004E0002002E0002000E025
:1005C800002002B010BD00BF3C8200080C000020D3
:1005D80083DE1B43FEF8FFFF00230140002001409B
:1005E80070B503689A6812F4806F0CD09B6813F496
:1005F800807F08D0036C43F020030364002380F855
:100608003C30012070BD0D460446FFF749FF064601
:1006180011E0B5F1FF3F0ED025B1FFF741FF801B78
:10062800A84208D9236C43F004032364002384F808
:100638003C30032070BD23681A6812F0020FE8D01E
:100648006FF012021A60236C43F40073236423686A
:100658009A6812F0405F17D1A269BAB9DA6A12F43F
:10066800700F03D09B6813F4806F11D1236C23F4AF
:1006780080732364236C13F4805F0BD1236C43F0E5
:1006880001032364002070BD002070BD002070BDF0
:10069800002070BD002070BD0368D86C704700BF93
:1006A800006C704710B50446C31E042B03D90948D3
:1006B800A42103F061F904F00700074AD36823F482
:1006C800E0631B041B0C43EA0020044B0343D36084
:1006D80010BD00BF6C82000800ED00E00000FA05C4
:1006E80070B504460E4615460F2A03D91848BC2192
:1006F80003F042F90F2E03D91548BD2103F03CF948
:10070800144BDB68C3F30223C3F10702042A28BF92
:100718000422191D062901D9D81E00E00020012352
:1007280003FA02F2013A324002FA00F183405A1EFB
:100738002A400A43002C06DA04F00F041201D2B250
:10074800054B1A5570BD1201D2B2044B1A5570BD33
:100758006C82000800ED00E014ED00E000E400E029
:1007680010B5041E03DA0648D02103F005F9610923
:1007780004F01F040123A340024A42F8213010BDAF
:100788006C82000800E100E00138B0F1807F0AD2F5
:10079800064B5860F021064A82F823100020986022
:1007A80007221A6070470120704700BF10E000E080
:1007B80000ED00E010B50446042818BF002804D056
:1007C800094840F2B31103F0D7F8042C05D1074AC1
:1007D800136843F00403136010BD044A136823F040
:1007E8000403136010BD00BF6C82000810E000E035
:1007F800704700BFC8B110B5044602680C4B9A4256
:1008080003D00C48EE2103F0B7F8237913F0FF0F5B
:1008180004D1002363712046FFF7EAFF0223237106
:10082800002020610123237110BD0120704700BF03
:1008380000740040A082000838B504460D4600291F
:1008480018BF102904D01D484FF4B77103F094F86D
:100858006379012B30D0012363710222227122684F
:100868001168AB400B43136085B92268116813689F
:1008780003F03803382B14BF0023012313EA910334
:1008880015D0536843F00103536010E022681168E3
:10089800136803F46013B3F5601F14BF002301232A
:1008A80013EA914303D0536843F0020353600123D2
:1008B80023710020607138BD022038BDA082000875
:1008C800F8B504460E4615460B68002B18BF242BB6
:1008D80012D00C2B10D0142B0ED01C2B0CD0042BA8
:1008E8000AD02C2B08D0342B06D03C2B04D01C4823
:1008F80040F20E3103F040F87368002B18BF022B4A
:1009080004D0174840F20F3103F036F8002D18BF15
:10091800102D04D012484FF4447103F02DF8637978
:10092800012B1BD0012060710223237127683968CD
:1009380040F6FE73AB4021EA0302316873680B434B
:10094800AB4013433B6021680A68C023AB4022EAEE
:1009580003030B60207100206071F8BD0220F8BD10
:10096800A0820008F0B583B0074614461D46002350
:1009780001930E46994218BF102904D0144840F23A
:10098800463102F0F9FF002C18BF042C06D0082CC1
:1009980004D00F4840F2473102F0EEFF4FF6F073F3
:1009A8009D4204D90A484FF4527102F0E5FF3B68B2
:1009B800019326B9019B1C440834019403E0019B70
:1009C8001C4414340194019B1D60002003B0F0BD49
:1009D800A082000830B405682C6824F480242C60B8
:1009E800046863608368402B04D103689A600368D5
:1009F800D96003E0036899600368DA6030BC704727
:100A08000268D3B2103B0949A1FB03131B0908492B
:100A1800C95C4165032B04D9064B134004330365B5
:100A280002E0044B13400365006D7047ABAAAAAA05
:100A3800D082000800FCFFFF002800F00E8110B5EE
:100A480004460368864A87498B4218BF93422ED0D2
:100A5800183293422BD01832934228D0183293423E
:100A680025D01832934222D0183293421FD0183220
:100A780093421CD002F55672934218D01832934212
:100A880015D01832934212D0183293420FD0183230
:100A980093420CD01832934209D01832934206D0B0
:100AA8001832934203D07048EC2102F065FF636866
:100AB800002B18BFB3F1007F15D0B3F1806F12D0AF
:100AC800B3F1C06F0FD0B3F1006F0CD0B3F1206F4A
:100AD80009D0B3F1406F06D0B3F1606F03D062481C
:100AE800ED2102F049FFA368002B18BF402B05D069
:100AF800802B03D05C48EE2102F03EFFE368B3F59B
:100B0800007F18BF002B03D05748EF2102F034FFB5
:100B18002369B3F5806F18BF002B03D05248F0212A
:100B280002F02AFF6369002B18BFB3F5006F06D0E7
:100B3800B3F5805F03D04C48F12102F01DFFA36993
:100B4800002B18BFB3F5005F06D0B3F5804F03D074
:100B58004548F22102F010FFE369002B18BFB3F5F6
:100B6800807F05D0202B03D03F48F32102F004FFFB
:100B7800236A002B18BFB3F5803F09D0B3F5003FB7
:100B880006D0B3F5403F03D03748F42102F0F4FE15
:100B9800636A002B18BF042B03D03348F52102F0F9
:100BA800EBFE636A33B3A36A032B03D92E48FA21F9
:100BB80002F0E2FEE36A002B18BFB3F5000F09D07C
:100BC800B3F1807F06D0B3F1C07F03D02648FB2164
:100BD80002F0D2FE236B002B18BFB3F5001F09D01B
:100BE800B3F5800F06D0B3F5C00F03D01E48FC2123
:100BF80002F0C2FE022384F83530206802681B4BDD
:100C080013406168A2681143E268114322691143E5
:100C180062691143A2691143E2691143226A0A43D6
:100C28001343626A042A03D1E16A226B0A4313431D
:100C380003602268536923F00703616A0B430429A0
:100C480001D1A16A0B4353612046FFF7D9FE00206A
:100C5800E064012384F8353010BD0120704700BFDF
:100C68002860024010600240D88200083F8010F0DF
:100C7800F8B590F83440012C2FD01D4616460F4683
:100C88000446012380F83430022380F835306A1E88
:100C98004FF6FE739A4204D911484FF4E07102F0FE
:100CA8006BFE2268136823F001031360204639465F
:100CB80032462B46FFF78EFE2268136843F01E0368
:100CC80013602268536943F08003536122681368F4
:100CD80043F0010313600020F8BD0220F8BD00BFF7
:100CE800D882000838B50446056D2A68416D082386
:100CF8008B401A4219D003681A6812F0040F14D0F6
:100D08001A6822F004021A60426D08239340AB600F
:100D1800C36C43F00103C364042380F83530002317
:100D280080F83430836C03B198472A68616D584B5A
:100D38008B401A421AD023685A6912F0800F15D0D6
:100D48005A6922F080025A61626D514B9340AB6040
:100D5800E36C43F00203E364042384F83530002392
:100D680084F83430A36C0BB1204698472A68616D2B
:100D7800484B8B401A421AD023681A6812F0020FA7
:100D880015D01A6822F002021A60626D414B934036
:100D9800AB60E36C43F00403E364042384F8353068
:100DA800002384F83430A36C0BB1204698472A6896
:100DB800616D10238B401A422DD02268116811F002
:100DC800080F28D0116811F4802F11D0AB60236868
:100DD8001A6812F4002F03D1312384F8353016E055
:100DE8001B6813F4002F12D0412384F835300EE02D
:100DF800136813F4807F03D1136823F0080313608A
:100E0800626D10239340AB60312384F83530236C36
:100E18000BB1204698472A68616D20238B401A42FF
:100E280034D02268116811F0100F2FD0116811F416
:100E3800802F13D0AB6023681A6812F4002F04D1F6
:100E4800636C1BB32046984738BD1B6813F4002F0A
:100E58001CD0E36BD3B12046984738BD136813F410
:100E6800807F03D1136823F010031360626D202381
:100E78009340AB60E36CE364112384F835300023BE
:100E880084F83430E36B0BB12046984738BD00BF77
:100E980001008000040080002DE9F04F83B08046F7
:100EA8000F46B34BB34A904218BF98422BD003F574
:100EB8000063C31A18BF012302F50062904222D0D2
:100EC8000BB3AD4BC31A18BF012302F50062904261
:100ED80019D0C3B1A94BC31A18BF012302F5006288
:100EE800904210D07BB1A64BC31A18BF012302F55C
:100EF8000062904207D033B1A24B984203D0A24877
:100F0800C32102F039FD3B881BB99F48C42102F078
:100F180033FD7B68112B18BF012B20D9022B1ED063
:100F2800122B1CD0994A934219D002F58012934291
:100F380015D002F58012934211D0A2F5F81293420F
:100F48000DD002F58012934209D002F58012934227
:100F580005D0032B03D08C48C52102F00DFDBB68DA
:100F6800022B03D98848C62102F006FD0024F8E0C8
:100F7800A1460125A5403B6803EA050AAA4540F0B9
:100F8800EF807B68122B18BF022B1CD13B690F2BFB
:100F980018BF0C2B07D90D2B05D00E2B03D07A4880
:100FA800D72102F0E9FCE608083658F8261004F0C4
:100FB800070080000F23834021EA03023B69834036
:100FC800134348F82630D8F800304FEA440B03267C
:100FD80006FA0BF6F64306EA03027B6803F00303FE
:100FE80003FA0BF31343C8F800307B685A1E112B21
:100FF80018BF012A01D9122B1CD1FB68032B03D976
:101008006148EB2102F0B8FCD8F8083006EA030280
:10101800FB6803FA0BF31343C8F80830D8F8043018
:1010280023EA05037D68C5F3001505FA09F51D4394
:10103800C8F80450D8F80C303340BE6806FA0BF6EE
:101048001E43C8F80C607B6813F0805F00F088804E
:10105800002301934E4B5A6C42F480425A645B6CF5
:1010680003F480430193019BA308991C494A52F851
:10107800211004F0030080000F22824021EA0201BF
:101088003C4A904537D002F58062904531D002F550
:10109800806290452BD002F58062904525D002F5FC
:1010A800806290451FD002F58062904519D002F504
:1010B8008062904513D002F5806290450DD002F50C
:1010C8008062904507D002F58062904501D10922DF
:1010D80012E00A2210E008220EE007220CE00622A5
:1010E8000AE0052208E0042206E0032204E00222C6
:1010F80002E0012200E0002282400A43023325492F
:1011080041F82320244B1A686FEA0A0303EA020114
:10111800786810F4803F01D04AEA02011E4A116043
:10112800526803EA0201786810F4003F01D04AEAE5
:101138000201194A5160926803EA0201786810F4C2
:10114800801F01D04AEA0201134A9160D268134015
:10115800796811F4001F01D04AEA02030E4AD360ED
:1011680001340F2C7FF604AF03B0BDE8F08F00BF49
:10117800000402400000024000140240001C02402B
:1011880000240240002802400883000800001110D3
:101198000038024000380140003C014038B505469F
:1011A8000C4621B9054840F28D1102F0E5FB2B6988
:1011B800234201D0012038BD002038BD0883000833
:1011C80070B5064615460C4621B9094840F2AD11DE
:1011D80002F0D2FB012D04D905484FF4D77102F073
:1011E800CBFB0DB1B46170BD2404B46170BD00BF08
:1011F800088300082DE9F04180460E4617461D4633
:10120800069C0368224A23498B4218BF93420CD09C
:1012180002F58062934208D002F58062934204D0BE
:101228001D4841F2590102F0A7FBB5F1807F18BFB4
:10123800B5F1007F05D025B1174841F25A0102F0F7
:101248009BFBB4F5804F18BFB4F5105F0BD0231C7F
:1012580018BF0123B4F5005F05D023B10E4841F251
:101268005B0102F089FBD8F80020536823F07F73F4
:1012780023F4593323F47F7323F00303C6F30906D9
:1012880046EA074635432C431C435460BDE8F081C9
:1012980000580040005400403883000870B50446E8
:1012A8000D46FFF7FDF8064623689B6913F0100FFB
:1012B80012D1002070BDB5F1FF3F0DD025B1FFF769
:1012C800EFF8801BA84207D9012384F835300023A2
:1012D80084F83430032070BD23689A6912F0200F17
:1012E800E9D01022DA6123682022DA6123689A693A
:1012F80012F0010F01D10122DA612268536823F04C
:10130800FF7323F48B3323F4FF7323F0010353603B
:101318000423A363012084F83500002384F83430C3
:1013280070BD00BF70B504460D46FFF7B9F8064614
:1013380019E020462946FFF7B1FFD8B9B5F1FF3FBC
:1013480011D025B1FFF7ACF8801BA8420BD9A36BCD
:1013580043F02003A363012384F83530002384F885
:101368003430032070BD23689B6913F0020FE0D06E
:10137800002070BD012070BD2DE9F04105460E46E4
:1013880090461C46FFF78CF80746B8F1000F12D0BC
:101398002EE0B4F1FF3F0ED024B1FFF781F8C01B57
:1013A800A04208D9012385F83530002385F8343068
:1013B8000320BDE8F0812B689B6926EA0303C3F389
:1013C8001003002BE5D10020BDE8F081B4F1FF3F08
:1013D8000ED024B1FFF764F8C01BA04208D901233E
:1013E80085F83530002385F834300320BDE8F081D6
:1013F8002B689B6926EA0303C3F31003002BE5D08F
:101408000020BDE8F08100BF70B505460C46FFF727
:1014180047F8064616E028462146FFF73FFFC0B9C1
:1014280024B1FFF73DF8801BA0420BD9AB6B43F00A
:101438002003AB63012385F83530002385F8343069
:10144800032070BD2B689B6913F0200FE3D00020A8
:1014580070BD012070BD00BF70B504460D46FFF792
:101468001FF8064631E020462946FFF717FF0028F7
:1014780032D123689A6912F0200F14D02022DA6141
:101488002268536823F0FF7323F48B3323F4FF732C
:1014980023F0010353600023A363012084F835007F
:1014A80084F8343070BD25B1FEF7FAFF801BA842DE
:1014B8000BD9A36B43F02003A363012384F83530D1
:1014C800002384F83430032070BD23689B6913F02F
:1014D800040FC8D0002070BD012070BD002800F0A6
:1014E800A88010B504460368534A54498B4218BF74
:1014F80093420CD002F58062934208D002F58062D4
:10150800934204D04E4840F22B1102F035FAA368FA
:10151800B3F5806F04D34A484FF4967102F02CFA61
:10152800E368013B012B04D9454840F22D1102F034
:1015380023FA2369002B18BFB3F5004F04D04048A5
:101548004FF4977102F018FA6369FF2B04D93C48ED
:1015580040F22F1102F010FAA369072B04D938487A
:101568004FF4987102F008FAE369002B18BFB3F53D
:10157800002F04D0324840F2311102F0FDF9236AFD
:10158800002B18BFB3F5003F04D02D484FF49971D4
:1015980002F0F2F994F8353013F0FF0F05D100236B
:1015A80084F83430204603F065FA022384F8353095
:1015B8002268136823F0010313602268636823F02C
:1015C800706313612268936823F400439360A368EF
:1015D8005BB1E268012A04D1226843F400439360B6
:1015E80003E0226843F404439360E368022B03D1C9
:1015F80023684FF400625A6022685168114B0B430C
:1016080053602268216963690B43A16943EA012396
:10161800D3602268E169236A0B4313602268136868
:1016280043F0010313600020A063012384F83530E0
:1016380010BD0120704700BF005800400054004012
:101648003883000800800002704700BF38B310B527
:1016580004460368134A14498B4218BF93420CD0BE
:1016680002F58062934208D002F58062934204D06A
:101678000E4840F27D1102F07FF9022384F83530DC
:101688002268136823F0010313602046FFF7DCFF8C
:101698000020A06384F8350084F8340010BD0120D0
:1016A800704700BF005800400054004038830008CD
:1016B8002DE9F04383B004461D4690F83530DBB27F
:1016C800012B40F090800F461646002D18BF002AC7
:1016D80000F08B8003689B6913F4004F40F087800B
:1016E80090F83430012B00F08480012380F83430E6
:1016F800122380F8353000238363FF2D0AD94FF475
:1017080000530093FF224FF08073FFF773FD4FF0F3
:10171800FF080AE04FF400530093EAB24FF0007359
:10172800FFF768FDA84600E04E4620460A99FFF7F5
:10173800F9FD20B1A36B042B5DD1012360E0236880
:1017480006F1010932789A62013DADB2B8F101089B
:101758000CBF01230023002D0CBF002303F001035D
:10176800FBB12046802100220A9BFFF705FE0028D6
:1017780043D1FF2D0BD90023009320463946FF2281
:101788004FF08073FFF736FD4FF0FF0809E00023A4
:10179800009320463946EAB24FF00073FFF72AFD5E
:1017A800A846002DC0D120460A99FFF72DFE034612
:1017B80020B1A36B042B22D1012321E02268202130
:1017C800D16121684A6822F0FF7222F48B3222F438
:1017D800FF7222F001024A60012284F835200022BB
:1017E80084F834200CE002230AE0012308E00223F5
:1017F80006E0022304E0032302E0032300E00323BE
:10180800184603B0BDE8F0832DE9F04383B00446E1
:101818001D4690F83530DBB2012B40F090800F4622
:101828001646002D18BF002A00F08B8003689B69BC
:1018380013F4004F40F0878090F83430012B00F00B
:101848008480012380F83430222380F83530002347
:101858008363FF2D0AD94FF410530093FF224FF0F2
:101868008073FFF7C7FC4FF0FF080AE04FF41053EE
:101878000093EAB24FF00073FFF7BCFCA84600E003
:101888004E4620460421FFF7E7FD20B1A36B042B49
:101898005DD1012360E006F1010923685B6A3370BA
:1018A800013DADB2B8F101080CBF01230023002DA2
:1018B8000CBF002303F00103FBB120468021002266
:1018C8000A9BFFF759FD002843D1FF2D0BD90023B0
:1018D800009320463946FF224FF08073FFF78AFCB9
:1018E8004FF0FF0809E00023009320463946EAB28A
:1018F8004FF00073FFF77EFCA846002DC0D12046AC
:101908001921FFF781FD034620B1A36B042B22D1D7
:10191800012321E022682021D16121684A6822F050
:10192800FF7222F48B3222F4FF7222F001024A6025
:10193800012284F83520002284F834200CE00223A8
:101948000AE0012308E0022306E0022304E003235F
:1019580002E0032300E00323184603B0BDE8F08348
:101968002DE9F04782B00024019490F83540E4B2A4
:10197800012C40F08C800468A46914F4004F40F0F6
:10198800888090F83440012C00F085801F469046EE
:1019980089460646012380F83430022380F8353022
:1019A800002383633268F368012B04D1C9F309016A
:1019B8003E4B0B4303E0C9F3090343F42053536040
:1019C800FEF76EFD824611E0B7F1FF3F0ED02FB152
:1019D800FEF766FDCAEB0000B84207D9012386F876
:1019E8003530002386F8343003235BE03568AB6973
:1019F80013F0200F08D1AB6913F0100F04D196F83B
:101A08003540E4B2032CDFD1AB6913F0100F12D1CB
:101A18003046202100223B46FFF7AEFC0346002853
:101A28003BD132682021D161012286F8352000227D
:101A380086F8342036E03046202100223B46FFF766
:101A48009BFC60BB33681022DA6133682022DA61BC
:101A5800019B5A1C019243450ED13268536843F4E6
:101A6800804353603046202100223B46FFF784FC28
:101A7800B8B933682022DA61019B434592D3012328
:101A880086F83530002386F8343003230AE0022331
:101A980008E0022306E0022304E0032302E0032314
:101AA80000E00323184602B0BDE8F08700200002DA
:101AB80010B582B0002301931C4B1A6C42F080527F
:101AC8001A641B6C03F080530193019B184A136836
:101AD80043F480331360FEF7E3FC044605E0FEF7A9
:101AE800DFFC001BB0F57A7F1AD8114B5B6813F442
:101AF800803FF4D00E4A136843F400331360FEF7B6
:101B0800CFFC044605E0FEF7CBFC001BB0F57A7F5E
:101B180008D8074B5B6813F4003FF4D0002002E0BC
:101B2800032000E0032002B010BD00BF00380240CF
:101B38000070004030B583B0044603680F2B04D909
:101B48009B484FF4807101F017FF236813F0010FD1
:101B580000F08E806368002B18BFB3F5803F07D074
:101B6800B3F5A02F04D092484FF4837101F004FF1D
:101B7800904B9B6803F00C03042B0AD08D4B9B6899
:101B880003F00C03082B0DD18A4B5B6813F4800F0C
:101B980008D0884B1B6813F4003F69D06368002B9A
:101BA80066D15BE2834B1A6822F480321A601A68A5
:101BB80022F480221A601A6822F480321A60FEF732
:101BC8006FFC054605E0FEF76BFC401B642800F23D
:101BD8004782784B1B6813F4003FF4D1754A1368A9
:101BE80023F4803313606368B3F5803F09D113464B
:101BF800126822F480221A601A6842F480321A604D
:101C080015E0B3F5A02F09D16A4B1A6842F4802277
:101C18001A601A6842F480321A6008E0654B1A6844
:101C280022F480221A601A6822F480321A606368EB
:101C38007BB1FEF735FC054605E0FEF731FC401B9D
:101C4800642800F20F825B4B1B6813F4003FF4D04A
:101C58000EE0FEF725FC054605E0FEF721FC401BDB
:101C6800642800F20182534B1B6813F4003FF4D13F
:101C7800236813F0020F6ED0E368012B04D94C4897
:101C880040F2471101F078FE23691F2B04D9484818
:101C98004FF4A47101F070FE464B9B6813F00C0FD3
:101CA8000AD0444B9B6803F00C03082B1BD1414B13
:101CB8005B6813F4800F16D13E4B1B6813F0020FBC
:101CC80003D0E368012B40F0D1813A48036823F040
:101CD800F8012369F82292FAA2F2B2FA82F293404A
:101CE8000B43036037E0E3680BB3324A136843F0F1
:101CF80001031360FEF7D4FB054605E0FEF7D0FBB1
:101D0800401B642800F2B4812A4B1B6813F0020FB1
:101D1800F4D02848036823F0F8012369F82292FADE
:101D2800A2F2B2FA82F293400B43036013E0214A15
:101D3800136823F001031360FEF7B2FB054605E0C4
:101D4800FEF7AEFB401B642800F29481194B1B6818
:101D580013F0020FF4D1236813F0080F37D063692A
:101D6800012B04D912484FF4C47101F005FE6369D0
:101D7800A3B1104A536F43F001035367FEF790FB7A
:101D8800054605E0FEF78CFB401B642800F27481D1
:101D9800084B5B6F13F0020FF4D018E0054A536F3D
:101DA80023F001035367FEF77BFB05460AE000BFFB
:101DB8007883000800380240FEF772FB401B642855
:101DC80000F25C81B64B5B6F13F0020FF4D123680D
:101DD80013F0040F00F09480A368052B18BF012BA3
:101DE80004D9B0484FF4D97101F0C6FD002301931E
:101DF800AB4B1A6C42F080521A641B6C03F0805390
:101E08000193019BA84A136843F480731360FEF79B
:101E180047FB054605E0FEF743FB401B642800F23C
:101E28002F81A14B1B6813F4807FF4D09C4B1A6F51
:101E380022F001021A671A6F22F004021A671A6F59
:101E480022F001021A67FEF72BFB054607E0FEF7B2
:101E580027FB401B41F28833984200F21381904BD4
:101E68001B6F13F0020FF2D18D4A136F23F0010399
:101E78001367A368012B09D11346126F22F00402DD
:101E88001A671A6F42F001021A6714E0052B09D18C
:101E9800834B1A6F42F004021A671A6F42F001026C
:101EA8001A6708E07E4B1A6F22F004021A671A6F4D
:101EB80022F001021A67A3688BB1FEF7F1FA054612
:101EC80007E0FEF7EDFA401B41F28833984200F232
:101ED800DB80734B1B6F13F0020FF2D010E0FEF79C
:101EE800DFFA054607E0FEF7DBFA401B41F28833CC
:101EF800984200F2CB806A4B1B6F13F0020FF2D1AD
:101F0800A369022B04D967484FF4FB7101F034FD33
:101F1800A369002B00F0BC80614A926802F00C02B1
:101F2800082A00F0B780022B40F08380E369002B79
:101F380018BFB3F5800F04D05A4840F2FF1101F0E2
:101F48001BFD236A023B3D2B04D956484FF4007110
:101F580001F012FD636A323BB3F5BF7F04D95148E3
:101F680040F2012101F008FDA36A022B18BF042BDF
:101F780008D0062B06D0082B04D04A4840F202218C
:101F880001F0FAFCE36A023B0D2B04D9454840F204
:101F9800032101F0F1FC424A136823F080731360B7
:101FA800FEF77EFA054604E0FEF77AFA401B64283D
:101FB80072D83B4B1B6813F0007FF5D1226A636A25
:101FC80047F6C07191FAA1F1B1FA81F18B401A4339
:101FD800A36A5B08013B4FF4403191FAA1F1B1FAD1
:101FE80081F18B401343E26943EA0201E36A4FF04F
:101FF800706292FAA2F2B2FA82F203FA02F241EAAB
:10200800020343F00053264A5360136843F0807379
:102018001360FEF745FA044604E0FEF741FA001B98
:1020280064283BD81E4B1B6813F0007FF5D00020B6
:102038003DE01B4A136823F080731360FEF730FA03
:10204800044604E0FEF72CFA001B64282ED8144B33
:102058001B6813F0007FF5D1002028E0012026E05E
:10206800032024E0032022E0032020E001201EE0DA
:1020780003201CE003201AE0032018E0032016E0E8
:10208800032014E0032012E0032010E003200EE0F8
:1020980000200CE001200AE0032008E0032006E00D
:1020A800003802407883000800700040032003B025
:1020B80030BD00BF70B504460D460368013B0E2BCA
:1020C80004D98A4840F2622101F056FC0F2D04D948
:1020D800864840F2632101F04FFC854B1B6803F0F2
:1020E8000F03AB4280F08F80814A136823F00F03FF
:1020F8002B431360136803F00F03AB4240F0578182
:10210800236813F0020F1ED0A368002B18BF802B82
:1021180012D0902B10D0A02B0ED0B02B0CD0C02BEF
:102128000AD0D02B08D0E02B06D0F02B04D06F4873
:1021380040F2792101F020FC6E498B6823F0F0020F
:10214800A36813438B60236813F0010F00F0EB8042
:102158006368022B04D965484FF4207101F00CFC28
:102168006268012A05D1634B1B6813F4003F0ED146
:102178001FE1022A05D15F4B1B6813F0007F06D1CF
:1021880019E15C4B1B6813F0020F00F016815949E6
:102198008B6823F0030313438B60FEF781F9054630
:1021A8006368012B0FD107E0FEF77AF9401B41F273
:1021B8008833984200F203814E4B9B6803F00C036E
:1021C800042BF1D1AFE0022B17D107E0FEF768F935
:1021D800401B41F28833984200F2F380454B9B68DC
:1021E80003F00C03082BF1D19DE0FEF759F9401BD1
:1021F80041F28833984200F2E6803E4B9B6813F028
:102208000C0FF2D18FE0236813F0020F1ED0A368E1
:10221800002B18BF802B12D0902B10D0A02B0ED0E3
:10222800B02B0CD0C02B0AD0D02B08D0E02B06D076
:10223800F02B04D02D484FF4327101F09DFB2D494D
:102248008B6823F0F002A36813438B60236813F0B4
:10225800010F5DD06368022B04D9244840F2CF21D6
:1022680001F08AFB6268012A05D1224B1B6813F42E
:10227800003F0ED1A9E0022A05D11E4B1B6813F0BE
:10228800007F06D1A3E01B4B1B6813F0020F00F080
:10229800A08018498B6823F0030313438B60FEF773
:1022A800FFF806466368012B0FD107E0FEF7F8F840
:1022B800801B41F28833984200F28D800D4B9B6859
:1022C80003F00C03042BF1D122E0022B1BD106E012
:1022D800FEF7E6F8801B41F2883398427DD8054B1B
:1022E8009B6803F00C03082BF2D111E078830008F7
:1022F800003C024000380240FEF7D2F8801B41F251
:10230800883398426BD8384B9B6813F00C0FF3D185
:10231800364A136823F00F032B431360136803F046
:102328000F03AB425DD1236813F0040F1AD0E368A2
:10233800002B18BFB3F5805F0DD0B3F5A05F0AD0AE
:10234800B3F5C05F07D0B3F5E05F04D0284840F28A
:102358001E3101F011FB24498B6823F4E052E36835
:1023680013438B60236813F0080F1BD02369002BDD
:1023780018BFB3F5805F0DD0B3F5A05F0AD0B3F5F1
:10238800C05F07D0B3F5E05F04D0194840F22531AB
:1023980001F0F2FA144A936823F46043216943EA8E
:1023A800C10393600020FEF753F8002070BD0120A0
:1023B80070BD012070BD012070BD012070BD0320DB
:1023C80070BD032070BD032070BD012070BD0120C9
:1023D80070BD012070BD032070BD032070BD0320B7
:1023E80070BD012070BD00BF00380240003C0240B3
:1023F80078830008214B9B6803F00C03042B3AD028
:10240800082B01D01E4870471C4B586800F03F004D
:102418005B6813F4800F0FD01A4BB3FBF0F3174A25
:10242800506847F6C072104092FAA2F2B2FA82F2ED
:10243800D04000FB03F30EE0114BB3FBF0F30F4A5F
:10244800506847F6C072104092FAA2F2B2FA82F2CD
:10245800D04000FB03F3094A506800F440304FF4C1
:10246800403292FAA2F2B2FA82F2D0400130400031
:10247800B3FBF0F070470348704700BF00380240D4
:102488000024F40080BA8C0108B5FFF7B3FF084BAD
:102498009B6803F0F003F02292FAA2F2B2FA82F2F9
:1024A800D340044AD35CD840034B186008BD00BF32
:1024B80000380240688300080C000020F0B583B0A3
:1024C80004460268644B13401BB96448872101F035
:1024D80053FA236813F0010F16D0636B002B18BF53
:1024E800B3F5000F03D05D488D2101F045FA5C4B30
:1024F8009A6822F400029A609968626B0A439A60AB
:10250800636B1BB1002702E0002700E00127236866
:1025180013F4002F1DD0E36B002B18BFB3F5801FF9
:1025280006D0B3F5001F03D04C489D2101F024FAD2
:102538004B49D1F88C3023F44012E36B1343C1F8B4
:102548008C30E36BB3F5801F00D101271BB1002548
:1025580002E0002500E00125236813F4801F1CD049
:10256800236C002B18BFB3F5800F06D0B3F5000F0E
:1025780003D03A48B12101F0FFF93949D1F88C303C
:1025880023F44002236C1343C1F88C30236CB3F559
:10259800800F00D1012703B90125236813F0807F3C
:1025A80000D0012713F0200F6CD0002301932C4B8F
:1025B8001A6C42F080521A641B6C03F0805301932A
:1025C800019B284A136843F480731360FDF768FF82
:1025D800064605E0FDF764FF801B642800F2F084DE
:1025E800204B1B6813F4807FF4D01D4B1A6F236BAC
:1025F800534013F4407F45D0194B196F21F44070B4
:102608001A6F42F480321A671A6F22F480321A67FE
:10261800186711F0020F10D0FDF742FF064607E0D9
:10262800FDF73EFF801B41F28833984200F2CA84CE
:102638000B4B1B6F13F0020FF2D0236B03F44072A5
:10264800B2F5407F12D10648826822F4F811064A92
:102658001A400A4382600EE0F9FFFF01A8830008D0
:102668000038024000700040FFFCFF0FBB4A93682F
:1026780023F4F8139360B94A116F236BC3F30B0368
:102688000B431367236813F0100F17D0A36B002BAD
:1026980018BFB3F1807F04D0B1484FF4807101F0C6
:1026A8006BF9AE4BD3F88C2022F08072C3F88C20E3
:1026B800D3F88C10A26B0A43C3F88C20236813F458
:1026C800804F16D0636E002B18BFB3F5803F07D03C
:1026D800B3F5003F04D0A2484FF4857101F04CF9DE
:1026E8009E49D1F8903023F44032636E1343C1F809
:1026F8009030236813F4004F16D0A36E002B18BF38
:10270800B3F5802F07D0B3F5002F04D094484FF4C9
:102718008A7101F031F99149D1F8903023F44022BF
:10272800A36E1343C1F89030236813F4803F16D08A
:10273800E36E002B18BFB3F5801F07D0B3F5001F59
:1027480004D087484FF48F7101F016F98349D1F806
:10275800903023F44012E36E1343C1F8903023689D
:1027680013F4003F16D0236F002B18BFB3F5800F6A
:1027780007D0B3F5000F04D079484FF4947101F0F5
:10278800FBF87649D1F8903023F44002236F1343C5
:10279800C1F89030236813F0400F14D0636C032BFA
:1027A80018BF012B06D9022B04D06D484FF499713C
:1027B80001F0E2F86949D1F8903023F00302636C24
:1027C8001343C1F89030236813F0800F16D0A36C20
:1027D800002B18BF042B08D00C2B06D0082B04D0D4
:1027E8005F484FF49E7101F0C7F85C49D1F890300A
:1027F80023F00C02A36C1343C1F89030236813F440
:10280800807F16D0E36C002B18BF102B08D0302B1C
:1028180006D0202B04D052484FF4A37101F0ACF835
:102828004E49D1F8903023F03002E36C1343C1F8DD
:102838009030236813F4007F16D0236D002B18BF47
:10284800402B08D0C02B06D0802B04D044484FF42E
:10285800A87101F091F84149D1F8903023F0C002F5
:10286800236D1343C1F89030236813F4806F19D097
:10287800636D002B18BFB3F5807F0AD0B3F5407F96
:1028880007D0B3F5007F04D035484FF4AD7101F09F
:1028980073F83249D1F8903023F44072636D1343D2
:1028A800C1F89030236813F4006F19D0A36D002B82
:1028B80018BFB3F5806F0AD0B3F5406F07D0B3F5F2
:1028C800006F04D026484FF4B27101F055F823493F
:1028D800D1F8903023F44062A36D1343C1F89030CF
:1028E800236813F4805F19D0E36D002B18BFB3F58C
:1028F800805F0AD0B3F5405F07D0B3F5005F04D01E
:1029080017484FF4B77101F037F81449D1F89030EF
:1029180023F44052E36D1343C1F89030236813F455
:10292800005F1FD0236E002B18BFB3F5804F0AD06D
:10293800B3F5404F07D0B3F5004F04D008484FF423
:10294800BC7101F019F80549D1F8903023F44042E0
:10295800236E1343C1F8903004E000BF00380240F2
:10296800A8830008236813F4800F13D0A36FB3F172
:10297800806F18BF002B04D03A484FF4C17100F0A3
:10298800FBFF3949D1F8903023F08062A36F1343DD
:10299800C1F89030236813F4001F18D0E36FB3F127
:1029A800006F18BF002B04D02E484FF4C67100F0FA
:1029B800E3FF2D49D1F8903023F00062E36F134311
:1029C800C1F89030E36FB3F1006F00D1012523689F
:1029D80013F0080F00D0012513F4802F19D0636F6E
:1029E800002B18BFB3F1807F0AD0B3F1007F07D066
:1029F800B3F1407F04D01B4840F2A31100F0BCFFA4
:102A08001949D1F8903023F04072636F1343C1F82D
:102A18009030236813F4000F15D0D4F88030B3F148
:102A2800805F18BF002B04D00E4840F2AD1100F0B3
:102A3800A3FF0D49D1F8903023F08052D4F88030AC
:102A48001343C1F8903027B92368B3F1007F40F0F1
:102A58007281054A136823F080631360FDF720FD37
:102A6800064609E0A883000800380240FDF718FD73
:102A7800801B642800F2A882B54B1B6813F0006F16
:102A8800F4D16368323BB3F5BF7F04D9B1484FF442
:102A9800E47100F071FF236813F0010F45D0636BF8
:102AA800002B42D1A368023B052B04D9A9484FF457
:102AB800E77100F061FFA648D0F8846006F440365C
:102AC8004FF4403292FAA2F3B3FA83F3DE40D0F81F
:102AD800843003F070634FF0706797FAA7FEBEFA70
:102AE8008EFE23FA0EF1636847F6C07E9EFAAEFEAC
:102AF800BEFA8EFE03FA0EF392FAA2F2B2FA82F24C
:102B080006FA02F21A4397FAA7F3B3FA83F301FA23
:102B180003F31A43A3684FF0E04191FAA1F1B1FA27
:102B280081F18B401343C0F88430236813F4002FDD
:102B380003D0E26BB2F5801F06D013F4801F59D082
:102B4800236CB3F5800F55D1E368023B0D2B04D9F4
:102B580080484FF4EF7100F00FFF636A013B1F2BB1
:102B680004D97C484FF4F07100F006FF7848D0F89B
:102B7800846006F440364FF4403E9EFAAEF3B3FA52
:102B880083F3DE40D0F8843003F0E0434FF0E047B1
:102B980097FAA7F2B2FA82F223FA02F1626847F6CC
:102BA800C07393FAA3F3B3FA83F302FA03F39EFA1A
:102BB800AEF2B2FA82F206FA02F243EA0206E268DA
:102BC8004FF0706393FAA3F3B3FA83F39A40324356
:102BD80097FAA7F3B3FA83F301FA03F31343C0F8A0
:102BE8008430D0F88C3023F01F02636A013B134312
:102BF800C0F88C30236813F0807F43D02369032BFF
:102C080004D9544840F2F31100F0B6FE504ED6F8FD
:102C1800840000F070604FF0706292FAA2F1B1FA8D
:102C280081F1C840D6F8843003F0E0434FF0E04724
:102C380097FAA7FEBEFA8EFE23FA0EF1636847F6EE
:102C4800C07E9EFAAEFEBEFA8EFE03FA0EFC236923
:102C58004FF4403E9EFAAEFEBEFA8EFE03FA0EF325
:102C68004CEA030392FAA2F2B2FA82F200FA02F2F2
:102C78001A4397FAA7F3B3FA83F301FA03F313435A
:102C8800C6F88430236813F0007F40D02369032BF3
:102C980004D9304840F2022100F06EFEA368023BDE
:102CA800052B04D92B4840F2032100F065FEE368A8
:102CB800023B0D2B04D927484FF4017100F05CFE4C
:102CC800626847F6C07393FAA3F3B3FA83F302FA80
:102CD80003F322694FF4403191FAA1F1B1FA81F17D
:102CE8008A401A43E3684FF0706191FAA1F1B1FA92
:102CF80081F18B401A43A3684FF0E04191FAA1F1AA
:102D0800B1FA81F18B401343114AC2F88430104A5A
:102D1800136843F080631360FDF7C2FB064605E0C5
:102D2800FDF7BEFB801B642800F25081084B1B682E
:102D380013F0006FF4D0002D00F04A81044A1368A4
:102D480023F080531360FDF7ABFB05460AE000BF94
:102D580000380240A8830008FDF7A2FB401B642846
:102D680000F238819E4B1B6813F0005FF4D1636951
:102D7800323BB3F5BF7F04D99A4840F2322100F0C4
:102D8800FBFD236813F4002F01D0E26B2AB113F482
:102D9800801F58D0236C002B55D1A369023B0D2B03
:102DA80004D9904840F2392100F0E6FDA36A013BBE
:102DB8001F2B04D98B4840F23B2100F0DDFD8848E9
:102DC800D0F8885005F440354FF4403292FAA2F317
:102DD800B3FA83F3DD40D0F8883003F0E0434FF0D6
:102DE800E04696FAA6F7B7FA87F723FA07F1676974
:102DF80047F6C07393FAA3F3B3FA83F39F4092FAAA
:102E0800A2F2B2FA82F205FA02F247EA0205A269D0
:102E18004FF0706393FAA3F3B3FA83F39A402A430B
:102E280096FAA6F3B3FA83F301FA03F31343C0F84F
:102E38008830D0F88C3023F4F853A26A013A43EA78
:102E48000223C0F88C30236813F4001F46D0E36FC8
:102E5800B3F1006F42D1236A032B04D9614840F2D1
:102E68004E2100F089FD5E4ED6F8880000F07060B3
:102E78004FF0706292FAA2F3B3FA83F3D840D6F80F
:102E8800883003F0E0434FF0E04595FAA5F7B7FA2C
:102E980087F723FA07F1636947F6C07797FAA7F728
:102EA800B7FA87F703FA07FE236A4FF4403797FA11
:102EB800A7F7B7FA87F7BB404EEA030392FAA2F2E4
:102EC800B2FA82F200FA02F21A4395FAA5F3B3FABB
:102ED80083F301FA03F31343C6F88830236813F029
:102EE800080F58D0E369023B052B04D93D4840F24E
:102EF8005D2100F041FDE36A002B18BFB3F5803F68
:102F08000AD0B3F5003F07D0B3F5403F04D03548A9
:102F180040F25E2100F030FD3148D0F8885005F0CD
:102F280070654FF0706292FAA2F1B1FA81F1CD406A
:102F3800D0F8883003F440334FF4403191FAA1F6C9
:102F4800B6FA86F6F340676947F6C07696FAA6F6AB
:102F5800B6FA86F6B74091FAA1F1B1FA81F18B4041
:102F68003B4392FAA2F2B2FA82F205FA02F2134352
:102F7800E2694FF0E04191FAA1F1B1FA81F18A409A
:102F88001343C0F88830D0F88C3023F44032E36A19
:102F98001343C0F88C30124A136843F0805313600F
:102FA800FDF77EFA044604E0FDF77AFA001B642870
:102FB80012D80B4B1B6813F0005FF5D000200CE013
:102FC80003200AE0032008E0032006E0032004E0D1
:102FD800002002E0032000E0032003B0F0BD00BFA2
:102FE80000380240A88300082DE9F04105460F4645
:102FF80016461C46FDF754FA804637E0B4F1FF3F09
:1030080034D02CB1FDF74CFAC8EB0000A0422DD308
:103018002A68536823F0E00353606B68B3F5827F36
:103028000BD1AB68B3F5806F18BFB3F5004F04D16F
:103038002A68136823F040031360AB6AB3F5005F96
:103048000BD12A68136823F400531B041B0C13606C
:103058002A68136843F400531360012385F85D3030
:10306800002385F85C300320BDE8F0812B689B685D
:103078003B40B342C2D10020BDE8F0812DE9F041C8
:1030880082B007460D4614461E46FDF709FA8046EB
:1030980041E0B5F5C06F08BF002C05D1137BDBB24A
:1030A8008DF807309DF80730B6F1FF3F33D02EB1C9
:1030B800FDF7F6F9C8EB0000B0422CD33A68536824
:1030C80023F0E00353607B68B3F5827F0BD1BB68C4
:1030D800B3F5806F18BFB3F5004F04D13A68136891
:1030E80023F040031360BB6AB3F5005F0BD13A6865
:1030F800136823F400531B041B0C13603A6813680D
:1031080043F400531360012387F85D30002387F8E8
:103118005C30032005E03A6893682B40A342B8D19D
:10312800002002B0BDE8F08138B504460D464FF4E2
:10313800C05100222B46FFF7A1FF28B1236E43F0B0
:103148002003236603231AE02046802100222B4611
:10315800FFF74AFF28B1236E43F0200323660323B9
:103168000DE020464FF4C06100222B46FFF786FF92
:10317800034620B1236E43F0200323660323184639
:1031880038BD00BF704700BF002800F0228110B58D
:1031980004460368904A91498B4218BF934213D062
:1031A80002F5806293420FD002F5784293420BD029
:1031B80002F5E052934207D002F58062934203D0B1
:1031C8008748CC2100F0D8FB6368002B18BFB3F503
:1031D800827F03D08248CD2100F0CEFBA368002B6C
:1031E80018BFB3F5806F06D0B3F5004F03D07C4805
:1031F800CE2100F0C1FBE368B3F5706F18BFB3F5DB
:10320800606F24D0B3F5506F21D0B3F5406F1ED056
:10321800B3F5306F1BD0B3F5206F18D0B3F5106F2E
:1032280015D0B3F5006F12D0B3F5E06F0FD0B3F53A
:10323800C06F0CD0B3F5A06F09D0B3F5806F06D07E
:10324800B3F5407F03D06648CF2100F095FB236992
:10325800002B18BF022B03D06148D02100F08CFB53
:103268006369012B03D95E48D12100F085FBA3696E
:10327800B3F5007F18BF002B06D0B3F5802F03D01D
:103288005748D22100F078FB636B082B18BF002B3E
:1032980003D05348D32100F06FFBE369002B18BF1C
:1032A800082B0FD0102B0DD0182B0BD0202B09D0AA
:1032B800282B07D0302B05D0382B03D04848D421F1
:1032C80000F05AFB236A002B18BF802B03D0444818
:1032D800D52100F051FB636A002B18BF102B03D0D7
:1032E8003F48D62100F048FBA36A002B18BFB3F56E
:1032F800005F03D03A48D72100F03EFBE36A013B68
:103308004FF6FE72934203D93548D82100F034FBBA
:10331800236B022B03D93248D92100F02DFB94F8F6
:103328005D3023B984F85C302046FFF72BFF022379
:1033380084F85D302268136823F040031360E36863
:10334800B3F5E06F01D9002201E04FF48052B3F5E4
:10335800706F18BFB3F5E06F01D00021A162216B37
:1033680039B9B3F5E06F02D90223236301E00123E1
:10337800236320686168A368194323691943636953
:103388001943A36903F400730B43E1690B43216AF2
:103398000B43A16A19430160236B022B04D12168F6
:1033A8000B6843F400630B602068618B01F0040133
:1033B800636A1943636B1943E3680B431343436020
:1033C8002368E26A1A6100202066012384F85D30D0
:1033D80010BD0120704700BF003800400030014098
:1033E800DC830008F0B583B004460F4616461D4638
:1033F8008368002B18BFB3F5004F04D067484FF41B
:10340800CC7100F0B9FA94F85C30012B00F0BD8063
:10341800012384F85C3094F85D30012B07D0012338
:1034280084F85D30002384F85C300223B2E0002E7B
:1034380018BF002F06D1012384F85D30002284F8DC
:103448005C20A7E0032384F85D3000232366A7638C
:10345800A687E6872364A4F84430A4F84630A36816
:10346800B3F5004F04D12268136843F48043136016
:10347800A36AB3F5005F0BD12268136823F40053E5
:103488001B041B0C13602268136843F40053136079
:1034980023681A6812F0400F03D11A6842F04002FC
:1034A8001A60E368B3F5E06F19D849E020460221B5
:1034B8000A462B46FFF798FD38B1012384F85D30A2
:1034C800002384F85C30032364E02368A26B12882D
:1034D800DA60A36B0233A363E38F013BE387E38FD7
:1034E800002BE3D12FE0012B19D0204602210A46F8
:1034F8002B46FFF779FD38B1012384F85D300023AE
:1035080084F85C30032345E02368A26B1288DA60F4
:10351800A36B0233A363E38F023BE38710E02046EB
:1035280002210A462B46FFF75FFD00282FD12268AB
:10353800A36B591CA1631B781373E38F013BE387CB
:10354800E38F002BCFD1A36AB3F5005F04D12268C3
:10355800136843F48053136020462946FFF7E4FDBF
:103568000346B0B9A26832B901922268D1680191C4
:1035780092680192019A012284F85D20002284F861
:103588005C20226E32B1012304E0022302E003230F
:1035980000E00323184603B0F0BD00BFDC83000839
:1035A80070B504460E4615468368002B18BFB3F560
:1035B800004F04D042484FF49D6100F0DDF994F8C3
:1035C8005D30012B76D1002D18BF002E74D094F8F1
:1035D8005C30012B72D0012384F85C30032384F81B
:1035E8005D3000232366A663A587E5872364A4F8D6
:1035F8004430A4F84630A368B3F5004F04D12268DC
:10360800136843F480431360A36AB3F5005F0BD1DA
:103618002268136823F400531B041B0C13602268F0
:10362800136843F400531360636D264A1A64636D8C
:10363800254ADA63636D254A9A642268536823F43D
:1036480080435360E368B3F5E06F1AD8636D9B69F4
:10365800B3F5005F15D1E38F13F0010F08D122688D
:10366800536823F480435360E38F5B08E38708E0E3
:103678002268536843F480435360E38F5B08013347
:10368800E3872268606DA16B0C32E38FFDF7F0FAD7
:1036980023681A6812F0400F03D11A6842F04002FA
:1036A8001A602268536843F002035360002084F8CC
:1036B8005C0070BD022070BD012070BD022070BD8D
:1036C800DC830008E136000815370008F1360008E9
:1036D800704700BF704700BF08B5806BFFF7FAFF5F
:1036E80008BD00BF704700BF08B5806B026853680B
:1036F80023F003035360036E43F0100303660123B2
:1037080080F85D30FFF7EEFF08BD00BF00B583B05D
:10371800836B0268126812F4807F18D119684A68AE
:1037280022F002024A609A6832B901921A68D16896
:10373800019192680192019A0022DA87012283F8A6
:103748005D201A6E1AB11846FFF7CCFF02E0184642
:10375800FFF7BEFF03B05DF804FB00BF90F85D0003
:10376800704700BF704700BF704700BF704700BF79
:10377800704700BF10B5044603681A6912F0020FBB
:1037880017D0DA6812F0020F13D06FF002021A6134
:103798000123037603689B6913F0030F02D0FFF738
:1037A800E3FF04E0FFF7DEFF2046FFF7DFFF00231B
:1037B800237623681A6912F0040F19D0DA6812F018
:1037C800040F15D06FF004021A61022323762368D0
:1037D8009B6913F4407F03D02046FFF7C5FF05E03F
:1037E8002046FFF7BFFF2046FFF7C0FF00232376E0
:1037F80023681A6912F0080F19D0DA6812F0080F56
:1038080015D06FF008021A61042323762368DB6958
:1038180013F0030F03D02046FFF7A6FF05E020466C
:10382800FFF7A0FF2046FFF7A1FF002323762368B8
:103838001A6912F0100F19D0DA6812F0100F15D0AB
:103848006FF010021A61082323762368DB6913F4EA
:10385800407F03D02046FFF787FF05E02046FFF7AB
:1038680081FF2046FFF782FF0023237623681A6929
:1038780012F0010F09D0DA6812F0010F05D06FF0CD
:1038880001021A61204602F065FB23681A6912F0EA
:10389800800F09D0DA6812F0800F05D06FF080022F
:1038A8001A61204600F030F823681A6912F4807F04
:1038B80009D0DA6812F0800F05D06FF080021A6123
:1038C800204600F021F823681A6912F0400F09D049
:1038D800DA6812F0400F05D06FF040021A612046F6
:1038E800FFF746FF23681A6912F0200F09D0DA683B
:1038F80012F0200F05D06FF020021A61204600F068
:1039080001F810BD704700BF704700BFFEE700BF59
:1039180008B5034800F05EF80120FFF7F7FF00BF85
:103928000C84000808B50D4B1B6813B90C4A0B4BE7
:103938001A600A4B1A68C31C23F00303134409498D
:103948008B4206D904F040F80C2303604FF0FF3097
:1039580008BD02490B60104608BD00BF501D00207D
:10396800645E002000FC042001230360014B0B600F
:10397800704700BF0400002008B503460A46034804
:10398800194600F005F8FFF7C3FF00BF6084000880
:103998000FB480B582B000AF07F114033B600C4848
:1039A80080213A693B6804F047F878607B68002B0F
:1039B80005DD7B680648194600F056F878607B6894
:1039C80018460837BD46BDE8804004B0704700BFC0
:1039D800581D002080B582B000AF7860786803F089
:1039E800F9FF03467868194600F03EF804480121BB
:1039F80000F03AF8034618460837BD4680BD00BFB8
:103A08008C8400082DE9F04385B004460F46435CDA
:103A180013BB042528462146ABBE04461FE03546A5
:103A2800102E28BF1025002306E014F8011B04AA55
:103A38001A4402F8101C0133AB42F6D304AA13440B
:103A4800002203F8102CE9464FF004084046494686
:103A5800ABBE8046761B00E00E46002EDFD138460E
:103A680005B0BDE8F08300BF08B5FFF7CBFF08BD80
:103A780008B500F097F8054B054A9A60D3F88820F6
:103A880042F47002C3F8882008BD00BF00ED00E0D2
:103A980000000008F8B504460D4617461E4626489D
:103AA800FFF776FF25482168FFF772FF2448616811
:103AB800FFF76EFF2348A168FFF76AFF2248E16815
:103AC800FFF766FF21482169FFF762FF2048616917
:103AD800FFF75EFF1F48A169FFF75AFF1E48E1691B
:103AE800FFF756FF1D48FFF753FF1D482946FFF70C
:103AF8004FFF1C4CE16A1C48FFF74AFF216B1B482B
:103B0800FFF746FFE16B1A48FFF742FF15F0800FF9
:103B180003D018483946FFF73BFF15F4004F03D090
:103B280015483146FFF734FF1448FFF731FF1448B2
:103B38000699FFF72DFFF8BDBC840008CC84000867
:103B4800DC840008EC840008FC8400080C8500086C
:103B58001C8500082C8500083C8500084C85000859
:103B68005885000800ED00E06885000878850008A1
:103B78008885000898850008A8850008B885000889
:103B8800C085000883691A888A4207D10268033A07
:103B9800012A05D80233836101207047002070474D
:103BA8000020704710B40F4AD2F8883043F47003ED
:103BB800C2F888300C4B196841F0010119600020E7
:103BC80098601C68094921401960094959601968B9
:103BD80021F480211960D8604FF0006393605DF88C
:103BE800044B704700ED00E000380240FFFFF6FE8E
:103BF80010300024224B9B6803F00C03042B07D0E1
:103C0800082B09D0002B2DD11E4A1F4B1A602CE01F
:103C18001E4A1D4B1A6028E0194B5A685B6803F06E
:103C28003F0312F4800F09D0184AB2FBF3F2144B89
:103C38005B68C3F3881303FB02F208E0114AB2FB86
:103C4800F3F30F4A5168C1F3881101FB03F20C4BDF
:103C58005B68C3F3014301335B00B2FBF3F30A4A29
:103C6800136002E0074A084B1A60054B9B68C3F3D0
:103C78000313074AD15C044A1368CB4013607047AA
:103C8800003802400024F4000C00002080BA8C01A7
:103C98000486000810B582B0BDF81040009400F00A
:103CA80025FA02B010BD00BF00B583B0064BB3F9CA
:103CB8000020064BB3F9003000900020014600F0C8
:103CC80015FA03B05DF804FBBC200020C2200020D8
:103CD8002DE9F04385B090461E46BDF93070BDF819
:103CE800345080B21FFA83F989B2BCB200EB0902E2
:103CF800013A0B19013B92B29BB200F0CFF9204B6D
:103D0800186899880122FDF75BFA1E4B1868998894
:103D18000022FDF755FA4FF6FF739D4220D119FB9B
:103D280004F2520092B218484146FFF739FC164B8C
:103D380093F85D30012BFAD118E023B238F813302C
:103D480003EA0502120A8DF804202B408DF805308D
:103D58000D4801A90222FFF723FC0134A4B200E0B8
:103D6800002423B207FB06F29342E6DB054B1868F2
:103D780099880122FDF724FA05B0BDE8F08300BF59
:103D8800448600084C8600081420002070B50646BA
:103D9800104B186899880022FDF712FA0E4B186824
:103DA80099880022FDF70CFA0C4B1D689C88284660
:103DB80021460022FDF704FA09490E80094801222C
:103DC8001346FFF70FFB284621460122FDF7F8F9B5
:103DD80070BD00BF448600083C8600084C86000879
:103DE800602100201420002070B50646104B18688A
:103DF80099880122FDF7E4F90E4B1868998800228A
:103E0800FDF7DEF90C4B1D689C88284621460022E8
:103E1800FDF7D6F909490E80094801221346FFF734
:103E2800E1FA284621460122FDF7CAF970BD00BF14
:103E3800448600083C8600084C8600086021002063
:103E48001420002038B5934B1D689C8828462146CD
:103E58000122FDF7B5F9052000F0A6FB284621460A
:103E68000022FDF7ADF9142000F09EFB28462146FC
:103E78000122FDF7A5F9962000F096FB864B1868FD
:103E880099880022FDF79CF9EF20FFF77FFF0320B8
:103E9800FFF7AAFF8020FFF7A7FF0220FFF7A4FF84
:103EA800CF20FFF773FF0020FFF79EFFC120FFF729
:103EB8009BFF3020FFF798FFED20FFF767FF642096
:103EC800FFF792FF0320FFF78FFF1220FFF78CFF09
:103ED8008120FFF789FFE820FFF758FF8520FFF7CB
:103EE80083FF0020FFF780FF7820FFF77DFFCB20BE
:103EF800FFF74CFF3920FFF777FF2C20FFF774FFFF
:103F08000020FFF771FF3420FFF76EFF0220FFF754
:103F18006BFFF720FFF73AFF2020FFF765FFEA2045
:103F2800FFF734FF0020FFF75FFF0020FFF75CFF7B
:103F3800C020FFF72BFF2320FFF756FFC120FFF714
:103F480025FF1020FFF750FFC520FFF71FFF3E2079
:103F5800FFF74AFF2820FFF747FFC720FFF716FFA4
:103F68008620FFF741FF3620FFF710FF4820FFF7B4
:103F78003BFF3A20FFF70AFF5520FFF735FFB12036
:103F8800FFF704FF0020FFF72FFF1820FFF72CFF93
:103F9800B620FFF7FBFE0820FFF726FF8220FFF779
:103FA80023FF2720FFF720FFF220FFF7EFFE002076
:103FB800FFF71AFF2620FFF7E9FE0120FFF714FF9D
:103FC800E020FFF7E3FE0F20FFF70EFF3120FFF799
:103FD8000BFF2B20FFF708FF0C20FFF705FF0E2033
:103FE800FFF702FF0820FFF7FFFE4E20FFF7FCFE59
:103FF800F120FFF7F9FE3720FFF7F6FE0720FFF75D
:10400800F3FE1020FFF7F0FE0320FFF7EDFE0E2071
:10401800FFF7EAFE0920FFF7E7FE0020FFF7E4FEBE
:10402800E120FFF7B3FE0020FFF7DEFE0E20FFF7CA
:10403800DBFE1420FFF7D8FE0320FFF7D5FE112082
:10404800FFF7D2FE0720FFF7CFFE3120FFF7CCFEA7
:10405800C120FFF7C9FE4820FFF7C6FE0820FFF77A
:10406800C3FE0F20FFF7C0FE0C20FFF7BDFE312076
:10407800FFF7BAFE3620FFF7B7FE0F20FFF7B4FEB2
:104088001120FFF783FE782000F08EFA2920FFF731
:104098007DFE38BD1C8600084C860008F8B507462A
:1040A8000D4616461C462A20FFF770FE380AFFF711
:1040B8009BFEF8B2FFF798FE300AFFF795FEF0B2C4
:1040C800FFF792FE2B20FFF761FE280AFFF78CFE10
:1040D8002846FFF789FE200AFFF786FE2046FFF7ED
:1040E80083FE2C20FFF752FEF8BD00BF2DE9F04FEC
:1040F80083B000AF14461E463D8EC7F804D0634B0C
:104108001B881AB2904280F2BB80614A12880FFA6B
:1041180082FE714580F2B48000EB040E0EF1FF3E82
:104128000FFA83FCE64501DB1B1A1CB28B19013B15
:104138000FFA82FE734501DB521A16B280B289B2B9
:104148000219013A8B19013B92B29BB2FFF7A6FF05
:10415800504B186899880122FDF732F84E4B1A68BF
:104168003A60B3F804B0104659460022FDF728F823
:1041780004FB06F44FEA440909F1070323F0070397
:10418800ADEB030D6C464B4604E02A0AE2545A1C78
:10419800A554023B002BF8D14B460DE0E25CB2EB94
:1041A800152F04D15A1CA15CEAB2914203D03B49B5
:1041B8000A6801320A60023B002BEFD1384BA3FB9F
:1041C8000923DB0B9EB209EB030A1FFA8AFA4FF0A8
:1041D800000823E0E25CB2EB152F04D15A1CA15C65
:1041E800EAB2914203D02D490A6801320A60023BC3
:1041F80000E04B46002BEDD12A48FFF7AFFA012823
:10420800FAD1284804EB08014FF6FF72FFF7C8F906
:10421800013EB6B208F57F4808F1FF08002EE8D144
:10422800BAF1000F24D01F4B93F85D30012BFAD15F
:1042380010E014F80930B3EB152F05D109F101038B
:10424800E25CEBB29A4203D0144A1368013313605C
:10425800A9F10209B9F1000FEBD1124804EB0801EA
:104268005246FFF79DF90F4B93F85D30012BFAD1B9
:10427800386859460122FCF7A3FFD7F804D001E0BB
:10428800D7F804D00C37BD46BDE8F08FBC2000201D
:10429800C2200020448600084C860008D81D002053
:1042A800018000801420002010B504463620FFF756
:1042B8006DFD04F0030003282ED8DFE800F0020D9E
:1042C80018234820FFF790FDF022144B1A804FF472
:1042D800A072134B1A8010BD2820FFF785FD4FF4FC
:1042E800A0720E4B1A80F0220D4B1A8010BD882048
:1042F800FFF77AFDF022094B1A804FF4A072084BA1
:104308001A8010BDE820FFF76FFD4FF4A072034B31
:104318001A80F022024B1A8010BD00BFBC2000207A
:10432800C220002080B586B000AF0E4A0D4B1B6B33
:1043380043F0010313634FF480737B600123BB6078
:1043480002233B610123FB603B1D07481946FCF72C
:10435800A3FD05484FF480710022FCF731FF1837A0
:10436800BD4680BD00380240000002400A4B1B6871
:104378000A4AA2FB03239B09013BB3F1807F09D2C0
:10438800074A5360F021074B83F8231000239360FA
:1043980007231360704700BF0C000020D34D621044
:1043A80010E000E000ED00E0034B1B681BB1024A7F
:1043B8001368013B136070477821002030B595B031
:1043C80000240194234B1A6C42F080521A641B6C2F
:1043D80003F080530193019B02941F4B1A6842F427
:1043E80040421A601B6803F440430293029B012376
:1043F80008934FF4803309934FF480030F931A23E3
:1044080010934FF4D8731193022512950823139330
:104418000E9508A8FDF78EFBFDF74AFB0F230393C3
:10442800049505944FF4A05306934FF480530793D3
:1044380003A80621FDF73EFEFEF726F8074BA3FB6F
:1044480000308009FCF7A0F90420FCF7B3F915B097
:1044580030BD00BF0038024000700040D34D6210EC
:1044680010B5BFF34F8FBFF36F8F1D4B0021C3F8FB
:1044780050125A6942F400325A61BFF34F8FBFF3AA
:104488006F8FC3F88410BFF34F8FD3F88040C4F305
:104498004E3000E01846C4F3C90200E01A4643F65D
:1044A800E07303EA401343EA82730D49C1F86032AE
:1044B800531E002AF2D1431E0028EBD1BFF34F8FC1
:1044C8004B6943F480334B61BFF34F8FBFF36F8F5A
:1044D800FBF7D2FFFFF772FFFFF78CFB10BD00BFA1
:1044E80000ED00E008B519486421FCF779F8184890
:1044F8006421FCF775F817486421FCF771F818BBBC
:104508001248FCF7CDF810F4007F1DD01048FCF7D6
:10451800C7F810F4007F17D00E48FCF7C1F810F464
:10452800007F11D00948FCF7B7F880B20A4B188011
:104538000748FCF7B1F880B2084B18800548FCF72B
:10454800ABF880B2064B188008BD00BF281F0020BA
:10455800701F002004210020A01E0020B81F00208A
:104568007A20002008B50C48FBF7A0FF18B10B4AC9
:104578001378013313700A48FBF798FF18B1074AFC
:104588001378013313700748FBF790FF18B1034AFB
:1045980013780133137008BD281F00200C20002059
:1045A800701F002004210020034B1860024B1B6879
:1045B800002BFBD1704700BFBC1F00202DE9F04F36
:1045C80087B0802301934FF00208CDF810800125B1
:1045D8000295002405940394B84801A9FCF75CFCF3
:1045E8004FF0400ACDF804A0CDF81080029505944C
:1045F8000394B24801A9FCF74FFC4FF40053019310
:1046080004941127029705940394AD4801A9FCF777
:1046180043FCAB484FF400512246FCF7D1FD01950D
:10462800CDF81080029403950594A64801A9FCF7DB
:1046380033FCCDF80480CDF81080029403950594DE
:10464800A04801A9FCF728FC4FF400730193CDF8AA
:104658001080029403950594984801A9FCF71CFC66
:104668004FF0040BCDF804B04FF00309CDF80890D3
:10467800039495480DEB0B01FCF70EFC08260196F8
:10468800CDF80890039490480DEB0B01FCF704FC5F
:1046980030230193CDF8089003948B480DEB0B0160
:1046A800FCF7FAFBCDF804B0029504940394834810
:1046B8000DEB0B01FCF7F0FB804859462A46FCF746
:1046C8007FFD802301930295049403947E480DEBAB
:1046D8000B01FCF7E1FB7C4880212246FCF770FDCA
:1046E800CDF8048002950494039475480DEB0B01F2
:1046F800FCF7D2FB724841462246FCF761FDCDF833
:1047080004A00295049403946F480DEB0B01FCF789
:10471800C3FB6D4851462A46FCF752FD01950295A8
:104728000494039468480DEB0B01FCF7B5FB66484D
:1047380029462246FCF744FDCDF804A002950494CE
:10474800039460480DEB0B01FCF7A6FB5D4851464E
:104758002A46FCF735FD01960297049403945948BC
:104768000DEB0B01FCF798FB564831462246FCF747
:1047780027FD4FF4004301930295049403944F4896
:104788000DEB0B01FCF788FB4C484FF400412A461F
:10479800FCF716FD4FF4005301930295049403941B
:1047A80046480DEB0B01FCF777FB44484FF40051EA
:1047B8002A46FCF705FD20230193029504940394EF
:1047C80040480DEB0B01FCF767FB3E4820212A46C9
:1047D800FCF7F6FC102701970295049403943948D6
:1047E8000DEB0B01FCF758FB364839462A46FCF717
:1047F800E7FC4FF40067019702950494039433484B
:104808000DEB0B01FCF748FB304839462A46FCF70C
:10481800D7FC4FF4804701970295049403942948E4
:104828000DEB0B01FCF738FB264839462A46FCF706
:10483800C7FC4FF480530193CDF808900494039477
:1048480022480DEB0B01FCF727FB20484FF4805161
:104858002246FCF7B5FCCDF80480CDF80890049406
:10486800039416480DEB0B01FCF716FB4FF4806818
:10487800CDF8048002950494039414480DEB0B01C1
:10488800FCF70AFB114841462A46FCF799FC0197B8
:104898000295049403940D480DEB0B01FCF7FCFA08
:1048A8000A4839462A46FCF78BFC202301930294D8
:1048B8000494039505480DEB0B0109E00004024040
:1048C800000802400010024000000240000C0240B4
:1048D800FCF7E2FACDF804A002940494039560482A
:1048E8000DEB0B01FCF7D8FA01960294049403959A
:1048F8005B480DEB0B01FCF7CFFA80230193029480
:104908000494039556480DEB0B01FCF7C5FA4FF4D8
:104918000053019302950494039452480DEB0B0144
:10492800FCF7BAFA4F484FF400512246FCF748FC0E
:104938004FF48079CDF804900494029503954A4881
:104948000DEB0B01FCF7A8FA474849462246FCF74D
:1049580037FC4FF4004301930494029503944148B3
:104968000DEB0B01FCF798FA3E484FF400412A463C
:10497800FCF726FC8023019304940294039439489D
:104988000DEB0B01FCF788FACDF804B004940295FE
:10499800039436480DEB0B01FCF77EFA3348594671
:1049A8002A46FCF70DFCCDF8048004940295039484
:1049B8002C480DEB0B01FCF76FFA2A4841462A46B2
:1049C800FCF7FEFBCDF80490049402950394244868
:1049D8000DEB0B01FCF760FA214849462246FCF72B
:1049E800EFFB019604940295039420480DEB0B010C
:1049F800FCF752FA1D4831462246FCF7E1FBCDF898
:104A0800049004940295039416480DEB0B01FCF7EF
:104A180043FA144831462246FCF7D2FBCDF804B0DD
:104A28000494029503940F480DEB0B01FCF734FA3C
:104A38000C4859462246FCF7C3FBCDF80490049471
:104A4800029503940A480DEB0B01FCF725FA084878
:104A580049462A46FCF7B4FB07B0BDE8F08F00BF13
:104A6800000C024000100240000002400008024012
:104A780000040240F0B587B00E4B9A8801920227D5
:104A880004971226029601250395042405941868B4
:104A98000DEB0401FCF700FA074B9A880192049782
:104AA80002960395059418680DEB0401FCF7F4F9D8
:104AB80007B0F0BD648600082C86000800B585B0F4
:104AC8008DF80C008DF80D10642300930448E02144
:104AD80003AA0223FCF7ECFD05B05DF804FB00BF58
:104AE80080200020F8B51D4603FB0121CC01B4FB52
:104AF800F3F4A4F50074D201B2FBF3F703FB172714
:104B0800C6B23046E1B2FFF7D9FF701CC0B2C4F399
:104B18000721FFF7D3FFB01CC4F3014101EB870164
:104B2800C0B2C9B2FFF7CAFFF01CC0B2C7F3871101
:104B3800FFF7C4FF301DC0B2C7F38731FFF7BEFFD0
:104B4800701DC0B2C7F38751FFF7B8FFB01DC0B2E0
:104B5800E9B2FFF7B3FFF01DC0B2C5F30721FFF7B5
:104B6800ADFF06F10800C0B2C5F30741FFF7A6FF85
:104B780006F10900C0B2C5F30561FFF79FFFF8BD54
:104B880030B587B08DF80F0000238DF817300B4C27
:104B9800642500952046E0210DF10F020123FCF762
:104BA80087FD00952046E0210DF117020123FCF74F
:104BB8002BFE9DF8170007B030BD00BF80200020F5
:104BC80070B50E4900EB40028B188D5C5E789C78BE
:104BD80094B10146FF2C04D128463146FFF76EFFF9
:104BE80070BD2846FFF7CCFF20EA0400C1B234406C
:104BF80028462143FFF762FF70BD00BF1800002060
:104C080010B5E6201021FFF759FFF120E521FFF745
:104C180055FF002403E02046FFF7D2FF0134B4F526
:104C2800AF7FF8DBDA200121FFF7AAFF00F00400CC
:104C3800C0B206E0DA200121FFF7A2FF00F004006D
:104C4800C0B20028F6D131200121FFF799FF00F00A
:104C58007F013120FFF732FFF6200221FFF72EFFF8
:104C6800F1206521FFF72AFFDA200121FFF788FFED
:104C780000F0150005E0DA200121FFF781FF00F0C0
:104C880015000028F7D1EB200121FFF779FF014635
:104C98002D20FFF713FFEC200121FFF771FF0146DC
:104CA8002E20FFF70BFF2F200121FFF769FF044695
:104CB800ED200121FFF764FF00F0030104F0FC047C
:104CC8002F202143FFF7FAFE31200121FFF758FF7B
:104CD80060F07F013120C9B2FFF7F0FEE620002125
:104CE800FFF7ECFE1F20C121FFF7E8FE3520C921A0
:104CF80040F2B92240F2BF23FFF7F4FE1F20C02183
:104D0800FFF7DCFE10BD00BF2DE9F0414400124B57
:104D18009C421ED9114B9C421BD8114BD3E900670A
:104D280000253046394622462B4602F09DFB804638
:104D38003046394622462B4602F096FB01E05208DF
:104D48006408084B9C42FAD8352041462346FFF7B1
:104D5800C9FEBDE8F08100BF3F4B4C008093DC14D6
:104D680010000020A086010010B4BFF34F8FBFF3DE
:104D78006F8F1B4B0021C3F850125A6942F400325E
:104D88005A61BFF34F8FBFF36F8FC3F88410BFF31F
:104D98004F8FD3F88040C4F34E3000E01846C4F378
:104DA800C90200E01A4643F6E07303EA401343EAF7
:104DB80082730B49C1F86032531E002AF2D1431E98
:104DC8000028EBD1BFF34F8F4B6943F480334B611D
:104DD800BFF34F8FBFF36F8F5DF8044B704700BF71
:104DE80000ED00E0022956DC30B4002347E0012939
:104DF80019D0022929D0002940D11418C4F500740B
:104E08009C420ADAC2F500749C4206DD224C04EB8F
:104E180083044FF07E55256030E01F4C04EB83047B
:104E2800002525602AE0934209DD14189C4206DD1E
:104E3800194C04EB83044FF07E5525601EE0164C98
:104E480004EB83040025256018E01418C4F50075E8
:104E58009D4203DAC2F500759D4203DC934208DDEA
:104E6800A34206DA0C4C04EB83044FF07E55256010
:104E780004E0094C04EB8304002525600133B3F5F5
:104E8800007FB4DB044B03F5806100220A6003F263
:104E9800FC731A6030BC704784210020F0B40024F1
:104EA80028E0E200871897ED007A224EB31893EDB8
:104EB800006A67EE066A151D054495ED007A1346EB
:104EC80004331E44D6ED007A27EE277A36EEC77AE9
:104ED800194E324482ED007A95ED007A67EE877AB2
:104EE80097ED007A26EE076A77EE867A3344C3EDAB
:104EF800007A0134FF2CD4DD002316E0002B03DAFE
:104F080000EB830200241460B3F5007F03DB00EBA1
:104F180083020024146000EB830403EB4105064A76
:104F280002EB8502126822600133B3F5007FE5DBEE
:104F3800F0BC7047842100203452002088B0002241
:104F48000092294B196B41F001011963196B01F0AB
:104F58000101009100990192196B41F00201196356
:104F6800196B01F00201019101990292196B41F04C
:104F780004011963196B01F004010291029903926B
:104F8800196B41F008011963196B01F008010391CD
:104F980003990492196B41F010011963196B01F020
:104FA8001001049104990592196B41F400111963D9
:104FB800196B01F40011059105990692196B41F4DA
:104FC80080011963196B01F4800106910699079213
:104FD8001A6C42F480021A641B6C03F48003079372
:104FE800079B08B0704700BF0038024038B5054637
:104FF800144C154B23604FF0C06363604023A360DB
:105008000023E3604FF4806222616361A361E3617E
:105018004FF40032226263620323A3624FF4000359
:10502800E3624FF4001323632046FBF705FD6C652C
:10503800A5630F2004210A46FBF752FB3B20FBF730
:105048008FFB38BDF81D002058640240024A1368DF
:1050580001331360704700BFF41D00200023064A87
:105068001360064A13607F21054A1160054A1360E0
:105078006422054B1A607047842900208021002093
:10508800AC39002088290020585E00202F4B1B785F
:10509800002B5AD110B52E4B18689988FCF77EF86A
:1050A80044002C4B18689988FCF778F820442A4B60
:1050B80018602A4B1B68984242D00BB9012813D0BC
:1050C800012B01D1032808D0032B01D1022806D0D7
:1050D800022B06D138B1002006E0184604E0012072
:1050E80002E0002000E001201D4B18601D4B1868ED
:1050F8009988FCF753F8B8B9194B1B6823B11A4AB9
:1051080013880133138003E0174A1388013B138087
:10511800154B1B885B08154A1188B3FBF1F201FB9C
:105128001233134A13800BE00D4B1B6823B1114A4D
:1051380013680133136003E00E4A1368013B1360E0
:10514800054B1A68054B1A6010BD70476E1E00208B
:105158001486000834860008802100208429002055
:10516800B851002024860008E81D0020C21C002039
:10517800701E00205C5E002008B50B49D1E90023B1
:10518800013243F10003C1E90023FFF70DF9FFF7EE
:105198007DFFFBF77DF9054B1B681BB1034A1368BC
:1051A800013B136008BD00BFE01D0020BC1F0020AC
:1051B800002308E000EB83010B4A02EB830212682C
:1051C8000A6001339BB2094A1288B3EB420FF1DB44
:1051D80005E000EB83020021116001339BB2B3F5B7
:1051E800007FF6D3704700BF385A0020D21C002039
:1051F80008B59FED147A002308E000EB8302D2ED96
:10520800007A67EEA77A37EE277A01338B42F4DB10
:1052180007EE901AB8EEE70A87EE007AB5EEC07A84
:10522800F1EE10FA0BDBB1EEC70AB4EE400AF1EE6C
:1052380010FA06D0B0EE470A01F032FC08BD9FED27
:10524800010A08BD0000000010B4002304E001EBCF
:105258008302002414600133B3F5007FF7DBC30039
:10526800C818034A026042605DF8044B704700BFEB
:105278006666663F904B1B7813F0FF0F00F01A81AB
:1052880010B586B08D4B1B68012B74D18C4B1868F8
:1052980000283DD101A84FF480710022012301F0BC
:1052A800EBFA01A8874901F0C7FA874B1B6893B945
:1052B800864B1B78012B0AD10DE09A0081491144D5
:1052C800096883480244116001339BB200E000235F
:1052D800B3F5007FF1D37B487E4B1968FFF7DEFDFD
:1052E800794B1B68012B16D1784B1B78012B0AD1FF
:1052F80011E09A0073491144096875480244116025
:1053080001339BB200E00023B3F5007FF1D302E044
:105318006C49FFF799FF01A84FF4807101221346E9
:1053280001F0AAFA01A8674901F086FA6A4B1B78CE
:10533800022B14D1634869494FF4807201F0F6FAE0
:1053480000230AE0654A02EB830211685D4A02EB1A
:10535800C3000160416001339BB2FF2BF2D9594869
:105368004FF40071FFF744FF5D4B83ED000A002204
:10537800524B1A6096E05B4B1B68012B47D1504B90
:10538800186888B901A84FF480710022012301F040
:1053980073FA554C01A8214601F04EFA20464D4BB0
:1053A8001968FFF77BFD02E04F49FFF74DFF01A8A1
:1053B8004FF480710122134601F05EFA01A84A49B0
:1053C80001F03AFA444B1B78022B14D14648434962
:1053D8004FF4807201F0AAFA00230AE03F4A02EB78
:1053E80083021168404A02EBC30001604160013347
:1053F8009BB2FF2BF2D93C484FF40071FFF7F8FE3F
:10540800374B83ED000A0022364B1A604AE0374BCF
:105418001B68012B46D12A4B186888B901A84FF49C
:1054280080710022012301F027FA314C01A821469E
:1054380001F002FA2046274B1968FFF72FFD02E01A
:105448002B49FFF701FF01A84FF480710122134691
:1054580001F012FA01A8264901F0EEF91E4B1B785B
:10546800022B14D122481D494FF4807201F05EFAD4
:1054780000230AE0194A02EB830211681C4A02EB76
:10548800C3000160416001339BB2FF2BF2D9184879
:105498004FF40071FFF7ACFE114B83ED000A0022B8
:1054A800124B1A600022044B1A700122114B1A6029
:1054B80006B010BD704700BF0D200020501E002010
:1054C800841E0020B84100205C1E0020DC1D002046
:1054D800B43900207C1E0020601E0020B84900203E
:1054E800641E0020EC1D00208C290020881E00204E
:1054F800AC310020681E002000B583B02E380B2880
:1055080075D8DFE800F006746A101A242E38424C69
:10551800566013200090019308B211B2394A0F2344
:10552800FEF7D6FB6BE013200090019308B211B28E
:10553800354A0F23FEF7CCFB61E01320009001935E
:1055480008B211B2314A0F23FEF7C2FB57E013200D
:105558000090019308B211B22D4A0F23FEF7B8FB51
:105568004DE013200090019308B211B2294A0F238D
:10557800FEF7AEFB43E013200090019308B211B28E
:10558800254A0F23FEF7A4FB39E01320009001936E
:1055980008B211B2214A0F23FEF79AFB2FE013201D
:1055A8000090019308B211B21D4A0F23FEF790FB39
:1055B80025E013200090019308B211B2194A0F2375
:1055C800FEF786FB1BE013200090019308B211B28E
:1055D800154A0F23FEF77CFB11E01320009001937E
:1055E80008B211B2114A0F23FEF772FB07E000233D
:1055F800009308B211B20F221323FEF74BFB03B03E
:105608005DF804FB4C18002010160020E40A002066
:10561800A808002098110020881A002030040020D3
:105628005C0F0020D4130020200D00206C06002001
:1056380008B50248FBF756FB08BD00BFF81D00205F
:1056480008B50248FEF796F808BD00BFC82000203C
:1056580008B5FFF70FFE0248FEF78CF808BD00BF3B
:10566800C01F002000B583B000230193234B1A6CA0
:1056780042F000521A641B6C03F000530193019B23
:105688001F48204B0360FBF7B5F808B1FFF7DEFCB5
:105698001D4900220A604A601948FBF711F908B150
:1056A800FFF7D4FC164818491022FBF709F908B18E
:1056B800FFF7CCFC124800210A468823FBF752F971
:1056C80008B1FFF7C3FC0E48102100228823FBF71E
:1056D80049F908B1FFF7BAFC09480021FBF7ACF813
:1056E80008B1FFF7B3FC06481021FBF7A5F808B18D
:1056F800FFF7ACFC03B05DF804FB00BF00380240C4
:105708001C520020007400408C1E002030B5A3B04D
:10571800FFF72AFBFAF7B0FEFFF710FCFEF74EFF83
:1057280000F01CFC3148FFF761FC4FF40043019383
:1057380000251B9501A8FCF7C1FE2D4C2D4B2360BD
:105748002046FBF783FF0123E3602561E5612562BD
:1057580040F20F33A360FE236361274B636020464A
:10576800FBF7BCFE10B12548FEF734F9012005E02F
:105778001F48E02164221346FCF7F2F80028F7D10D
:10578800FFF73EFA1E4B1868FFF7BEFAFEF7EEFD6C
:10579800FEF7C8FD1B484FF400510122FBF710FD2E
:1057A800194BB3F90020194BB3F90000801A184BB4
:1057B8001978FFF717FBFFF755FFFFF74FFCFEF7C8
:1057C80041FB0120FEF770FD332000210A464FF609
:1057D800FF73FFF791FE0020FEF766FA0020FEF740
:1057E80063FA1F20FEF760FAF8E700BF14200020D4
:1057F8008020002000580040322791408086000811
:10580800D41C002000100240801E0020D01C002064
:10581800601E002008B5C0F30B03034800210A46A8
:10582800FBF7A0F808BD00BF1C52002008B5C0F364
:105838000B03034810210022FBF794F808BD00BFB2
:105848001C52002000000000914B1B78002B00F038
:1058580049832DE9F0418F4B1B88642B05D18E4875
:105868004FF400510122FBF7ABFCFEF73BFE8B4BDC
:105878001B68012B00F0E080022B00F0E881002B70
:1058880040F0E982864B1B683BBB824B1D886E004B
:10589800844B1B889BB2844A1068181A01F01CFBC1
:1058A8000022824B01F07EFB814C04EBC50501F020
:1058B8008BFD2860751C7F4B1B889BB27E4A106845
:1058C800181A01F009FB0022784B01F06BFB04EB7E
:1058D800850401F079FD206026E06E4B1D886E007E
:1058E800DFF8DC81B8F8000080B2744B1F68C01B79
:1058F80001F0F2FA00226D4B01F054FB6C4C04EB02
:10590800C50501F061FD2860751CB8F8000080B27B
:10591800C01B01F0E1FA0022644B01F043FB04EBE9
:10592800850401F051FD2060654B1B889BB2654AD8
:105938001288934203D9624B1A88624B1A805D4BD6
:105948001B889BB25F4A1288934203D9594B1A8825
:105958005C4B1A804F4B198848005B4A02EBC10226
:10596800D2ED007A594B93ED007AF4EEC77AF1EE56
:1059780010FA01DDC3ED007A534B03EB8003D3ED3E
:10598800016A524B93ED007AF4EEC76AF1EE10FA11
:1059980001DDC3ED006ADFED4E5A67EEA57A4D4B87
:1059A80093ED007A67EE877A9FED4B6A77EE867AF9
:1059B800FDEEE77A17EE900A484BC3ED007A66EEE3
:1059C800A56A27EE267A37EE067AFDEEC77A17EE35
:1059D800903A434AC2ED007A314A1268012A0BD143
:1059E800404A1268904201DD3E4A10603D4A126802
:1059F800934201DD3B4A136080B2FFF70BFF384B3F
:105A08001888FFF713FF234B1A88374B1B88C3F1FD
:105A1800FF018A42C0F21F82A3F580731344244811
:105A280000EBC2010D68314901EBC304256000EBAE
:105A3800C202526862600EE2194B1B68002B57D1F4
:105A4800144B1D886E00174B1B889BB2164A1068B2
:105A5800181A01F041FA0022144B01F0A3FA1A4C6B
:105A680004EBC50501F0B0FC2860751C114B1B88C0
:105A78009BB2114A1068181A01F02EFA00220B4B3B
:105A880001F090FA04EB850401F09EFC206056E0DA
:105A98007D200020C420002000100240F01D0020BE
:105AA8005C1E00207A200020CC1C00200000303F23
:105AB800B8410020B81F0020C81C0020C41C0020CA
:105AC800A01E00206C1E00208C290020781E0020BB
:105AD80000008045D81C002000000045541E00200E
:105AE800581E0020741E0020D21C0020385A0020A6
:105AF8006D4B1D886E00DFF8C081B8F8000080B2D9
:105B08006A4B1F68C01B01F0E7F90022684B01F0DF
:105B180049FA684C04EBC50501F056FC2860751C71
:105B2800B8F8000080B2C01B01F0D6F90022604B23
:105B380001F038FA04EB850401F046FC20605E4B66
:105B48001B889BB25D4A1288934203D95A4B1A8824
:105B58005A4B1A805A4B1B889BB2584A1288934258
:105B680003D9574B1A88554B1A804F4B1988480050
:105B7800544A02EBC102D2ED007A534B93ED007AFE
:105B8800F4EEC77AF1EE10FA01DDC3ED007A4D4B61
:105B980003EB8003D3ED016A4B4B93ED007AF4EEEF
:105BA800C76AF1EE10FA01DDC3ED006ADFED475A6E
:105BB80067EEA57A464B93ED007A67EE877A9FEDFC
:105BC800456A77EE867AFDEEE77A17EE900A424B41
:105BD800C3ED007A66EEA56A27EE267A37EE067AD6
:105BE800FDEEC77A17EE903A3C4AC2ED007A3C4A7D
:105BF8001268012A0BD13B4A1268904201DD394AEA
:105C08001060384A1268934201DD364A136080B248
:105C1800FFF700FE314B1888FFF708FE224B1A8861
:105C2800314B1B88C3F1FF018A42C0F21481A3F5EE
:105C3800807313441F4800EBC2010D682B4901EB28
:105C4800C304256000EBC2025268626003E1244B82
:105C58001B68002B52D1144B1D886E00244B1B88E7
:105C68009BB2244A1068181A01F036F90022104B2A
:105C780001F098F9134C04EBC50501F0A5FB286069
:105C8800751C0F4B1B889BB21B4A1068181A01F031
:105C980023F90022064B01F085F904EB850401F095
:105CA80093FB206051E000BFC4200020C41C0020EA
:105CB8000000303F8C290020A01E00206C1E002010
:105CC800B81F0020AC310020781E0020000080455D
:105CD800D81C002000000045541E0020581E00203B
:105CE8005C1E0020741E0020D21C0020385A0020A0
:105CF8007A200020CC1C0020C81C00207C4B1D886A
:105D08006E00DFF8FC81B8F8000080B2794B1F689C
:105D1800C01B01F0E1F80022774B01F043F9774C02
:105D280004EBC50501F050FB2860751CB8F80000AD
:105D380080B2C01B01F0D0F800226F4B01F032F99D
:105D480004EB850401F040FB20606D4B1B889BB27F
:105D58006C4A1288934203D9694B1A88694B1A8096
:105D6800694B1B889BB2674A1288934203D9664BDA
:105D78001A88644B1A805E4B19884800634A02EB04
:105D8800C102D2ED007A624B93ED007AF4EEC77A45
:105D9800F1EE10FA01DDC3ED007A5C4B03EB8003F2
:105DA800D3ED016A5A4B93ED007AF4EEC76AF1EE2F
:105DB80010FA01DDC3ED006ADFED565A67EEA57AE9
:105DC800554B93ED007A67EE877A9FED546A77EE2C
:105DD800867AFDEEE77A17EE900A514BC3ED007A0A
:105DE80066EEA56A27EE267A37EE067AFDEEC77AC2
:105DF80017EE903A4B4AC2ED007A4B4A1268012AD4
:105E08000BD14A4A1268904201DD484A1060474A5D
:105E18001268934201DD454A136080B2FFF7FAFC2D
:105E2800404B1888FFF702FD314B1A88404B1B88FE
:105E3800C3F1FF018A420EDBA3F5807313442F4898
:105E480000EBC2010D683B4901EBC304256000EB80
:105E5800C202526862602E4C206801F04FF822A3FB
:105E6800D3E9002301F09EF801F0AEFA2060204A41
:105E7800138801339BB21380FF2B2FD92E484FF480
:105E880000510022FBF79CF901222C4B1A70284B79
:105E98001A88174B1A802A4B1B68012B0BD0022B30
:105EA80013D0DBB90123274A1360254A136026481B
:105EB800FFF77EF912E00122244B1A600222204BE0
:105EC8001A600E48FFF774F908E00122204B1A60A7
:105ED80000221B4B1A600D48FFF76AF9FEF742FBD8
:105EE800BDE8F081704700BF1EA7E8482EFFEF3FCE
:105EF800C4200020C41C00200000303FAC3100202A
:105F0800A01E00206C1E0020B81F0020B8410020F1
:105F1800781E002000008045D81C002000000045A5
:105F2800541E0020581E00205C1E0020741E0020F5
:105F3800D21C0020385A0020001002400D200020FA
:105F4800F01D0020501E00208C290020EC1D002090
:105F5800881E002008B5FFF777FC08BD2DE9F04141
:105F680086B0002400942D4B5A6C42F480525A6437
:105F78005B6C03F480530093009B294B9A88019231
:105F8800022504950295052705970394186801A929
:105F9800FAF782FF234B9A8801920495029503949D
:105FA8000597186801A9FAF777FF1F4B9A8801929D
:105FB80004950294012603960597186801A9FAF733
:105FC8006BFF1A4B9F8801970495029603940594DA
:105FD800D3F80080404601A9FAF75EFF40463946EB
:105FE8003246FBF7EDF81248124B036084604FF419
:105FF800827343604FF4E063C360056146614FF408
:1060080000738361C4610462846244620723C362CB
:10601800FDF7BAF806B0BDE8F08100BF00380240CD
:106028003C860008548600085C8600084C860008F8
:106038001420002000300140704700BF704700BFA7
:10604800FEE700BFFEE700BFFEE700BFFEE700BFB8
:10605800FEE700BF2DE9F04F49084F1C00242646F3
:1060680062E0A6423FD24FEAC50C00EB0C09D9F812
:1060780000A04FEAC40E00EB0E08D8F800B0C9F82B
:1060880000B0C8F800A00CF1040C8444DCF80080CF
:106098000EF1040E8644DEF80090CCF80090CEF89D
:1060A800008006EB070C4FEACC0C00EB0C09D9F882
:1060B80000A007EB040E4FEACE0E00EB0E08D8F84E
:1060C80000B0C9F800B0C8F800A00CF1040C844472
:1060D800DCF800800EF1040E8644DEF80090CCF85F
:1060E8000090CEF800800135ED0000EB050CDCF8DF
:1060F80000800C44E40000EB040EDEF80090CCF8BD
:106108000090CEF8008004350544D5F800E004344A
:106118000444D4F800C0C5F800C0C4F800E01C88E6
:1061280003EB42030236B6B23546A1F1020E7645BC
:1061380097D9BDE8F08F00BF2DE9F04F2DED048B06
:1061480087B00491029203934FEA9109CDF8009029
:106158004FF00008C2460591CB46154608EB0B02E6
:1061680002EB0B0303EB0B014FEAC80400EB040935
:10617800D9ED006A04340444D4ED004AD20000EB9F
:10618800020C9CED004A0432024492ED006ADB00E6
:1061980000EB030E9EED007A043303440193D3ED24
:1061A800005AC900471897ED005A04310144D1ED4F
:1061B800007A36EE872A74EE052A74EEA50A36EEC2
:1061C800271A4FEA0A16AB1993ED003AD3ED013AB4
:1061D80076EEC76A34EE455A74EEE55A76EE677A7B
:1061E80032EE227A89ED007A30EE817A84ED007AF7
:1061F80076EEA71A35EEC50A72EE624A30EEC12A6B
:1062080036EEE77A35EE256A4FEACA042E19D6ED3E
:10621800005A96ED014A0AEB4A04E4002E19D6ED1D
:10622800006AD6ED017A61EEA50A60EE252A24EE11
:10623800831A22EE035A67EE265A66EE266A20EE85
:10624800040A21EE844A22EE232A64EEA34A26EEAB
:10625800276A67EE277A30EE803A32EEC44A71EE4A
:10626800023A35EE645A35EE867A76EEE77ACCED68
:10627800003A82ED005A8EED003A019B83ED004A08
:1062880087ED007AC1ED007A039B9A4408F1010872
:10629800009B013B00937FF461AFD946DDF814B051
:1062A800039B9B009BB20193049B9B08049303935D
:1062B800ADE04FEA9906002300939A460AEB4A0399
:1062C8004FEACA02029C21461144D1ED008A2244B9
:1062D80092ED018A4FEA0A12A11891ED000AD1ED58
:1062E800010ADB00E21892ED001AD2ED011A019BB7
:1062F8009A44009DAA1993199919EC0000EB040817
:1063080098ED004A0434044494ED006AD20000EB8E
:10631800020CDCED005A04320244D2ED007ADB00B4
:1063280000EB030E9EED005A0433034493ED007A0C
:10633800C9004718D7ED004A04310144D1ED006A7D
:1063480034EE453A35EEE42A76EE472A77EEE63A19
:1063580034EE055A75EEA45A36EE077A77EEA67A29
:1063680073EE234A32EEC24A35EE659A77EE679AA3
:1063780073EE636A32EE226A75EE255AC8ED005A4A
:1063880077EE277AC4ED007A24EEA85A64EE285AEC
:1063980029EE003A69EE803A26EE817A66EE017AB5
:1063A80024EE084A64EE884A69EEA09A29EE209AFB
:1063B80026EE216A66EEA16A35EE044A75EEE44AD5
:1063C80073EE299A33EEC99A37EE066A77EEE66AD3
:1063D800CCED009A82ED009A8EED004AC3ED004A9A
:1063E80087ED006AC1ED006A4D44AB4582D8009B39
:1063F80001331A460093731E9342BFF45FAF019BAB
:106408009B009BB20193039B9B080393B146039B9C
:10641800042B3FF64EAF049B90ED004A90ED016AC5
:10642800D0ED026AD0ED034AD0ED045AD0ED057ADA
:1064380090ED067A90ED075A34EE253A74EE655AD7
:1064480036EE274A76EE677A76EE873A34EE856A34
:1064580036EEC77A74EEC56A33EE232A74EE062A3E
:1064680073EE633A34EE466A75EEA64A37EEC75ABB
:1064780075EEE66A77EE277A80ED002AC0ED012AEC
:10648800C0ED023A80ED036AC0ED044A80ED055A7A
:10649800C0ED066AC0ED077A2030013BBCD107B0D9
:1064A800BDEC048BBDE8F08F2DE9F04F2DED068B88
:1064B80087B00491029203934FEA9109CDF80090B6
:1064C8004FF00008C2460591CB46154608EB0B0273
:1064D80002EB0B0303EB0B014FEAC80400EB0409C2
:1064E800D9ED006A04340444D4ED004ADB0000EB23
:1064F800030E9EED007A04330344019393ED005A92
:10650800D20000EB020C9CED004A0432024492EDEA
:10651800006AC9004718D7ED005A04310144D1ED8B
:10652800007A36EE872A74EE252A74EE850A36EE4E
:10653800271A4FEA0A16AB1993ED003AD3ED013A40
:1065480076EEC76A74EE655A34EEC55A76EE677A07
:1065580032EE227A89ED007A30EE817A84ED007A83
:1065680076EEE71A35EE258A72EE624A30EEC12AD7
:1065780036EEA77A35EE656A4FEACA042E19D6EDCB
:10658800005A96ED014A0AEB4A04E4002E19D6EDAA
:10659800006AD6ED017A61EEA50A68EE252A24EE96
:1065A800831A22EE035A67EE265A66EE266A28EE0A
:1065B800048A21EE844A22EE232A64EEA34A26EEB8
:1065C800276A67EE277A30EEC83A32EE844A71EECF
:1065D800423A35EE245A35EEC67A76EEA77ACCEDF5
:1065E800003A82ED005A8EED003A019B83ED004A95
:1065F80087ED007AC1ED007A039B9A4408F10108FF
:10660800009B013B00937FF461AFD946DDF814B0DD
:10661800039B9B009BB20193049B9B0804930393E9
:10662800ADE04FEA9906002300939A460AEB4A0325
:106638004FEACA02029C2146114491ED009A224475
:10664800D2ED018A4FEA0A12A11891ED008AD1ED24
:10665800010ADB00E21892ED001AD2ED011A019B43
:106668009A44009DAA1993199919EC0000EB0408A3
:1066780098ED004A0434044494ED006AD20000EB1B
:10668800020CDCED005A04320244D2ED007ADB0041
:1066980000EB030E9EED005A0433034493ED007A99
:1066A800C9004718D7ED004A04310144D1ED006A0A
:1066B80034EE453A75EEE42A36EE472A77EEE63AA6
:1066C80034EE055A75EEA45A36EE077A77EEA67AB6
:1066D80073EE634A32EE224A75EE659A37EE67AA80
:1066E80073EE236A32EE626A75EE255AC8ED005AD7
:1066F80077EE277AC4ED007A24EE895A64EE095AB7
:1067080029EE883A6AEE083A26EE817A66EE017A30
:1067180024EE284A64EEA84A2AEE20AA69EEA09A36
:1067280026EE216A66EEA16A35EE444A75EEA44A61
:1067380033EE4AAA73EEA99A37EE466A77EEA66A4E
:106748008CED00AAC2ED009A8EED004AC3ED004A16
:1067580087ED006AC1ED006A4D44AB4582D8009BC5
:1067680001331A460093731E9342BFF45FAF019B37
:106778009B009BB20193039B9B080393B146039B29
:10678800042B3FF64EAF049B90ED004A90ED016A52
:10679800D0ED026AD0ED034AD0ED045A90ED057AA7
:1067A800D0ED067A90ED075A34EE253A74EE655A24
:1067B80036EE074A36EE477A76EEA73A34EE856A21
:1067C80076EEE77A74EEC56A33EE232A74EE062A6B
:1067D80073EE633A34EE466A75EEE64A37EE275AA8
:1067E80075EEA66A77EE677A22EE003A22EE804AC4
:1067F80063EE805A26EE006A64EE804A25EE005A5F
:1068080026EE807A67EE807A80ED003A80ED014AC4
:10681800C0ED025A80ED036AC0ED044A80ED055AC6
:1068280080ED067AC0ED077A2030013BACD107B085
:10683800BDEC068BBDE8F08F38B504460D4683786D
:10684800012B08D1084621886268A38994ED040ABF
:10685800FFF72AFE05E0084621886268A389FFF74A
:106868006BFCE378012B05D128462188E289A368CF
:10687800FFF7F0FB38BD00BF10B40180254C446021
:106888008270C370B1F5807F1FD004D8102930D032
:10689800402924D038E0B1F5806F0CD0B1F5805F85
:1068A80032D101238381C3811B4B83604FF0665330
:1068B8000361002029E004238381C381174B83608F
:1068C8004FF06A53036100201FE010238381C381C6
:1068D800134B83604FF06E530361002015E0402393
:1068E8008381C3810F4B83604FF072530361002093
:1068F8000BE04FF480738381C3810B4B83604FF0AF
:1069080076530361002000E0FF2040B25DF8044B9D
:10691800704700BF9C8E00089C860008A28600086D
:10692800BA8600081A8700089A8800082DE9F041FD
:1069380004460D461746960882E0D4ED007A94ED99
:10694800010A67EEA77A20EE000A77EE807AF5EE64
:10695800C07AF1EE10FA0DDBB1EEE70AB4EE400AA8
:10696800F1EE10FA03D0B0EE670A00F099F885ED61
:10697800000A01E000232B60D4ED027A94ED030AAB
:1069880067EEA77A20EE000A77EE807AF5EEC07AF5
:10699800F1EE10FA0DDBB1EEE70AB4EE400AF1EEC3
:1069A80010FA03D0B0EE670A00F07AF885ED010A14
:1069B80001E000236B60D4ED047A94ED050A67EEDC
:1069C800A77A20EE000A77EE807AF5EEC07AF1EE2B
:1069D80010FA0DDBB1EEE70AB4EE400AF1EE10FA58
:1069E80003D0B0EE670A00F05BF885ED020A01E01B
:1069F8000023AB60D4ED067A04F1200894ED070A71
:106A080067EEA77A20EE000A77EE807A05F1100487
:106A1800F5EEC07AF1EE10FA0DDBB1EEE70AB4EE4E
:106A2800400AF1EE10FA03D0B0EE670A00F038F829
:106A380085ED030A01E00023EB60013E254644464C
:106A4800002E7FF47AAF07F0030724E026460836C5
:106A5800D4ED007A94ED010A67EEA77A20EE000AD9
:106A680077EE807A2C1DF5EEC07AF1EE10FA0DDB88
:106A7800B1EEE70AB4EE400AF1EE10FA03D0B0EE38
:106A8800670A00F00DF885ED000A01E000232B608D
:106A9800013F25463446002FD8D1BDE8F08100BF1C
:106AA80010B52B4C2DED028B8AB0F0EE408A00F029
:106AB80053F894F90030B0EE408A01332DD0B0EE8F
:106AC800680A00F09BF840B3F5EEC08AF1EE10FAC0
:106AD80023D501211F4A002318EE900A8DE80600ED
:106AE800089300F00BFA2478CDE90401CDE90201FE
:106AF800CCB900220023CDE90623684600F07CF8D3
:106B0800D8B1089BF3B9DDE9060100F05DFC00EEA1
:106B1800100A0AB0BDEC028B10BDB0EE480A0AB0EC
:106B2800BDEC028B10BD0020002102460B4600F090
:106B380063FB022CCDE90601DFD100F045FF2123DC
:106B48000360DEE700F040FF089B0360DBE700BF5F
:106B5800DC1C00209C0E010810EE103A23F00042C5
:106B6800B2F1FF4F70B439D2B2B3002B3CDBB2F5AF
:106B7800000F4FEAE35109D213F4000239D15B0048
:106B880001321802FBD5C2F101021144A1F17F02C2
:106B9800C3F31603D10743F4000323D4002456108B
:106BA8005B00192125464FF08072A818984202DC34
:106BB8001B1A8518144401394FEA43034FEA52025D
:106BC800F3D113B104F001031C44641004F17C54A4
:106BD80004EBC65300EE103A70BC7047A0EE000AF2
:106BE80070BC70475B00D9E730EE400A80EE000ABF
:106BF800F2E701221144C9E70020704710EE103A6D
:106C080033F0004001D102207047A0F50003B3F132
:106C1800FE4F01D204207047421E054B9A4201D80C
:106C280003207047A0F1FF40B0FA80F04009704798
:106C3800FEFF7F0081F0004102E000BF83F00043C7
:106C480030B54FEA41044FEA430594EA050F08BFFF
:106C580090EA020F1FBF54EA000C55EA020C7FEAC3
:106C6800645C7FEA655C00F0E2804FEA5454D4EB40
:106C78005555B8BF6D420CDD2C4480EA020281EA0A
:106C8800030382EA000083EA010180EA020281EA42
:106C98000303362D88BF30BD11F0004F4FEA013194
:106CA8004FF4801C4CEA113102D0404261EB4101A3
:106CB80013F0004F4FEA03334CEA133302D0524229
:106CC80063EB430394EA050F00F0A780A4F10104E5
:106CD800D5F1200E0DDB02FA0EFC22FA05F280181F
:106CE80041F1000103FA0EF2801843FA05F3594105
:106CF8000EE0A5F120050EF1200E012A03FA0EFC84
:106D080028BF4CF0020C43FA05F3C01851EBE371AD
:106D180001F0004507D54FF0000EDCF1000C7EEBCA
:106D280000006EEB0101B1F5801F1BD3B1F5001F08
:106D38000CD349085FEA30004FEA3C0C04F1010427
:106D48004FEA445212F5800F80F09A80BCF1004F50
:106D580008BF5FEA500C50F1000041EB045141EAD2
:106D6800050130BD5FEA4C0C404141EB010111F4D3
:106D7800801FA4F10104E9D191F0000F04BF01467E
:106D88000020B1FA81F308BF2033A3F10B03B3F15C
:106D980020020CDA0C3208DD02F1140CC2F10C02EC
:106DA80001FA0CF021FA02F10CE002F11402D8BF4A
:106DB800C2F1200C01FA02F120FA0CFCDCBF41EA16
:106DC8000C019040E41AA2BF01EB0451294330BDE5
:106DD8006FEA04041F3C1CDA0C340EDC04F11404C2
:106DE800C4F1200220FA04F001FA02F340EA030099
:106DF80021FA04F345EA030130BDC4F10C04C4F1DF
:106E0800200220FA02F001FA04F340EA03002946BE
:106E180030BD21FA04F0294630BD94F0000F83F408
:106E2800801306BF81F480110134013D4EE77FEAEB
:106E3800645C18BF7FEA655C29D094EA050F08BF37
:106E480090EA020F05D054EA000C04BF1946104618
:106E580030BD91EA030F1EBF0021002030BD5FEA5C
:106E6800545C05D14000494128BF41F0004130BD84
:106E780014F580043CBF01F5801130BD01F00045D8
:106E880045F0FE4141F470014FF0000030BD7FEA4B
:106E9800645C1ABF194610467FEA655C1CBF0B4646
:106EA800024650EA013406BF52EA033591EA030F5D
:106EB80041F4002130BD00BF90F0000F04BF002155
:106EC800704730B54FF4806404F132044FF0000588
:106ED8004FF0000150E700BF90F0000F04BF002101
:106EE800704730B54FF4806404F1320410F0004567
:106EF80048BF40424FF000013EE700BF42004FEA62
:106F0800E2014FEA31014FEA02701FBF12F07F43DE
:106F180093F07F4F81F06051704792F0000F14BFDB
:106F280093F07F4F704730B54FF4607401F000451F
:106F380021F0004120E700BF50EA010208BF704776
:106F480030B54FF000050AE050EA010208BF70476B
:106F580030B511F0004502D5404261EB41014FF4D4
:106F6800806404F132045FEA915C3FF4DCAE4FF0D8
:106F780003025FEADC0C18BF03325FEADC0C18BFBF
:106F8800033202EBDC02C2F1200300FA03FC20FA10
:106F980002F001FA03FE40EA0E0021FA02F114445D
:106FA800C1E600BF70B54FF0FF0C4CF4E06C1CEA72
:106FB80011541DBF1CEA135594EA0C0F95EA0C0FE7
:106FC80000F0DEF82C4481EA030621EA4C5123EA5A
:106FD8004C5350EA013518BF52EA033541F4801189
:106FE80043F4801338D0A0FB02CE4FF00005E1FB3C
:106FF80002E506F00042E0FB03E54FF00006E1FB86
:1070080003569CF0000F18BF4EF0010EA4F1FF04C8
:10701800B6F5007F64F5407404D25FEA4E0E6D4108
:1070280046EB060642EAC62141EA55514FEAC52019
:1070380040EA5E504FEACE2EB4F1FD0C88BFBCF595
:10704800E06F1ED8BEF1004F08BF5FEA500E50F146
:10705800000041EB045170BD06F0004646EA01010C
:1070680040EA020081EA0301B4EB5C04C2BFD4EB3E
:107078000C0541EA045170BD41F480114FF0000E37
:10708800013C00F3AB8014F1360FDEBF002001F0A5
:10709800004170BDC4F10004203C35DA0C341BDC1F
:1070A80004F11404C4F1200500FA05F320FA04F0F1
:1070B80001FA05F240EA020001F0004221F0004125
:1070C80010EBD37021FA04F642EB06015EEA430E98
:1070D80008BF20EAD37070BDC4F10C04C4F12005C8
:1070E80000FA04F320FA05F001FA04F240EA02007B
:1070F80001F0004110EBD37041F100015EEA430E4C
:1071080008BF20EAD37070BDC4F1200500FA05F26B
:107118004EEA020E20FA04F301FA05F243EA0203EA
:1071280021FA04F001F0004121FA04F220EA0200F9
:1071380000EBD3705EEA430E08BF20EAD37070BD3F
:1071480094F0000F0FD101F00046400041EB01011F
:1071580011F4801F08BF013CF7D041EA060195F001
:10716800000F18BF704703F00046520043EB0303BB
:1071780013F4801F08BF013DF7D043EA06037047A8
:1071880094EA0C0F0CEA135518BF95EA0C0F0CD0B3
:1071980050EA410618BF52EA4306D1D181EA0301F9
:1071A80001F000414FF0000070BD50EA410606BFF3
:1071B8001046194652EA430619D094EA0C0F02D138
:1071C80050EA013613D195EA0C0F05D152EA03367D
:1071D8001CBF104619460AD181EA030101F000419B
:1071E80041F0FE4141F470014FF0000070BD41F0E4
:1071F800FE4141F4780170BD70B54FF0FF0C4CF4BE
:10720800E06C1CEA11541DBF1CEA135594EA0C0FDC
:1072180095EA0C0F00F0A7F8A4EB050481EA030E29
:1072280052EA03354FEA013100F088804FEA033310
:107238004FF0805545EA131343EA12634FEA0222DE
:1072480045EA111545EA10654FEA00260EF000419F
:107258009D4208BF964244F1FD0404F5407402D2F1
:107268005B084FEA3202B61A65EB03055B084FEA82
:1072780032024FF480104FF4002CB6EB020E75EB7F
:10728800030E22BFB61A754640EA0C005B084FEAA7
:107298003202B6EB020E75EB030E22BFB61A754624
:1072A80040EA5C005B084FEA3202B6EB020E75EB6F
:1072B800030E22BFB61A754640EA9C005B084FEAE7
:1072C8003202B6EB020E75EB030E22BFB61A7546F4
:1072D80040EADC0055EA060E18D04FEA051545EAE3
:1072E80016754FEA06164FEAC30343EA52734FEA8C
:1072F800C2025FEA1C1CC0D111F4801F0BD141EA05
:1073080000014FF000004FF0004CB6E711F4801F69
:1073180004BF01430020B4F1FD0C88BFBCF5E06F49
:107328003FF6AFAEB5EB030C04BFB6EB020C5FEA59
:10733800500C50F1000041EB045170BD0EF0004EAE
:107348004EEA113114EB5C04C2BFD4EB0C0541EAE0
:10735800045170BD41F480114FF0000E013C90E6DD
:1073680045EA060E8DE60CEA135594EA0C0F08BFA1
:1073780095EA0C0F3FF43BAF94EA0C0F0AD150EAA0
:1073880001347FF434AF95EA0C0F7FF425AF104633
:1073980019462CE795EA0C0F06D152EA03353FF45B
:1073A800FDAE1046194622E750EA410618BF52EAD8
:1073B80043067FF4C5AE50EA41047FF40DAF52EAAC
:1073C80043057FF4EBAE12E74FEA4102B2F1E04326
:1073D80024BFB3F5001CDCF1FE5C0DD901F0004CB4
:1073E8004FEAC0024CEA5070B2F1004F40EB830004
:1073F80008BF20F00100704711F0804F21D113F130
:107408003872BCBF01F00040704741F480114FEA68
:107418005252C2F11802C2F1200C10FA0CF320FAF1
:1074280002F018BF40F001004FEAC1234FEAD3230E
:1074380003FA0CFC40EA0C0023FA02F34FEA430378
:10744800CCE77FEA625307D150EA01331EBF4FF001
:10745800FE4040F44000704701F0004040F0FE401C
:1074680040F40000704700BF53B94AB9002908BF6B
:1074780000281CBF4FF0FF314FF0FF3000F03CB840
:1074880082B0EC462DE9005000F01EF8DDF804E06B
:1074980002B00CBC704700BF2DE9F041904606468B
:1074A8000F461D46069C00F029F808FB01FC86469D
:1074B800A8FB002300FB05C5B21A2B4467EB0303A6
:1074C800C4E90023BDE8F0812DE9F8431D461746BD
:1074D80080468946089E00F053F900FB05F3A0FB9F
:1074E800074507FB0137B8EB04043D4469EB050584
:1074F800C6E90045BDE8F883704700BF00292DE9BB
:10750800F047C0F2A2800026002BC0F298808C467B
:1075180090469E46154604460F46CBBB8A4256D92E
:10752800B2FA82F33BB1C3F120029F409D409C40D8
:1075380020FA02F21743280C220C1FFA85FEB7FB2B
:10754800F0F100FB11770EFB01F342EA0747BB425B
:1075580007D97F1980F00181BB4240F2FE800239D1
:107568002F44FF1AA4B2B7FBF0F300FB13770EFB0E
:1075780003FE44EA0747BE4506D97F1980F0EB8031
:10758800BE4540F2E880023B43EA0143002203E0A3
:107598008B420FD900221346341C4FF0000518BF48
:1075A8000124604265EB450158405140001969418A
:1075B800BDE8F087B3FA83F2002A40F08380804563
:1075C80040F2CD808B42C0F0CA801346E4E712B97E
:1075D8000123B3FBF2F5B5FA85F2002A3BD1781BFB
:1075E8004FEA154E1FFA85FC0122210CB0FBFEF86C
:1075F8000EFB18000CFB08F341EA0047BB4208D910
:107608007F1980F0B080BB4240F2AD80A8F102083B
:107618002F44FF1AA4B2B7FBFEF30EFB13770CFB43
:1076280003FC44EA0747BC4506D97F1980F09980D6
:10763800BC4540F29680023B43EA0843ACE752421D
:107648006FEA060663EB430361E740424FF0FF36FB
:1076580061EB410158E79540C2F1200107FA02F3B6
:107668004FEA154ECF4024FA01F194401FFA85FCE9
:107678001943B7FBFEF24FEA11480EFB12770CFBD9
:1076880002F348EA0747BB4205D97F1971D2BB42CA
:107698006FD9023A2F44FF1A89B2B7FBFEF80EFBE6
:1076A80018770CFB08F041EA0743984206D95B19A2
:1076B80061D298425FD9A8F102082B44181A48EA07
:1076C800024292E7C2F1200703FA02FE08FA02F525
:1076D800914028FA07F32CFA07FCF84043EA0E0E0B
:1076E80008434FEA1E48070C1FFA8EFABCFBF8F94C
:1076F80008FB19CC0AFB09F147EA0C4C614507D98C
:107708001CEB0E0C32D2614530D9A9F10209F444C0
:10771800C1EB0C0C80B2BCFBF8F308FB13CC0AFBE2
:1077280003FA40EA0C418A4506D911EB0E0125D22D
:107738008A4523D9023B714443EA0943CAEB010154
:10774800A3FB0589494503D303D19440444500D29E
:10775800013B002220E7013B16E7013901E701233D
:107768001AE7013B68E708F1FF3852E709F1FF39EA
:10777800CEE7013A8FE708F1FF389FE7013BDBE7E7
:107788002DE9F043002B40D18A42044615464AD9D8
:10779800B2FA82F30F464BB1C3F12006994000FAC2
:1077A80003F402FA03F5F04040EA0107290C260C1D
:1077B8001FFA85FEB7FBF1F001FB10770EFB00F214
:1077C80046EA07439A4207D95B1980F0EA809A4251
:1077D80040F2E78002382B449A1AA4B2B2FBF1F3C4
:1077E80001FB13220EFB03FE44EA0242964506D92A
:1077F800521980F0DA80964540F2D780023B43EA7E
:10780800004000263146BDE8F0838B4244D8B3FAE5
:1078180083F6002E45D1824240F2BF808B42C0F0F1
:10782800BC803046EEE712B90125B5FBF2F5B5FA92
:1078380085F2002A7BD14A1B2F0C1FFA85FE0126F0
:10784800230CB2FBF7F007FB10220EFB00FC43EA07
:1078580002418C4507D9491980F0A1808C4540F236
:107868009E8002382944CCEB0101A4B2B1FBF7F3A6
:1078780007FB13110EFB03FE44EA0144A64506D993
:10788800641980F09080A64540F28D80023B43EA5F
:1078980000403146BDE8F083002630463146BDE859
:1078A800F083C6F12005B34002FA06F701FA06F4A0
:1078B800EA40E94020FA05F51A4325434FEA124CFD
:1078C8004FEA154E93B2B1FBFCF80CFB181103FB01
:1078D80008F44EEA01418C4206D9891869D28C42D3
:1078E80067D9A8F102081144091BADB2B1FBFCF439
:1078F8000CFB141103FB04FE45EA01439E4505D920
:107908009B1854D29E4552D9023C134444EA084479
:10791800CEEB0303A4FB07894B4503D351D1B040F9
:1079280040454ED20026601E3146BDE8F083C2F1C4
:107938002006954001FA02F300FA02F42F0CF140F8
:10794800F0401FFA85FEB1FBF7F6184307FB161146
:107958000EFB06F24FEA104C4CEA01439A4205D955
:107968005B1929D29A4227D9023E2B449B1A80B22E
:10797800B3FBF7FC07FB1C330EFB0CF140EA034397
:10798800994206D95B1919D2994217D9ACF1020C60
:107998002B445A1A4CEA064652E7012032E70138CE
:1079A80061E7013818E7013B71E7013B27E7013C34
:1079B800ACE708F1FF3897E7013ED7E70CF1FF3C49
:1079C800E7E7204600261DE7014B1868704700BF0F
:1079D800401D0020034613F8012B002AFBD1181A7A
:1079E8000138704730B5141E9BB0054604DA8B2366
:1079F80003604FF0FF301CE04FF4027200910491D5
:107A08006946ADF80C2014BF04F1FF3222460292F9
:107A180005924FF6FF72ADF80E201A461E9B00F035
:107A280075F8431CBCBF8B232B6014B10022009B4C
:107A38001A701BB030BD000073B5064600930D46A2
:107A48001446044B31462A4618682346FFF7CAFFF6
:107A580002B070BD401D00202DE9F0478E688246B7
:107A68000C469046B342994640D38A8912F4906FE7
:107A78003AD02568022309696F1A656905EB45053F
:107A880095FBF3F57B1C4B449D4238BF1D465305BF
:107A98000FD5294600F038FB064698B121693A46C9
:107AA80000F0C8FAA38923F4906343F08003A3810C
:107AB80013E02A4600F07EFB064670B9504621695D
:107AC80000F0DEFA0C234FF0FF30CAF80030A3892B
:107AD80043F04003A381BDE8F08726613E44656119
:107AE800ED1B26604E46A560B14500D24E46324693
:107AF8002068414600F0A9FAA36800209B1BA360F8
:107B080023681E442660BDE8F08700002DE9F04395
:107B18009DB006460D46904603938B891C060CD5EE
:107B28000B6953B9402100F0EFFA2860286110B9B9
:107B38000C233360CCE040236B610023099320239E
:107B48008DF8293030238DF82A3043461C4613F827
:107B5800012B1AB9B4EB08090FD002E0252AF5D198
:107B6800F8E73046294642464B46FFF775FF013095
:107B780000F0A980099B4B4409932378002B00F05F
:107B8800A28000234FF0FF3204F101080493079309
:107B9800059206938DF853301A934446DFF84891BE
:107BA800052208F101084846217800F035FA049BBF
:107BB80030B1C9EB00000122824013430493ECE783
:107BC800D80644BF20228DF85320190744BF2B2222
:107BD8008DF8532022782A2A02D0079923460EE0EE
:107BE800039A0134111D1268002A0391BBBF524247
:107BF80043F0020307920792B8BF04930AE01C46B9
:107C080001332278303A092A03D80A2000FB0121DF
:107C1800F5E7079123782E2B1AD163782A2B0AD1FE
:107C2800039B02341A1D1B68002B0392B8BF4FF048
:107C3800FF3305930CE0611C00220C4601312378C8
:107C4800303B092B03D80A2000FB0232F5E70592E6
:107C5800DFF8988003222178404600F0DDF938B13A
:107C6800C8EB00004023049A013483401343049373
:107C780021780622194804F101088DF8281000F02F
:107C8800CBF988B1164B33B9039B073323F00703AD
:107C98000833039313E003AB304604A92A46009344
:107CA800104BAFF3008007E003AB304604A92A4627
:107CB80000930C4B00F092F8421C074603D0099B36
:107CC8003B44099341E7AB895B0601D4099801E07D
:107CD8004FF0FF301DB0BDE8F08300BFB00E0108C3
:107CE80000000000617A0008A60E0108AC0E010829
:107CF8002DE9F84391461F468A6806460B690C46EB
:107D0800DDF820809342B8BF1346C9F8003091F8D7
:107D1800432012B10133C9F800302368990642BFE5
:107D2800D9F800300233C9F80030256815F0060587
:107D38001CD094F843302268003318BF0123920600
:107D48001FD5E1185A1C30200233224481F8430021
:107D580094F8451082F8431013E03046394604F190
:107D680019020123C047013007D00135E368D9F86B
:107D780000209B1A9D42F0DBDBE74FF0FF30BDE8A7
:107D8800F8833046394604F14302C0470130F4D045
:107D98002268D9F800504FF0000902F00602E368A3
:107DA800042A226908BF5D1BA36814BF002525EAC1
:107DB800E5759342C4BF9B1AED18A9450ADA304607
:107DC800394604F11A020123C0470130D5D009F120
:107DD8000109F2E70020BDE8F88300002DE9FF4122
:107DE8000C46174698460646227E43310A9B6E2A61
:107DF80000F0AF8012D8632A23D00AD8002A00F0F6
:107E0800BC80582A40F0CB8084F84520DFF800E297
:107E180057E0642A1ED0692A1CD0C0E0732A00F0FB
:107E2800B08009D86F2A2ED0702A40F0B880226816
:107E380042F0200222603FE0752A24D0782A3BD005
:107E4800ADE01A6804F14205111D1960136884F841
:107E58004230A8E020681A6810F0800F02D0101D88
:107E6800186008E010F0400F02F10400186002D01A
:107E7800B2F9003000E01368002B3EDA2D225B4295
:107E880084F8432039E020681A6810F0800F02D087
:107E9800101D186007E010F0400F02F10400186090
:107EA80001D0138800E01368227EDFF864E16F2AAE
:107EB8000CBF08220A221CE07822DFF858E184F877
:107EC80045202268186812F0800F00F104051D6033
:107ED80003D1550601D5038800E00368D00744BFE5
:107EE80042F0200222601BB9226822F020022260A0
:107EF8001022002084F8430002E0DFF814E10A228F
:107F08006568002DA560A2BF206820F004002060ED
:107F180003B965B10D46B3FBF2F002FB10331EF84E
:107F2800033005F8013D03460028F4D100E00D4672
:107F3800082A0BD12368DA0708D5236962689A42B0
:107F4800DEBF302305F8013C05F1FF35491B2161EF
:107F58002EE025681A6815F0800F606903D0151D9A
:107F68001D60136808E015F0400F02F104051D605C
:107F7800136801D0188000E0186000230D462361C3
:107F880016E01A68111D19600021156862682846F4
:107F980000F042F808B1401B6060636804E004F137
:107FA800420584F8422001232361002384F84330EA
:107FB800CDF800803046214603AA3B46FFF798FEDD
:107FC800013002D14FF0FF301FE0304639462A46D3
:107FD8002369C0470130F5D023689B0705D4E068C2
:107FE800039B9842B8BF18460FE00025E368039A40
:107FF8009B1A9D42F3DA3046394604F119020123EF
:10800800C0470130DED00135F0E704B0BDE8F081AB
:10801800B70E0108C80E0108C9B2024410B5904253
:10802800034605D01C7801308C42F8D1184610BDA3
:10803800002010BD431E0A4410B5914204D011F827
:10804800014B03F8014FF8E710BD814201EB020331
:1080580010B501D3421E0BE09842FBD28118D21A08
:10806800D34204D013F8014D01F8014DF8E710BDD3
:10807800994204D011F8014B02F8014FF8E710BDFE
:1080880030B500293DD051F8042C0B1F1D49002A9A
:108098000C46B8BF9B180A6812B95A600B6030BD0D
:1080A80093420DD219685818904201BF5A58521875
:1080B8001A60426823605A6030BD994203D80A4664
:1080C80051680029F9D1146815199D420AD11B6815
:1080D8002344D0181360884213D1086803441360FE
:1080E8004B680DE002D90C23036030BD1C681819D9
:1080F800884202BF086849680019596008BF1860BB
:10810800536030BD981E002070B5CC1C064624F084
:10811800030408340C2C38BF0C24002C03DA0C237D
:108128000020336070BD8C42F9D3204A1368104692
:108138001946A1B10A68121B0ED40B2A03D90A608A
:108148008B188C501FE08B420BBF5A684A6802603C
:108158005A6018BF0B4616E00B464968E9E7144D0C
:108168002B681BB9304600F04BF828603046214692
:1081780000F046F8421C0346D1D0C51C25F0030583
:1081880085420AD11C6003F10B001A1D20F007007C
:10819800821A0AD05142995070BD3046E91A00F04F
:1081A8002FF80130BBD02B46ECE770BD981E00209D
:1081B800941E0020F8B5074615460E4621B911460B
:1081C800BDE8F840FFF7A0BF1AB9FFF759FF2846E6
:1081D800F8BD00F025F8A8420ED238462946FFF728
:1081E80093FF044650B131462A46FFF723FF38462D
:1081F8003146FFF745FF01E03046F8BD2046F8BD9F
:1082080038B50023054C054608462360FBF78AFB72
:10821800431C02D1236803B12B6038BD9C1E00208B
:1082280051F8040C0028BEBF091851F8043CC018C6
:10823800043870472E2E2F73797374656D2F7372FF
:10824800632F73746D333266372D68616C2F7374C6
:108258006D3332663778785F68616C5F6164632E6E
:10826800630000002E2E2F73797374656D2F73725F
:10827800632F73746D333266372D68616C2F737496
:108288006D3332663778785F68616C5F636F7274DC
:1082980065782E63000000002E2E2F7379737465A5
:1082A8006D2F7372632F73746D333266372D686167
:1082B8006C2F73746D3332663778785F68616C5FE2
:1082C8006461632E63000000000610160006101695
:1082D8002E2E2F73797374656D2F7372632F7374D9
:1082E8006D333266372D68616C2F73746D33326667
:1082F8003778785F68616C5F646D612E6300000099
:108308002E2E2F73797374656D2F7372632F7374A8
:108318006D333266372D68616C2F73746D33326636
:108328003778785F68616C5F6770696F2E630000EB
:108338002E2E2F73797374656D2F7372632F737478
:108348006D333266372D68616C2F73746D33326606
:108358003778785F68616C5F6932632E630000006C
:1083680000000000010203040102030406070809D3
:108378002E2E2F73797374656D2F7372632F737438
:108388006D333266372D68616C2F73746D333266C6
:108398003778785F68616C5F7263632E63000000F2
:1083A8002E2E2F73797374656D2F7372632F737408
:1083B8006D333266372D68616C2F73746D33326696
:1083C8003778785F68616C5F7263635F65782E6386
:1083D800000000002E2E2F73797374656D2F737251
:1083E800632F73746D333266372D68616C2F737425
:1083F8006D3332663778785F68616C5F7370692EA9
:108408006300000061626F727428292C2065786906
:1084180074696E672E2E2E002C2066756E63746943
:108428006F6E3A2000000000617373657274696FA3
:108438006E2022257322206661696C65643A206685
:10844800696C6520222573222C206C696E652025B5
:1084580064257325730A00006173736572745F7015
:108468006172616D2829206661696C65643A2066CD
:10847800696C6520222573222C206C696E65202585
:10848800640A00000A0000006D61696E2861726765
:10849800633D25642C20617267763D5B0000000017
:1084A8002C20000022257322000000005D293B0AD1
:1084B80000000000537461636B206672616D653A59
:1084C8000A000000205230203D2020253038580A6C
:1084D80000000000205231203D2020253038580A65
:1084E80000000000205232203D2020253038580A54
:1084F80000000000205233203D2020253038580A43
:108508000000000020523132203D20253038580A22
:1085180000000000204C52203D2020253038580A09
:1085280000000000205043203D2020253038580A04
:108538000000000020505352203D20253038580AB2
:10854800000000004653522F4641523A0A000000EC
:108558002043465352203D2020253038580A000039
:108568002048465352203D2020253038580A000024
:108578002044465352203D2020253038580A000018
:108588002041465352203D2020253038580A00000B
:10859800204D4D464152203D20253038580A0000D4
:1085A8002042464152203D2020253038580A0000FC
:1085B8004D6973630A000000204C522F4558435FF1
:1085C80052455455524E3D20253038580A00000077
:1085D8005B486172644661756C745D0A0000000056
:1085E8005B4275734661756C745D0A005B55736117
:1085F80067654661756C745D0A0000000000000044
:1086080000000000010203040607080900100240E8
:108618000200000000040240400000000004024084
:1086280000020000000402400008000000100240A0
:10863800010000000004024008000000000402409D
:10864800800000000000024000800000000402409A
:108658002000000000040240100000000004024056
:108668000004000025396C64000000002534640013
:10867800252D346400000000493243206469646E8B
:10868800277420496E697420636F72726563746C15
:108698007900000000040002000600010005000344
:1086A8000007800080048002800680018005800326
:1086B8008007400040044002400640014005400356
:1086C8004007C000C004C002C006C001C005C00306
:1086D800C0072000200420022006200120052003D6
:1086E8002007A000A004A002A006A001A005A003E6
:1086F800A007600060046002600660016005600316
:108708006007E000E004E002E006E001E005E003C5
:10871800E0071000100410021006100110051003E5
:108728001007900090049002900690019005900325
:108738009007500050045002500650015005500355
:108748005007D000D004D002D006D001D005D00305
:10875800D0073000300430023006300130053003D5
:108768003007B000B004B002B006B001B005B003E5
:10877800B007700070047002700670017005700315
:108788007007F000F004F002F006F001F005F003C5
:10879800F00708000804080208060801080508038D
:1087A80008078800880488028806880188058803E5
:1087B8008807480048044802480648014805480315
:1087C8004807C800C804C802C806C801C805C803C5
:1087D800C807280028042802280628012805280395
:1087E8002807A800A804A802A806A801A805A803A5
:1087F800A8076800680468026806680168056803D5
:108808006807E800E804E802E806E801E805E80384
:10881800E8071800180418021806180118051803A4
:1088280018079800980498029806980198059803E4
:108838009807580058045802580658015805580314
:108848005807D800D804D802D806D801D805D803C4
:10885800D807380038043802380638013805380394
:108868003807B800B804B802B806B801B805B803A4
:10887800B8077800780478027806780178057803D4
:108888007807F800F804F802F806F801F805F80384
:10889800F8070400040404020406040104050403A0
:1088A8000407840084048402840684018405840304
:1088B8008407440044044402440644014405440334
:1088C8004407C400C404C402C406C401C405C403E4
:1088D800C4072400240424022406240124052403B4
:1088E8002407A400A404A402A406A401A405A403C4
:1088F800A4076400640464026406640164056403F4
:108908006407E400E404E402E406E401E405E403A3
:10891800E4071400140414021406140114051403C3
:108928001407940094049402940694019405940303
:108938009407540054045402540654015405540333
:108948005407D400D404D402D406D401D405D403E3
:10895800D4073400340434023406340134053403B3
:108968003407B400B404B402B406B401B405B403C3
:10897800B4077400740474027406740174057403F3
:108988007407F400F404F402F406F401F405F403A3
:10899800F4070C000C040C020C060C010C050C036B
:1089A8000C078C008C048C028C068C018C058C03C3
:1089B8008C074C004C044C024C064C014C054C03F3
:1089C8004C07CC00CC04CC02CC06CC01CC05CC03A3
:1089D800CC072C002C042C022C062C012C052C0373
:1089E8002C07AC00AC04AC02AC06AC01AC05AC0383
:1089F800AC076C006C046C026C066C016C056C03B3
:108A08006C07EC00EC04EC02EC06EC01EC05EC0362
:108A1800EC071C001C041C021C061C011C051C0382
:108A28001C079C009C049C029C069C019C059C03C2
:108A38009C075C005C045C025C065C015C055C03F2
:108A48005C07DC00DC04DC02DC06DC01DC05DC03A2
:108A5800DC073C003C043C023C063C013C053C0372
:108A68003C07BC00BC04BC02BC06BC01BC05BC0382
:108A7800BC077C007C047C027C067C017C057C03B2
:108A88007C07FC00FC04FC02FC06FC01FC05FC0362
:108A9800FC070200020402020206020102050203A8
:108AA8000207820082048202820682018205820312
:108AB8008207420042044202420642014205420342
:108AC8004207C200C204C202C206C201C205C203F2
:108AD800C2072200220422022206220122052203C2
:108AE8002207A200A204A202A206A201A205A203D2
:108AF800A207620062046202620662016205620302
:108B08006207E200E204E202E206E201E205E203B1
:108B1800E2071200120412021206120112051203D1
:108B28001207920092049202920692019205920311
:108B38009207520052045202520652015205520341
:108B48005207D200D204D202D206D201D205D203F1
:108B5800D2073200320432023206320132053203C1
:108B68003207B200B204B202B206B201B205B203D1
:108B7800B207720072047202720672017205720301
:108B88007207F200F204F202F206F201F205F203B1
:108B9800F2070A000A040A020A060A010A050A0379
:108BA8000A078A008A048A028A068A018A058A03D1
:108BB8008A074A004A044A024A064A014A054A0301
:108BC8004A07CA00CA04CA02CA06CA01CA05CA03B1
:108BD800CA072A002A042A022A062A012A052A0381
:108BE8002A07AA00AA04AA02AA06AA01AA05AA0391
:108BF800AA076A006A046A026A066A016A056A03C1
:108C08006A07EA00EA04EA02EA06EA01EA05EA0370
:108C1800EA071A001A041A021A061A011A051A0390
:108C28001A079A009A049A029A069A019A059A03D0
:108C38009A075A005A045A025A065A015A055A0300
:108C48005A07DA00DA04DA02DA06DA01DA05DA03B0
:108C5800DA073A003A043A023A063A013A053A0380
:108C68003A07BA00BA04BA02BA06BA01BA05BA0390
:108C7800BA077A007A047A027A067A017A057A03C0
:108C88007A07FA00FA04FA02FA06FA01FA05FA0370
:108C9800FA0706000604060206060601060506038C
:108CA80006078600860486028606860186058603F0
:108CB8008607460046044602460646014605460320
:108CC8004607C600C604C602C606C601C605C603D0
:108CD800C6072600260426022606260126052603A0
:108CE8002607A600A604A602A606A601A605A603B0
:108CF800A6076600660466026606660166056603E0
:108D08006607E600E604E602E606E601E605E6038F
:108D1800E6071600160416021606160116051603AF
:108D280016079600960496029606960196059603EF
:108D3800960756005604560256065601560556031F
:108D48005607D600D604D602D606D601D605D603CF
:108D5800D60736003604360236063601360536039F
:108D68003607B600B604B602B606B601B605B603AF
:108D7800B6077600760476027606760176057603DF
:108D88007607F600F604F602F606F601F605F6038F
:108D9800F6070E000E040E020E060E010E050E0357
:108DA8000E078E008E048E028E068E018E058E03AF
:108DB8008E074E004E044E024E064E014E054E03DF
:108DC8004E07CE00CE04CE02CE06CE01CE05CE038F
:108DD800CE072E002E042E022E062E012E052E035F
:108DE8002E07AE00AE04AE02AE06AE01AE05AE036F
:108DF800AE076E006E046E026E066E016E056E039F
:108E08006E07EE00EE04EE02EE06EE01EE05EE034E
:108E1800EE071E001E041E021E061E011E051E036E
:108E28001E079E009E049E029E069E019E059E03AE
:108E38009E075E005E045E025E065E015E055E03DE
:108E48005E07DE00DE04DE02DE06DE01DE05DE038E
:108E5800DE073E003E043E023E063E013E053E035E
:108E68003E07BE00BE04BE02BE06BE01BE05BE036E
:108E7800BE077E007E047E027E067E017E057E039E
:108E88007E07FE00FE04FE02FE06FE01FE05FE034E
:108E9800FE0701000000803F00000000ECFF7F3F5C
:108EA800D40FC93AB1FF7F3FC70F493B4EFF7F3F01
:108EB800C1CB963BC4FE7F3F890FC93B13FE7F3F62
:108EC8003053FB3B39FD7F3F59CB163C39FC7F3F84
:108ED80002ED2F3C11FB7F3F900E493CC1F97F3FCB
:108EE8000030623C4AF87F3F4B517B3CACF67F3FF9
:108EF80038398A3CE6F47F3FB6C9963CF8F27F3FA2
:108F08001C5AA33CE3F07F3F69EAAF3CA7EE7F3FE2
:108F18009B7ABC3C43EC7F3FB00AC93CB8E97F3F31
:108F2800A69AD53C05E77F3F7B2AE23C2BE47F3FAE
:108F38002DBAEE3C29E17F3FB949FB3C00DE7F3F7B
:108F480090EC033DAFDA7F3F2F340A3D37D77F3FA0
:108F5800B87B103D98D37F3F2CC3163DD1CF7F3FC0
:108F6800880A1D3DE2CB7F3FCC51233DCCC77F3FD4
:108F7800F698293D8FC37F3F07E02F3D2ABF7F3FEB
:108F8800FC26363D9EBA7F3FD56D3C3DEAB57F3F16
:108F980091B4423D0FB17F3F2FFB483D0DAC7F3F61
:108FA800AF414F3DE3A67F3F0E88553D91A17F3FDE
:108FB8004CCE5B3D189C7F3F6814623D78967F3F9E
:108FC800625A683DB1907F3F38A06E3DC28A7F3FAC
:108FD800E9E5743DAB847F3F742B7B3D6D7E7F3F1D
:108FE8006CB8803D08787F3F0ADB833D7B717F3F0B
:108FF80094FD863DC76A7F3F0A208A3DEC637F3F28
:109008006A428D3DE95C7F3FB464903DBF557F3F28
:10901800E786933D6D4E7F3F05A9963DF4467F3F19
:109028000ACB993D543F7F3FF9EC9C3D8D377F3FFC
:10903800CF0EA03D9D2F7F3F8C30A33D87277F3FDC
:109048003052A63D491F7F3FBA73A93DE4167F3FC2
:109058002B95AC3D580E7F3F80B6AF3DA4057F3FB2
:10906800BBD7B23DC9FC7E3FDAF8B53DC7F37E3FBA
:10907800DD19B93D9DEA7E3FC33ABC3D4CE17E3FD8
:109088008D5BBF3DD4D77E3F397CC23D34CE7E3F19
:10909800C69CC53D6DC47E3F36BDC83D7FBA7E3F88
:1090A80086DDCB3D69B07E3FB7FDCE3D2DA67E3F28
:1090B800C81DD23DC99B7E3FB93DD53D3D917E3F00
:1090C800895DD83D8B867E3F377DDB3DB17B7E3F1A
:1090D800C49CDE3DB0707E3F2EBCE13D88657E3F7E
:1090E80076DBE43D385A7E3F9AFAE73DC14E7E3F33
:1090F8009A19EB3D23437E3F7638EE3D5E377E3F3F
:109108002E57F13D722B7E3FC075F43D5E1F7E3FAA
:109118002C94F73D24137E3F73B2FA3DC2067E3F7E
:1091280092D0FD3D38FA7D3F4577003E88ED7D3F82
:109138002E06023EB1E07D3F0295033EB2D37D3F4D
:10914800C223053E8CC67D3F6EB2063E40B97D3FC8
:109158000541083ECCAB7D3F86CF093E309E7D3F22
:10916800F35D0B3E6E907D3F4AEC0C3E85827D3F61
:109178008B7A0E3E74747D3FB708103E3D667D3F86
:10918800CC96113EDE577D3FCA24133E59497D3F98
:10919800B2B2143EAC3A7D3F8340163ED82B7D3F99
:1091A8003DCE173EDD1C7D3FE05B193EBC0D7D3F8B
:1091B8006BE91A3E73FE7C3FDE761C3E03EF7C3F74
:1091C80038041E3E6CDF7C3F7B911F3EAECF7C3F58
:1091D800A51E213EC9BF7C3FB6AB223EBDAF7C3F3A
:1091E800AD38243E8A9F7C3F8CC5253E318F7C3F1D
:1091F8005152273EB07E7C3FFCDE283E086E7C3F05
:109208008D6B2A3E3A5D7C3F04F82B3E444C7C3FF4
:1092180061842D3E283B7C3FA2102F3EE5297C3FF0
:10922800C99C303E7A187C3FD428323EE9067C3F00
:10923800C4B4333E31F57B3F9840353E53E37B3F22
:1092480050CC363E4DD17B3FEC57383E20BF7B3F5C
:109258006CE3393ECDAC7B3FCF6E3B3E539A7B3FB0
:1092680015FA3C3EB2877B3F3E853E3EEA747B3F23
:109278004910403EFC617B3F379B413EE74E7B3FB8
:109288000726433EAB3B7B3FB9B0443E48287B3F73
:109298004D3B463EBE147B3FC2C5473E0E017B3F59
:1092A8001850493E37ED7A3F4FDA4A3E3AD97A3F6D
:1092B80067644C3E16C57A3F60EE4D3ECBB07A3FB0
:1092C80038784F3E599C7A3FF101513EC1877A3F29
:1092D800898B523E02737A3F0115543E1C5E7A3FD9
:1092E800589E553E10497A3F8F27573EDD337A3FC7
:1092F800A4B0583E841E7A3F97395A3E04097A3FF3
:109308006AC25B3E5EF3793F1A4B5D3E91DD793F61
:10931800A8D35E3E9DC7793F135C603E83B1793F19
:109328005CE4613E439B793F836C633EDC84793F18
:1093380086F4643E4E6E793F667C663E9A57793F66
:109348002204683EC040793FBA8B693EBF29793F05
:109358002F136B3E9812793F7F9A6C3E4AFB783FF9
:10936800AB216E3ED6E3783FB2A86F3E3BCC783F48
:10937800942F713E7BB4783F51B6723E939C783FF0
:10938800E83C743E8684783F5AC3753E526C783FF9
:10939800A649773EF853783FCCCF783E773B783F65
:1093A800CB557A3ED122783FA4DB7B3E040A783F36
:1093B80056617D3E10F1773FE1E67E3EF7D7773F75
:1093C8002236803EB7BE773FC0F8803E51A5773F32
:1093D8004ABB813EC58B773FC07D823E1372773F83
:1093E8002240833E3A58773F7002843E3C3E773FA6
:1093F800AAC4843E1724773FCE86853ECC09773FA2
:10940800DF48863E5BEF763FDA0A873EC4D4763F74
:10941800C1CC873E07BA763F938E883E249F763F1D
:109428005050893E1B84763FF8118A3EEC68763F9F
:109438008AD38A3E974D763F07958B3E1B32763FFF
:109448006E568C3E7A16763FC0178D3EB3FA753F3E
:10945800FCD88D3EC6DE753F229A8E3EB3C2753F5C
:10946800325B8F3E7BA6753F2C1C903E1C8A753F55
:1094780010DD903E976D753FDD9D913EED50753F37
:10948800945E923E1D34753F351F933E2717753FF6
:10949800BFDF933E0BFA743F31A0943EC9DC743FA2
:1094A8008D60953E62BF743FD220963ED5A1743F31
:1094B80000E1963E2284743F17A1973E4966743FA7
:1094C8001661983E4B48743FFE20993E272A743F08
:1094D800CEE0993EDD0B743F86A09A3E6EED733F59
:1094E80027609B3ED9CE733FAF1F9C3E1FB0733F92
:1094F80020DF9C3E3F91733F789E9D3E3972733FBB
:10950800B85D9E3E0E53733FDF1C9F3EBE33733FD4
:10951800EEDB9F3E4714733FE59AA03EACF4723FE2
:10952800C259A13EEBD4723F8718A23E04B5723FE0
:1095380033D7A23EF894723FC595A33EC774723FD5
:109548003F54A43E7054723F9F12A53EF433723FBD
:10955800E5D0A53E5213723F128FA63E8CF2713FA2
:10956800254DA73E9FD1713F1F0BA83E8EB0713F7E
:10957800FEC8A83E578F713FC486A93EFB6D713F58
:109588006F44AA3E7A4C713F0102AB3ED42A713F28
:1095980077BFAB3E0809713FD47CAC3E17E7703FFC
:1095A800153AAD3E02C5703F3CF7AD3EC6A2703FCE
:1095B80049B4AE3E6680703F3A71AF3EE15D703FA0
:1095C800102EB03E373B703FCBEAB03E6718703F75
:1095D8006BA7B13E73F56F3FEF63B23E5AD26F3F50
:1095E8005820B33E1BAF6F3FA5DCB33EB88B6F3F2F
:1095F800D698B43E30686F3FEC54B53E83446F3F15
:10960800E610B63EB0206F3FC3CCB63EBAFC6E3F04
:109618008488B73E9ED86E3F2A44B83E5DB46E3FFC
:10962800B2FFB83EF88F6E3F1EBBB93E6D6B6E3F02
:109638006E76BA3EBE466E3FA031BB3EEB216E3F12
:10964800B6ECBB3EF2FC6D3FAFA7BC3ED5D76D3F35
:109658008B62BD3E93B26D3F4A1DBE3E2D8D6D3F60
:10966800EBD7BE3EA1676D3F6F92BF3EF2416D3FA3
:10967800D54CC03E1D1C6D3F1E07C13E24F66C3FF5
:1096880048C1C13E07D06C3F557BC23EC5A96C3F5F
:109698004435C33E5E836C3F15EFC33ED45C6C3FDC
:1096A800C8A8C43E24366C3F5C62C53E500F6C3F70
:1096B800D21BC63E58E86B3F29D5C63E3BC16B3F1F
:1096C800628EC73EFB996B3F7C47C83E95726B3FE5
:1096D8007700C93E0C4B6B3F53B9C93E5E236B3FC5
:1096E8001072CA3E8CFB6A3FAE2ACB3E95D36A3FC6
:1096F8002CE3CB3E7BAB6A3F8B9BCC3E3C836A3FE3
:10970800CA53CD3ED95A6A3FEA0BCE3E52326A3F1F
:10971800EAC3CE3EA7096A3FCA7BCF3ED7E0693F7E
:109728008A33D03EE4B7693F2AEBD03ECC8E693FFE
:10973800AAA2D13E9165693F095AD23E323C693F9F
:109748004811D33EAE12693F67C8D33E07E9683F68
:10975800647FD43E3CBF683F4136D53E4C95683F58
:10976800FDECD53E396B683F99A3D63E0341683F6F
:10977800135AD73EA816683F6B10D83E2AEC673FAD
:10978800A3C6D83E87C1673FB97CD93EC196673F1B
:10979800AD32DA3ED86B673F80E8DA3ECA40673FB1
:1097A800319EDB3E9915673FC153DC3E45EA663F73
:1097B8002E09DD3ECCBE663F79BEDD3E3093663F66
:1097C800A273DE3E7167663FA928DF3E8E3B663F87
:1097D8008DDDDF3E880F663F4F92E03E5EE3653FDA
:1097E800EE46E13E10B7653F6AFBE13EA08A653F61
:1097F800C4AFE23E0B5E653FFA63E33E5431653F1A
:109808000E18E43E7904653FFECBE43E7BD7643F07
:10981800CB7FE53E59AA643F7533E63E147D643F2D
:10982800FBE6E63EAC4F643F5D9AE73E2122643F8B
:109838009C4DE83E73F4633FB700E93EA1C6633F21
:10984800AEB3E93EAC98633F8166EA3E956A633FF2
:109858003019EB3E5A3C633FBBCBEB3EFC0D633FFC
:10986800217EEC3E7BDF623F6330ED3ED7B0623F46
:1098780080E2ED3E1082623F7994EE3E2653623FCD
:109888004C46EF3E1A24623FFBF7EF3EEAF4613F95
:1098980085A9F03E98C5613FEA5AF13E2296613F9C
:1098A800290CF23E8A66613F43BDF23ED036613FE5
:1098B800386EF33EF206613F071FF43EF2D6603F72
:1098C800B1CFF43ECFA6603F3580F53E8976603F44
:1098D8009330F63E2146603FCBE0F63E9615603F5A
:1098E800DC90F73EE9E45F3FC840F83E19B45F3FBB
:1098F8008EF0F83E27835F3F2DA0F93E12525F3F5E
:10990800A54FFA3EDB205F3FF7FEFA3E81EF5E3F50
:1099180022AEFB3E05BE5E3F275DFC3E678C5E3F88
:10992800040CFD3EA65A5E3FBBBAFD3EC3285E3F0F
:109938004A69FE3EBEF65D3FB217FF3E97C45D3FE3
:10994800F3C5FF3E4D925D3F063A003FE15F5D3F44
:10995800FF90003F532D5D3FE4E7003FA3FA5C3FD3
:10996800B53E013FD1C75C3F7395013FDD945C3F35
:109978001CEC013FC7615C3FB142023F8E2E5C3F49
:109988003299023F34FB5B3F9FEF023FB8C75B3F12
:10999800F845033F1A945B3F3D9C033F5A605B3F89
:1099A8006DF2033F792C5B3F8948043F75F85A3FB5
:1099B800919E043F50C45A3F84F4043F09905A3F93
:1099C800624A053FA05B5A3F2CA0053F16275A3F25
:1099D800E2F5053F6AF2593F824B063F9CBD593F6D
:1099E8000EA1063FAD88593F86F6063F9C53593F66
:1099F800E84B073F6A1E593F36A1073F17E9583F12
:109A08006FF6073FA1B3583F924B083F0B7E583F74
:109A1800A1A0083F5348583F9BF5083F7912583F8B
:109A28007F4A093F7FDC573F4E9F093F63A6573F58
:109A380009F4093F2670573FAD480A3FC739573FD9
:109A48003D9D0A3F4803573FB7F10A3FA7CC563F11
:109A58001C460B3FE595563F6B9A0B3F025F563FFE
:109A6800A5EE0B3FFE27563FC9420C3FD9F0553FA4
:109A7800D7960C3F93B9553FD0EA0C3F2C82553FFF
:109A8800B33E0D3FA44A553F81920D3FFB12553F0F
:109A980038E60D3F31DB543FDA390E3F47A3543FD8
:109AA800658D0E3F3B6B543FDBE00E3F0F33543F59
:109AB8003B340F3FC3FA533F84870F3F55C2533F90
:109AC800B8DA0F3FC789533FD52D103F1851533F80
:109AD800DC80103F4918533FCDD3103F59DF523F28
:109AE800A726113F49A6523F6B79113F186D523F87
:109AF80019CC113FC633523FB01E123F54FA513FA2
:109B08003071123FC2C0513F9AC3123F1087513F74
:109B1800EE15133F3D4D513F2A68133F4A13513FFD
:109B280050BA133F37D9503F5F0C143F039F503F43
:109B3800585E143FAF64503F39B0143F3B2A503F42
:109B48000402153FA8EF4F3FB753153FF4B44F3FFA
:109B580054A5153F1F7A4F3FD9F6153F2B3F4F3F6E
:109B68004748163F17044F3F9F99163FE4C84E3F9A
:109B7800DFEA163F908D4E3F073C173F1C524E3F81
:109B8800188D173F89164E3F12DE173FD5DA4D3F25
:109B9800F52E183F029F4D3FC07F183F10634D3F81
:109BA80073D0183FFD264D3F0F21193FCBEA4C3F9C
:109BB8009471193F79AE4C3F00C2193F08724C3F6F
:109BC80055121A3F78354C3F93621A3FC7F84B3FFE
:109BD800B8B21A3FF8BB4B3FC6021B3F097F4B3F49
:109BE800BB521B3FFA414B3F99A21B3FCC044B3F52
:109BF8005FF21B3F7FC74A3F0C421C3F138A4A3F14
:109C0800A2911C3F874C4A3F1FE11C3FDC0E4A3F94
:109C180084301D3F12D1493FD17F1D3F2993493FD1
:109C280006CF1D3F2155493F221E1E3FFA16493FC8
:109C3800266D1E3FB3D8483F12BC1E3F4E9A483F80
:109C4800E50A1F3FCA5B483F9F591F3F271D483FF2
:109C580041A81F3F65DE473FCBF61F3F849F473F24
:109C68003B45203F8560473F9393203F6721473F0F
:109C7800D2E1203F2AE2463FF92F213FCEA2463FBC
:109C8800067E213F5463463FFBCB213FBB23463F23
:109C9800D719223F03E4453F9967223F2DA4453F4A
:109CA80043B5223F3964453FD302233F2624453F2D
:109CB8004B50233FF5E3443FA99D233FA5A3443FD1
:109CC800EEEA233F3763443F1A38243FAB22443F30
:109CD8002C85243F00E2433F25D2243F38A1433F4F
:109CE800041F253F5160433FCB6B253F4C1F433F2B
:109CF80077B8253F29DE423F0A05263FE89C423FC8
:109D08008451263F895B423FE39D263F0B1A423F21
:109D18002AEA263F70D8413F5636273FB796413F3B
:109D28006882273FE154413F61CE273FEC12413F13
:109D3800401A283FDAD0403F0566283FA98E403FA9
:109D4800B0B1283F5C4C403F41FD283FF009403FFF
:109D5800B848293F67C73F3F1594293FC0843F3F14
:109D680057DF293FFC413F3F802A2A3F1BFF3E3FE8
:109D78008E752A3F1BBC3E3F82C02A3FFF783E3F7C
:109D88005B0B2B3FC5353E3F1B562B3F6EF23D3FCD
:109D9800BFA02B3FF9AE3D3F4AEB2B3F676B3D3FE2
:109DA800B9352C3FB8273D3F0F802C3FECE33C3FB3
:109DB80049CA2C3F03A03C3F69142D3FFC5B3C3F44
:109DC8006F5E2D3FD9173C3F59A82D3F98D33B3F95
:109DD80029F22D3F3B8F3B3FDE3B2E3FC14A3B3FA5
:109DE80078852E3F29063B3FF7CE2E3F75C13A3F77
:109DF8005B182F3FA47C3A3FA5612F3FB7373A3F06
:109E0800D3AA2F3FACF2393FE6F32F3F85AD393F58
:109E1800DE3C303F4268393FBB85303FE122393F65
:109E28007CCE303F65DD383F2217313FCB97383F36
:109E3800AD5F313F1652383F1DA8313F430C383FC4
:109E480071F0313F55C6373FAA38323F4A80373F15
:109E5800C780323F233A373FC9C8323FDFF3363F26
:109E6800AF10333F7FAD363F7A58333F0467363FF4
:109E780029A0333F6C20363FBCE7333FB8D9353F84
:109E8800342F343FE792353F8F76343FFB4B353FD5
:109E9800CFBD343FF304353FF304353FCFBD343FE6
:109EA800FB4B353F8F76343FE792353F342F343FB5
:109EB800B8D9353FBCE7333F6C20363F29A0333F44
:109EC8000467363F7A58333F7FAD363FAF10333F94
:109ED800DFF3363FC9C8323F233A373FC780323FA6
:109EE8004A80373FAA38323F55C6373F71F0313F75
:109EF800430C383F1DA8313F1652383FAD5F313F04
:109F0800CB97383F2217313F65DD383F7CCE303F55
:109F1800E122393FBB85303F4268393FDE3C303F64
:109F280085AD393FE6F32F3FACF2393FD3AA2F3F37
:109F3800B7373A3FA5612F3FA47C3A3F5B182F3FC4
:109F480075C13A3FF7CE2E3F29063B3F78852E3F15
:109F5800C14A3B3FDE3B2E3F3B8F3B3F29F22D3F23
:109F680098D33B3F59A82D3FD9173C3F6F5E2D3FF3
:109F7800FC5B3C3F69142D3F03A03C3F49CA2C3F82
:109F8800ECE33C3F0F802C3FB8273D3FB9352C3FD1
:109F9800676B3D3F4AEB2B3FF9AE3D3FBFA02B3FE0
:109FA8006EF23D3F1B562B3FC5353E3F5B0B2B3FAB
:109FB800FF783E3F82C02A3F1BBC3E3F8E752A3F3A
:109FC8001BFF3E3F802A2A3FFC413F3F57DF293F86
:109FD800C0843F3F1594293F67C73F3FB848293F92
:109FE800F009403F41FD283F5C4C403FB0B1283F5D
:109FF800A98E403F0566283FDAD0403F401A283FE7
:10A00800EC12413F61CE273FE154413F6882273F30
:10A01800B796413F5636273F70D8413F2AEA263F38
:10A028000B1A423FE39D263F895B423F8451263FFE
:10A03800E89C423F0A05263F29DE423F77B8253F84
:10A048004C1F433FCB6B253F5160433F041F253FC7
:10A0580038A1433F25D2243F00E2433F2C85243FCB
:10A06800AB22443F1A38243F3763443FEEEA233F8C
:10A07800A5A3443FA99D233FF5E3443F4B50233F0D
:10A088002624453FD302233F3964453F43B5223F49
:10A098002DA4453F9967223F03E4453FD719223F46
:10A0A800BB23463FFBCB213F5463463F067E213FFF
:10A0B800CEA2463FF92F213F2AE2463FD2E1203F78
:10A0C8006721473F9393203F8560473F3B45203FAB
:10A0D800849F473FCBF61F3F65DE473F41A81F3FA0
:10A0E800271D483F9F591F3FCA5B483FE50A1F3F4E
:10A0F8004E9A483F12BC1E3FB3D8483F266D1E3FBC
:10A10800FA16493F221E1E3F2155493F06CF1D3FE3
:10A118002993493FD17F1D3F12D1493F84301D3FCC
:10A12800DC0E4A3F1FE11C3F874C4A3FA2911C3F6F
:10A13800138A4A3F0C421C3F7FC74A3F5FF21B3FCE
:10A14800CC044B3F99A21B3FFA414B3FBB521B3FEC
:10A15800097F4B3FC6021B3FF8BB4B3FB8B21A3FC3
:10A16800C7F84B3F93621A3F78354C3F55121A3F58
:10A1780008724C3F00C2193F79AE4C3F9471193FA9
:10A18800CBEA4C3F0F21193FFD264D3F73D0183FB6
:10A1980010634D3FC07F183F029F4D3FF52E183F7B
:10A1A800D5DA4D3F12DE173F89164E3F188D173FFF
:10A1B8001C524E3F073C173F908D4E3FDFEA163F3B
:10A1C800E4C84E3F9F99163F17044F3F4748163F34
:10A1D8002B3F4F3FD9F6153F1F7A4F3F54A5153FE8
:10A1E800F4B44F3FB753153FA8EF4F3F0402153F54
:10A1F8003B2A503F39B0143FAF64503F585E143F7C
:10A20800039F503F5F0C143F37D9503F50BA133F5C
:10A218004A13513F2A68133F3D4D513FEE15133FF6
:10A228001087513F9AC3123FC2C0513F3071123F4D
:10A2380054FA513FB01E123FC633523F19CC113F5A
:10A24800186D523F6B79113F49A6523FA726113F1F
:10A2580059DF523FCDD3103F4918533FDC80103FA0
:10A268001851533FD52D103FC789533FB8DA0F3FD8
:10A2780055C2533F84870F3FC3FA533F3B340F3FC8
:10A288000F33543FDBE00E3F3B6B543F658D0E3F71
:10A2980047A3543FDA390E3F31DB543F38E60D3FD0
:10A2A800FB12553F81920D3FA44A553FB33E0D3FE7
:10A2B8002C82553FD0EA0C3F93B9553FD7960C3FB7
:10A2C800D9F0553FC9420C3FFE27563FA5EE0B3F3C
:10A2D800025F563F6B9A0B3FE595563F1C460B3F76
:10A2E800A7CC563FB7F10A3F4803573F3D9D0A3F69
:10A2F800C739573FAD480A3F2670573F09F4093F11
:10A3080063A6573F4E9F093F7FDC573F7F4A093F6F
:10A318007912583F9BF5083F5348583FA1A0083F82
:10A328000B7E583F924B083FA1B3583F6FF6073F4B
:10A3380017E9583F36A1073F6A1E593FE84B073FC8
:10A348009C53593F86F6063FAD88593F0EA1063FFC
:10A358009CBD593F824B063F6AF2593FE2F5053FE3
:10A3680016275A3F2CA0053FA05B5A3F624A053F7B
:10A3780009905A3F84F4043F50C45A3F919E043FC9
:10A3880075F85A3F8948043F792C5B3F6DF2033FCB
:10A398005A605B3F3D9C033F1A945B3FF845033F7F
:10A3A800B8C75B3F9FEF023F34FB5B3F3299023FE8
:10A3B8008E2E5C3FB142023FC7615C3F1CEC013FFF
:10A3C800DD945C3F7395013FD1C75C3FB53E013FCB
:10A3D800A3FA5C3FE4E7003F532D5D3FFF90003F49
:10A3E800E15F5D3F063A003F4D925D3FF3C5FF3E9A
:10A3F80097C45D3FB217FF3EBEF65D3F4A69FE3E19
:10A40800C3285E3FBBBAFD3EA65A5E3F040CFD3E24
:10A41800678C5E3F275DFC3E05BE5E3F22AEFB3E7D
:10A4280081EF5E3FF7FEFA3EDB205F3FA54FFA3E25
:10A4380012525F3F2DA0F93E27835F3F8EF0F83E12
:10A4480019B45F3FC840F83EE9E45F3FDC90F73E4F
:10A458009615603FCBE0F63E2146603F9330F63ECE
:10A468008976603F3580F53ECFA6603FB1CFF43E98
:10A47800F2D6603F071FF43EF206613F386EF33EA6
:10A48800D036613F43BDF23E8A66613F290CF23EF9
:10A498002296613FEA5AF13E98C5613F85A9F03E90
:10A4A800EAF4613FFBF7EF3E1A24623F4C46EF3E69
:10A4B8002653623F7994EE3E1082623F80E2ED3E81
:10A4C800D7B0623F6330ED3E7BDF623F217EEC3EDA
:10A4D800FC0D633FBBCBEB3E5A3C633F3019EB3E70
:10A4E800956A633F8166EA3EAC98633FAEB3E93E46
:10A4F800A1C6633FB700E93E73F4633F9C4DE83E55
:10A508002122643F5D9AE73EAC4F643FFBE6E63E9E
:10A51800147D643F7533E63E59AA643FCB7FE53E20
:10A528007BD7643FFECBE43E7904653F0E18E43EDA
:10A538005431653FFA63E33E0B5E653FC4AFE23ECC
:10A54800A08A653F6AFBE13E10B7653FEE46E13EF3
:10A558005EE3653F4F92E03E880F663F8DDDDF3E4C
:10A568008E3B663FA928DF3E7167663FA273DE3ED9
:10A578003093663F79BEDD3ECCBE663F2E09DD3E98
:10A5880045EA663FC153DC3E9915673F319EDB3E85
:10A59800CA40673F80E8DA3ED86B673FAD32DA3EA3
:10A5A800C196673FB97CD93E87C1673FA3C6D83EED
:10A5B8002AEC673F6B10D83EA816683F135AD73E5F
:10A5C8000341683F99A3D63E396B683FFDECD53E01
:10A5D8004C95683F4136D53E3CBF683F647FD43ECA
:10A5E80007E9683F67C8D33EAE12693F4811D33EBA
:10A5F800323C693F095AD23E9165693FAAA2D13ED1
:10A60800CC8E693F2AEBD03EE4B7693F8A33D03E0F
:10A61800D7E0693FCA7BCF3EA7096A3FEAC3CE3E6F
:10A6280052326A3FEA0BCE3ED95A6A3FCA53CD3EF0
:10A638003C836A3F8B9BCC3E7BAB6A3F2CE3CB3E93
:10A6480095D36A3FAE2ACB3E8CFB6A3F1072CA3E56
:10A658005E236B3F53B9C93E0C4B6B3F7700C93E35
:10A6680095726B3F7C47C83EFB996B3F628EC73E35
:10A678003BC16B3F29D5C63E58E86B3FD21BC63E4F
:10A68800500F6C3F5C62C53E24366C3FC8A8C43E80
:10A69800D45C6C3F15EFC33E5E836C3F4435C33ECC
:10A6A800C5A96C3F557BC23E07D06C3F48C1C13E2F
:10A6B80024F66C3F1E07C13E1D1C6D3FD54CC03EA5
:10A6C800F2416D3F6F92BF3EA1676D3FEBD7BE3E33
:10A6D8002D8D6D3F4A1DBE3E93B26D3F8B62BD3ED0
:10A6E800D5D76D3FAFA7BC3EF2FC6D3FB6ECBB3E85
:10A6F800EB216E3FA031BB3EBE466E3F6E76BA3E42
:10A708006D6B6E3F1EBBB93EF88F6E3FB2FFB83E11
:10A718005DB46E3F2A44B83E9ED86E3F8488B73EEB
:10A72800BAFC6E3FC3CCB63EB0206F3FE610B63ED3
:10A7380083446F3FEC54B53E30686F3FD698B43EC3
:10A74800B88B6F3FA5DCB33E1BAF6F3F5820B33EBD
:10A758005AD26F3FEF63B23E73F56F3F6BA7B13EBE
:10A768006718703FCBEAB03E373B703F102EB03EC3
:10A77800E15D703F3A71AF3E6680703F49B4AE3ECE
:10A78800C6A2703F3CF7AD3E02C5703F153AAD3EDC
:10A7980017E7703FD47CAC3E0809713F77BFAB3EEA
:10A7A800D42A713F0102AB3E7A4C713F6F44AA3EF6
:10A7B800FB6D713FC486A93E578F713FFEC8A83E06
:10A7C8008EB0713F1F0BA83E9FD1713F254DA73E0C
:10A7D8008CF2713F128FA63E5213723FE5D0A53E10
:10A7E800F433723F9F12A53E7054723F3F54A43E0B
:10A7F800C774723FC595A33EF894723F33D7A23E03
:10A8080004B5723F8718A23EEBD4723FC259A13EED
:10A81800ACF4723FE59AA03E4714733FEEDB9F3ECF
:10A82800BE33733FDF1C9F3E0E53733FB85D9E3EA1
:10A838003972733F789E9D3E3F91733F20DF9C3E67
:10A848001FB0733FAF1F9C3ED9CE733F27609B3E1E
:10A858006EED733F86A09A3EDD0B743FCEE0993EC5
:10A86800272A743FFE20993E4B48743F1661983E54
:10A878004966743F17A1973E2284743F00E1963ED3
:10A88800D5A1743FD220963E62BF743F8D60953E3D
:10A89800C9DC743F31A0943E0BFA743FBFDF933E8E
:10A8A8002717753F351F933E1D34753F945E923EC2
:10A8B800ED50753FDD9D913E976D753F10DD903EE3
:10A8C8001C8A753F2C1C903E7BA6753F325B8F3EE1
:10A8D800B3C2753F229A8E3EC6DE753FFCD88D3EC8
:10A8E800B3FA753FC0178D3E7A16763F6E568C3E8A
:10A8F8001B32763F07958B3E974D763F8AD38A3E2B
:10A90800EC68763FF8118A3E1B84763F5050893EAA
:10A91800249F763F938E883E07BA763FC1CC873E08
:10A92800C4D4763FDA0A873E5BEF763FDF48863E3F
:10A93800CC09773FCE86853E1724773FAAC4843E4C
:10A948003C3E773F7002843E3A58773F2240833E30
:10A958001372773FC07D823EC58B773F4ABB813EED
:10A9680051A5773FC0F8803EB7BE773F2236803E7C
:10A97800F7D7773FE1E67E3E10F1773F56617D3E9F
:10A98800040A783FA4DB7B3ED122783FCB557A3E40
:10A99800773B783FCCCF783EF853783FA649773E4F
:10A9A800526C783F5AC3753E8684783FE83C743EC3
:10A9B800939C783F51B6723E7BB4783F942F713E9A
:10A9C8003BCC783FB2A86F3ED6E3783FAB216E3ED2
:10A9D8004AFB783F7F9A6C3E9812793F2F136B3E63
:10A9E800BF29793FBA8B693EC040793F2204683E4F
:10A9F8009A57793F667C663E4E6E793F86F4643E90
:10AA0800DC84793F836C633E439B793F5CE4613E21
:10AA180083B1793F135C603E9DC7793FA8D35E3E02
:10AA280091DD793F1A4B5D3E5EF3793F6AC25B3E2A
:10AA380004097A3F97395A3E841E7A3FA4B0583E9B
:10AA4800DD337A3F8F27573E10497A3F589E553E4F
:10AA58001C5E7A3F0115543E02737A3F898B523E41
:10AA6800C1877A3FF101513E599C7A3F38784F3E71
:10AA7800CBB07A3F60EE4D3E16C57A3F67644C3ED8
:10AA88003AD97A3F4FDA4A3E37ED7A3F1850493E75
:10AA98000E017B3FC2C5473EBE147B3F4D3B463E41
:10AAA80048287B3FB9B0443EAB3B7B3F0726433E3B
:10AAB800E74E7B3F379B413EFC617B3F4910403E60
:10AAC800EA747B3F3E853E3EB2877B3F15FA3C3EAB
:10AAD800539A7B3FCF6E3B3ECDAC7B3F6CE3393E18
:10AAE80020BF7B3FEC57383E4DD17B3F50CC363EA4
:10AAF80053E37B3F9840353E31F57B3FC4B4333E4A
:10AB0800E9067C3FD428323E7A187C3FC99C303E07
:10AB1800E5297C3FA2102F3E283B7C3F61842D3ED7
:10AB2800444C7C3F04F82B3E3A5D7C3F8D6B2A3EBB
:10AB3800086E7C3FFCDE283EB07E7C3F5152273EAB
:10AB4800318F7C3F8CC5253E8A9F7C3FAD38243EA3
:10AB5800BDAF7C3FB6AB223EC9BF7C3FA51E213EA0
:10AB6800AECF7C3F7B911F3E6CDF7C3F38041E3E9E
:10AB780003EF7C3FDE761C3E73FE7C3F6BE91A3E9A
:10AB8800BC0D7D3FE05B193EDD1C7D3F3DCE173E91
:10AB9800D82B7D3F8340163EAC3A7D3FB2B2143E7F
:10ABA80059497D3FCA24133EDE577D3FCC96113E5E
:10ABB8003D667D3FB708103E74747D3F8B7A0E3E2C
:10ABC80085827D3F4AEC0C3E6E907D3FF35D0B3EE7
:10ABD800309E7D3F86CF093ECCAB7D3F0541083E88
:10ABE80040B97D3F6EB2063E8CC67D3FC223053E0E
:10ABF800B2D37D3F0295033EB1E07D3F2E06023E73
:10AC080088ED7D3F4577003E38FA7D3F92D0FD3D87
:10AC1800C2067E3F73B2FA3D24137E3F2C94F73D63
:10AC28005E1F7E3FC075F43D722B7E3F2E57F13D6F
:10AC38005E377E3F7638EE3D23437E3F9A19EB3DE3
:10AC4800C14E7E3F9AFAE73D385A7E3F76DBE43DB7
:10AC580088657E3F2EBCE13DB0707E3FC49CDE3DE2
:10AC6800B17B7E3F377DDB3D8B867E3F895DD83D5E
:10AC78003D917E3FB93DD53DC99B7E3FC81DD23D24
:10AC88002DA67E3FB7FDCE3D69B07E3F86DDCB3D2C
:10AC98007FBA7E3F36BDC83D6DC47E3FC69CC53D6C
:10ACA80034CE7E3F397CC23DD4D77E3F8D5BBF3DDD
:10ACB8004CE17E3FC33ABC3D9DEA7E3FDD19B93D7C
:10ACC800C7F37E3FDAF8B53DC9FC7E3FBBD7B23D3E
:10ACD800A4057F3F80B6AF3D580E7F3F2B95AC3D16
:10ACE800E4167F3FBA73A93D491F7F3F3052A63D06
:10ACF80087277F3F8C30A33D9D2F7F3FCF0EA03D00
:10AD08008D377F3FF9EC9C3D543F7F3F0ACB993DFF
:10AD1800F4467F3F05A9963D6D4E7F3FE786933DFC
:10AD2800BF557F3FB464903DE95C7F3F6A428D3DEB
:10AD3800EC637F3F0A208A3DC76A7F3F94FD863DCA
:10AD48007B717F3F0ADB833D08787F3F6CB8803D8D
:10AD58006D7E7F3F742B7B3DAB847F3FE9E5743D7F
:10AD6800C28A7F3F38A06E3DB1907F3F625A683DEE
:10AD780078967F3F6814623D189C7F3F4CCE5B3DC0
:10AD880091A17F3F0E88553DE3A67F3FAF414F3DE0
:10AD98000DAC7F3F2FFB483D0FB17F3F91B4423D43
:10ADA800EAB57F3FD56D3C3D9EBA7F3FFC26363DD8
:10ADB8002ABF7F3F07E02F3D8FC37F3FF698293D8D
:10ADC800CCC77F3FCC51233DE2CB7F3F880A1D3D56
:10ADD800D1CF7F3F2CC3163D98D37F3FB87B103D22
:10ADE80037D77F3F2F340A3DAFDA7F3F90EC033DE2
:10ADF80000DE7F3FB949FB3C29E17F3F2DBAEE3C9D
:10AE08002BE47F3F7B2AE23C05E77F3FA69AD53CAF
:10AE1800B8E97F3FB00AC93C43EC7F3F9B7ABC3C12
:10AE2800A7EE7F3F69EAAF3CE3F07F3F1C5AA33CA3
:10AE3800F8F27F3FB6C9963CE6F47F3F38398A3C42
:10AE4800ACF67F3F4B517B3C4AF87F3F0030623C79
:10AE5800C1F97F3F900E493C11FB7F3F02ED2F3C2B
:10AE680039FC7F3F59CB163C39FD7F3F3053FB3BC4
:10AE780013FE7F3F890FC93BC4FE7F3FC1CB963B82
:10AE88004EFF7F3FC70F493BB1FF7F3FD40FC93A01
:10AE9800ECFF7F3F000000000000803FD40FC9BADC
:10AEA800ECFF7F3FC70F49BBB1FF7F3FC1CB96BBCC
:10AEB8004EFF7F3F890FC9BBC4FE7F3F3053FBBBAA
:10AEC80013FE7F3F59CB16BC39FD7F3F02ED2FBCE7
:10AED80039FC7F3F900E49BC11FB7F3F003062BCBC
:10AEE800C1F97F3F4B517BBC4AF87F3F38398ABC58
:10AEF800ACF67F3FB6C996BCE6F47F3F1C5AA3BCAC
:10AF0800F8F27F3F69EAAFBCE3F07F3F9B7ABCBCB5
:10AF1800A7EE7F3FB00AC9BC43EC7F3FA69AD5BCD9
:10AF2800B8E97F3F7B2AE2BC05E77F3F2DBAEEBC3C
:10AF38002BE47F3FB949FBBC29E17F3F90EC03BD7F
:10AF480000DE7F3F2F340ABDAFDA7F3FB87B10BDEC
:10AF580037D77F3F2CC316BD98D37F3F880A1DBDC6
:10AF6800D1CF7F3FCC5123BDE2CB7F3FF69829BD9F
:10AF7800CCC77F3F07E02FBD8FC37F3FFC2636BD80
:10AF88002ABF7F3FD56D3CBD9EBA7F3F91B442BD7D
:10AF9800EAB57F3F2FFB48BD0FB17F3FAF414FBDA3
:10AFA8000DAC7F3F0E8855BDE3A67F3F4CCE5BBD01
:10AFB80091A17F3F681462BD189C7F3F625A68BDAB
:10AFC80078967F3F38A06EBDB1907F3FE9E574BDAC
:10AFD800C28A7F3F742B7BBDAB847F3F6CB880BD3A
:10AFE8006D7E7F3F0ADB83BD08787F3F94FD86BD79
:10AFF8007B717F3F0A208ABDC76A7F3F6A428DBD49
:10B00800EC637F3FB46490BDE95C7F3FE78693BD06
:10B01800BF557F3F05A996BD6D4E7F3F0ACB99BDB1
:10B02800F4467F3FF9EC9CBD543F7F3FCF0EA0BD57
:10B038008D377F3F8C30A3BD9D2F7F3F3052A6BDFB
:10B0480087277F3FBA73A9BD491F7F3F2B95ACBDAA
:10B05800E4167F3F80B6AFBD580E7F3FBBD7B2BD69
:10B06800A4057F3FDAF8B5BDC9FC7E3FDD19B9BD3F
:10B07800C7F37E3FC33ABCBD9DEA7E3F8D5BBFBD33
:10B088004CE17E3F397CC2BDD4D77E3FC69CC5BD4E
:10B0980034CE7E3F36BDC8BD6DC47E3F86DDCBBD98
:10B0A8007FBA7E3FB7FDCEBD69B07E3FC81DD2BD19
:10B0B8002DA67E3FB93DD5BDC99B7E3F895DD8BDD4
:10B0C8003D917E3F377DDBBD8B867E3FC49CDEBDD8
:10B0D800B17B7E3F2EBCE1BDB0707E3F76DBE4BD28
:10B0E80088657E3F9AFAE7BD385A7E3F9A19EBBDCC
:10B0F800C14E7E3F7638EEBD23437E3F2E57F1BDCD
:10B108005E377E3FC075F4BD722B7E3F2C94F7BD31
:10B118005E1F7E3F73B2FABD24137E3F92D0FDBD01
:10B12800C2067E3F457700BE38FA7D3F2E0602BE36
:10B1380088ED7D3F029503BEB1E07D3FC22305BE89
:10B14800B2D37D3F6EB206BE8CC67D3F054108BEB8
:10B1580040B97D3F86CF09BECCAB7D3FF35D0BBECA
:10B16800309E7D3F4AEC0CBE6E907D3F8B7A0EBEC2
:10B1780085827D3FB70810BE74747D3FCC9611BEA2
:10B188003D667D3FCA2413BEDE577D3FB2B214BE72
:10B1980059497D3F834016BEAC3A7D3F3DCE17BE30
:10B1A800D82B7D3FE05B19BEDD1C7D3F6BE91ABEE5
:10B1B800BC0D7D3FDE761CBE73FE7C3F38041EBE90
:10B1C80003EF7C3F7B911FBE6CDF7C3FA51E21BE39
:10B1D800AECF7C3FB6AB22BEC9BF7C3FAD3824BEE4
:10B1E800BDAF7C3F8CC525BE8A9F7C3F515227BE90
:10B1F800318F7C3FFCDE28BEB07E7C3F8D6B2ABE43
:10B20800086E7C3F04F82BBE3A5D7C3F61842DBEFE
:10B21800444C7C3FA2102FBE283B7C3FC99C30BECB
:10B22800E5297C3FD42832BE7A187C3FC4B433BEAB
:10B23800E9067C3F984035BE31F57B3F50CC36BEA1
:10B2480053E37B3FEC5738BE4DD17B3F6CE339BEAF
:10B2580020BF7B3FCF6E3BBECDAC7B3F15FA3CBEDB
:10B26800539A7B3F3E853EBEB2877B3F491040BE26
:10B27800EA747B3F379B41BEFC617B3F072643BE98
:10B28800E74E7B3FB9B044BEAB3B7B3F4D3B46BE30
:10B2980048287B3FC2C547BEBE147B3F185049BEF5
:10B2A8000E017B3F4FDA4ABE37ED7A3F67644CBEEA
:10B2B8003AD97A3F60EE4DBE16C57A3F38784FBE10
:10B2C800CBB07A3FF10151BE599C7A3F898B52BE6F
:10B2D800C1877A3F011554BE02737A3F589E55BE06
:10B2E8001C5E7A3F8F2757BE10497A3FA4B058BEDC
:10B2F800DD337A3F97395ABE841E7A3F6AC25BBEF5
:10B3080004097A3F1A4B5DBE5EF3793FA8D35EBE4F
:10B3180091DD793F135C60BE9DC7793F5CE461BEF7
:10B3280083B1793F836C63BE439B793F86F464BEE7
:10B33800DC84793F667C66BE4E6E793F220468BE27
:10B348009A57793FBA8B69BEC040793F2F136BBEBD
:10B35800BF29793F7F9A6CBE9812793FAB216EBEA8
:10B368004AFB783FB2A86FBED6E3783F942F71BEF0
:10B378003BCC783F51B672BE7BB4783FE83C74BE94
:10B38800939C783F5AC375BE8684783FA64977BE9A
:10B39800526C783FCCCF78BEF853783FCB557ABE05
:10B3A800773B783FA4DB7BBED122783F56617DBED8
:10B3B800040A783FE1E67EBE10F1773F223680BE70
:10B3C800F7D7773FC0F880BEB7BE773F4ABB81BE8C
:10B3D80051A5773FC07D82BEC58B773F224083BE93
:10B3E8001372773F700284BE3A58773FAAC484BE6E
:10B3F8003C3E773FCE8685BE1724773FDF4886BE22
:10B40800CC09773FDA0A87BE5BEF763FC1CC87BEAF
:10B41800C4D4763F938E88BE07BA763F505089BE13
:10B42800249F763FF8118ABE1B84763F8AD38ABE52
:10B43800EC68763F07958BBE974D763F6E568CBE6F
:10B448001B32763FC0178DBE7A16763FFCD88DBE6C
:10B45800B3FA753F229A8EBEC6DE753F325B8FBE49
:10B46800B3C2753F2C1C90BE7BA6753F10DD90BE05
:10B478001C8A753FDD9D91BE976D753F945E92BEA7
:10B48800ED50753F351F93BE1D34753FBFDF93BE2A
:10B498002717753F31A094BE0BFA743F8D6095BE97
:10B4A800C9DC743FD22096BE62BF743F00E196BEED
:10B4B800D5A1743F17A197BE2284743F166198BE28
:10B4C8004966743FFE2099BE4B48743FCEE099BE52
:10B4D800272A743F86A09ABEDD0B743F27609BBE67
:10B4E8006EED733FAF1F9CBED9CE733F20DF9CBE6D
:10B4F8001FB0733F789E9DBE3F91733FB85D9EBE5F
:10B508003972733FDF1C9FBE0E53733FEEDB9FBE45
:10B51800BE33733FE59AA0BE4714733FC259A1BE1C
:10B52800ACF4723F8718A2BEEBD4723F33D7A2BEE9
:10B5380004B5723FC595A3BEF894723F3F54A4BEAC
:10B54800C774723F9F12A5BE7054723FE5D0A5BE66
:10B55800F433723F128FA6BE5213723F254DA7BE19
:10B568008CF2713F1F0BA8BE9FD1713FFEC8A8BEC9
:10B578008EB0713FC486A9BE578F713F6F44AABE73
:10B58800FB6D713F0102ABBE7A4C713F77BFABBE1A
:10B59800D42A713FD47CACBE0809713F153AADBEC0
:10B5A80017E7703F3CF7ADBE02C5703F49B4AEBE69
:10B5B800C6A2703F3A71AFBE6680703F102EB0BE13
:10B5C800E15D703FCBEAB0BE373B703F6BA7B1BEC1
:10B5D8006718703FEF63B2BE73F56F3F5820B3BE74
:10B5E8005AD26F3FA5DCB3BE1BAF6F3FD698B4BE2F
:10B5F800B88B6F3FEC54B5BE30686F3FE610B6BEEF
:10B6080083446F3FC3CCB6BEB0206F3F8488B7BEBB
:10B61800BAFC6E3F2A44B8BE9ED86E3FB2FFB8BE91
:10B628005DB46E3F1EBBB9BEF88F6E3F6E76BABE74
:10B638006D6B6E3FA031BBBEBE466E3FB6ECBBBE67
:10B64800EB216E3FAFA7BCBEF2FC6D3F8B62BDBE67
:10B65800D5D76D3F4A1DBEBE93B26D3FEBD7BEBE78
:10B668002D8D6D3F6F92BFBEA1676D3FD54CC0BE9B
:10B67800F2416D3F1E07C1BE1D1C6D3F48C1C1BED2
:10B6880024F66C3F557BC2BE07D06C3F4435C3BE21
:10B69800C5A96C3F15EFC3BE5E836C3FC8A8C4BE86
:10B6A800D45C6C3F5C62C5BE24366C3FD21BC6BE00
:10B6B800500F6C3F29D5C6BE58E86B3F628EC7BE97
:10B6C8003BC16B3F7C47C8BEFB996B3F7700C9BE47
:10B6D80095726B3F53B9C9BE0C4B6B3F1072CABE13
:10B6E8005E236B3FAE2ACBBE8CFB6A3F2CE3CBBEFE
:10B6F80095D36A3F8B9BCCBE7BAB6A3FCA53CDBE0A
:10B708003C836A3FEA0BCEBED95A6A3FEAC3CEBE33
:10B7180052326A3FCA7BCFBEA7096A3F8A33D0BE7E
:10B72800D7E0693F2AEBD0BEE4B7693FAAA2D1BEF1
:10B73800CC8E693F095AD2BE9165693F4811D3BE84
:10B74800323C693F67C8D3BEAE12693F647FD4BE3E
:10B7580007E9683F4136D5BE3CBF683FFDECD5BE22
:10B768004C95683F99A3D6BE396B683F135AD7BE2C
:10B778000341683F6B10D8BEA816683FA3C6D8BE61
:10B788002AEC673FB97CD9BE87C1673FAD32DABEC4
:10B79800C196673F80E8DABED86B673F319EDBBE53
:10B7A800CA40673FC153DCBE9915673F2E09DDBE0D
:10B7B80045EA663F79BEDDBECCBE663FA273DEBEFB
:10B7C8003093663FA928DFBE7167663F8DDDDFBE17
:10B7D8008E3B663F4F92E0BE880F663FEE46E1BE65
:10B7E8005EE3653F6AFBE1BE10B7653FC4AFE2BEEA
:10B7F800A08A653FFA63E3BE0B5E653F0E18E4BEA0
:10B808005431653FFECBE4BE7904653FCB7FE5BE8E
:10B818007BD7643F7533E6BE59AA643FFBE6E6BEB4
:10B82800147D643F5D9AE7BEAC4F643F9C4DE8BE13
:10B838002122643FB700E9BE73F4633FAEB3E9BEAB
:10B84800A1C6633F8166EABEAC98633F3019EBBE80
:10B85800956A633FBBCBEBBE5A3C633F217EECBE8F
:10B86800FC0D633F6330EDBE7BDF623F80E2EDBEDF
:10B87800D7B0623F7994EEBE1082623F4C46EFBE6D
:10B888002653623FFBF7EFBE1A24623F85A9F0BE3C
:10B89800EAF4613FEA5AF1BE98C5613F290CF2BE4D
:10B8A8002296613F43BDF2BE8A66613F386EF3BEA1
:10B8B800D036613F071FF4BEF206613FB1CFF4BE38
:10B8C800F2D6603F3580F5BECFA6603F9330F6BE16
:10B8D8008976603FCBE0F6BE2146603FDC90F7BE3C
:10B8E8009615603FC840F8BEE9E45F3F8EF0F8BEA9
:10B8F80019B45F3F2DA0F9BE27835F3FA54FFABE5D
:10B9080012525F3FF7FEFABEDB205F3F22AEFBBE5E
:10B9180081EF5E3F275DFCBE05BE5E3F040CFDBEA9
:10B92800678C5E3FBBBAFDBEA65A5E3F4A69FEBE43
:10B93800C3285E3FB217FFBEBEF65D3FF3C5FFBE2C
:10B9480097C45D3F063A00BF4D925D3FFF9000BF30
:10B95800E15F5D3FE4E700BF532D5D3FB53E01BFAA
:10B96800A3FA5C3F739501BFD1C75C3F1CEC01BFD4
:10B97800DD945C3FB14202BFC7615C3F329902BFB0
:10B988008E2E5C3F9FEF02BF34FB5B3FF84503BF41
:10B99800B8C75B3F3D9C03BF1A945B3F6DF203BF82
:10B9A8005A605B3F894804BF792C5B3F919E04BF76
:10B9B80075F85A3F84F404BF50C45A3F624A05BF21
:10B9C80009905A3F2CA005BFA05B5A3FE2F505BF7E
:10B9D80016275A3F824B06BF6AF2593F0EA106BF8F
:10B9E8009CBD593F86F606BFAD88593FE84B07BF57
:10B9F8009C53593F36A107BF6A1E593F6FF607BFD0
:10BA080017E9583F924B08BFA1B3583FA1A008BF00
:10BA18000B7E583F9BF508BF5348583F7F4A09BFE4
:10BA28007912583F4E9F09BF7FDC573F09F409BF81
:10BA380063A6573FAD480ABF2670573F3D9D0ABFD2
:10BA4800C739573FB7F10ABF4803573F1C460BBFDA
:10BA5800A7CC563F6B9A0BBFE595563FA5EE0BBF9B
:10BA6800025F563FC9420CBFFE27563FD7960CBF10
:10BA7800D9F0553FD0EA0CBF93B9553FB33E0DBF3F
:10BA88002C82553F81920DBFA44A553F38E60DBF21
:10BA9800FB12553FDA390EBF31DB543F658D0EBFBF
:10BAA80047A3543FDBE00EBF3B6B543F3B340FBF13
:10BAB8000F33543F84870FBFC3FA533FB8DA0FBF21
:10BAC80055C2533FD52D10BFC789533FDC8010BFE7
:10BAD8001851533FCDD310BF4918533FA72611BF64
:10BAE80059DF523F6B7911BF49A6523F19CC11BF9C
:10BAF800186D523FB01E12BFC633523F307112BF8D
:10BB080054FA513F9AC312BFC2C0513FEE1513BF3A
:10BB18001087513F2A6813BF3D4D513F50BA13BF9C
:10BB28004A13513F5F0C14BF37D9503F585E14BFBA
:10BB3800039F503F39B014BFAF64503F040215BF94
:10BB48003B2A503FB75315BFA8EF4F3F54A515BF29
:10BB5800F4B44F3FD9F615BF1F7A4F3F474816BF79
:10BB68002B3F4F3F9F9916BF17044F3FDFEA16BF81
:10BB7800E4C84E3F073C17BF908D4E3F188D17BF46
:10BB88001C524E3F12DE17BF89164E3FF52E18BFC6
:10BB9800D5DA4D3FC07F18BF029F4D3F73D018BF05
:10BBA80010634D3F0F2119BFFD264D3F947119BFFA
:10BBB800CBEA4C3F00C219BF79AE4C3F55121ABFB1
:10BBC80008724C3F93621ABF78354C3FB8B21ABF1F
:10BBD800C7F84B3FC6021BBFF8BB4B3FBB521BBF4E
:10BBE800097F4B3F99A21BBFFA414B3F5FF21BBF36
:10BBF800CC044B3F0C421CBF7FC74A3FA2911CBFDD
:10BC0800138A4A3F1FE11CBF874C4A3F84301DBF3F
:10BC1800DC0E4A3FD17F1DBF12D1493F06CF1DBF61
:10BC28002993493F221E1EBF2155493F266D1EBF3D
:10BC3800FA16493F12BC1EBFB3D8483FE50A1FBFDA
:10BC48004E9A483F9F591FBFCA5B483F41A81FBF34
:10BC5800271D483FCBF61FBF65DE473F3B4520BF4A
:10BC6800849F473F939320BF8560473FD2E120BF21
:10BC78006721473FF92F21BF2AE2463F067E21BFB1
:10BC8800CEA2463FFBCB21BF5463463FD71922BF04
:10BC9800BB23463F996722BF03E4453F43B522BF14
:10BCA8002DA4453FD30223BF3964453F4B5023BFE2
:10BCB8002624453FA99D23BFF5E3443FEEEA23BF71
:10BCC800A5A3443F1A3824BF3763443F2C8524BFBB
:10BCD800AB22443F25D224BF00E2433F041F25BFC7
:10BCE80038A1433FCB6B25BF5160433F77B825BF91
:10BCF8004C1F433F0A0526BF29DE423F845126BF19
:10BD0800E89C423FE39D26BF895B423F2AEA26BF63
:10BD18000B1A423F563627BF70D8413F688227BF6B
:10BD2800B796413F61CE27BFE154413F401A28BF33
:10BD3800EC12413F056628BFDAD0403FB0B128BFBA
:10BD4800A98E403F41FD28BF5C4C403FB84829BF01
:10BD5800F009403F159429BF67C73F3F57DF29BF08
:10BD6800C0843F3F802A2ABFFC413F3F8E752ABFCF
:10BD78001BFF3E3F82C02ABF1BBC3E3F5B0B2BBF55
:10BD8800FF783E3F1B562BBFC5353E3FBFA02BBF9C
:10BD98006EF23D3F4AEB2BBFF9AE3D3FB9352CBFA4
:10BDA800676B3D3F0F802CBFB8273D3F49CA2CBF6A
:10BDB800ECE33C3F69142DBF03A03C3F6F5E2DBFF1
:10BDC800FC5B3C3F59A82DBFD9173C3F29F22DBF3A
:10BDD80098D33B3FDE3B2EBF3B8F3B3F78852EBF42
:10BDE800C14A3B3FF7CE2EBF29063B3F5B182FBF0A
:10BDF80075C13A3FA5612FBFA47C3A3FD3AA2FBF94
:10BE0800B7373A3FE6F32FBFACF2393FDE3C30BFDD
:10BE180085AD393FBB8530BF4268393F7CCE30BFE6
:10BE2800E122393F221731BF65DD383FAD5F31BFB1
:10BE3800CB97383F1DA831BF1652383F71F031BF3C
:10BE4800430C383FAA3832BF55C6373FC78032BF88
:10BE58004A80373FC9C832BF233A373FAF1033BF94
:10BE6800DFF3363F7A5833BF7FAD363F29A033BF63
:10BE78000467363FBCE733BF6C20363F342F34BFEE
:10BE8800B8D9353F8F7634BFE792353FCFBD34BF41
:10BE9800FB4B353FF30435BFF304353FFB4B35BF50
:10BEA800CFBD343FE79235BF8F76343FB8D935BF21
:10BEB800342F343F6C2036BFBCE7333F046736BFAE
:10BEC80029A0333F7FAD36BF7A58333FDFF336BF03
:10BED800AF10333F233A37BFC9C8323F4A8037BF14
:10BEE800C780323F55C637BFAA38323F430C38BFE8
:10BEF80071F0313F165238BF1DA8313FCB9738BF7C
:10BF0800AD5F313F65DD38BF2217313FE12239BFD0
:10BF18007CCE303F426839BFBB85303F85AD39BFE5
:10BF2800DE3C303FACF239BFE6F32F3FB7373ABFBC
:10BF3800D3AA2F3FA47C3ABFA5612F3F75C13ABF52
:10BF48005B182F3F29063BBFF7CE2E3FC14A3BBFA8
:10BF580078852E3F3B8F3BBFDE3B2E3F98D33BBFC0
:10BF680029F22D3FD9173CBF59A82D3FFC5B3CBF98
:10BF78006F5E2D3F03A03CBF69142D3FECE33CBF2F
:10BF880049CA2C3FB8273DBF0F802C3F676B3DBF88
:10BF9800B9352C3FF9AE3DBF4AEB2B3F6EF23DBFA2
:10BFA800BFA02B3FC5353EBF1B562B3FFF783EBF7A
:10BFB8005B0B2B3F1BBC3EBF82C02A3F1BFF3EBF13
:10BFC8008E752A3FFC413FBF802A2A3FC0843FBF6D
:10BFD80057DF293F67C73FBF1594293FF00940BF86
:10BFE800B848293F5C4C40BF41FD283FA98E40BF5F
:10BFF800B0B1283FDAD040BF0566283FEC1241BFF8
:10C00800401A283FE15441BF61CE273FB79641BF50
:10C018006882273F70D841BF5636273F0B1A42BF68
:10C028002AEA263F895B42BFE39D263FE89C42BF40
:10C038008451263F29DE42BF0A05263F4C1F43BFD5
:10C0480077B8253F516043BFCB6B253F38A143BF2D
:10C05800041F253F00E243BF25D2243FAB2244BF43
:10C068002C85243F376344BF1A38243FA5A344BF17
:10C07800EEEA233FF5E344BFA99D233F262445BFAD
:10C088004B50233F396445BFD302233F2DA445BFFE
:10C0980043B5223F03E445BF9967223FBB2346BF10
:10C0A800D719223F546346BFFBCB213FCEA246BFE0
:10C0B800067E213F2AE246BFF92F213F672147BF6D
:10C0C800D2E1203F856047BF9393203F849F47BFBD
:10C0D8003B45203F65DE47BFCBF61F3F271D48BFC6
:10C0E80041A81F3FCA5B48BF9F591F3F4E9A48BF90
:10C0F800E50A1F3FB3D848BF12BC1E3FFA1649BF16
:10C10800266D1E3F215549BF221E1E3F299349BF58
:10C1180006CF1D3F12D149BFD17F1D3FDC0E4ABF5C
:10C1280084301D3F874C4ABF1FE11C3F138A4ABF1A
:10C13800A2911C3F7FC74ABF0C421C3FCC044BBF97
:10C148005FF21B3FFA414BBF99A21B3F097F4BBFD0
:10C15800BB521B3FF8BB4BBFC6021B3FC7F84BBFC8
:10C16800B8B21A3F78354CBF93621A3F08724CBF79
:10C1780055121A3F79AE4CBF00C2193FCBEA4CBFEB
:10C188009471193FFD264DBF0F21193F10634DBF14
:10C1980073D0183F029F4DBFC07F183FD5DA4DBFFF
:10C1A800F52E183F89164EBF12DE173F1C524EBFA0
:10C1B800188D173F908D4EBF073C173FE4C84EBF00
:10C1C800DFEA163F17044FBF9F99163F2B3F4FBF1B
:10C1D8004748163F1F7A4FBFD9F6153FF4B44FBFF3
:10C1E80054A5153FA8EF4FBFB753153F3B2A50BF83
:10C1F8000402153FAF6450BF39B0143F039F50BFCE
:10C20800585E143F37D950BF5F0C143F4A1351BFD3
:10C2180050BA133F3D4D51BF2A68133F108751BF95
:10C22800EE15133FC2C051BF9AC3123F54FA51BF13
:10C238003071123FC63352BFB01E123F186D52BF45
:10C2480019CC113F49A652BF6B79113F59DF52BF34
:10C25800A726113F491853BFCDD3103F185153BFDC
:10C26800DC80103FC78953BFD52D103F55C253BF3F
:10C27800B8DA0F3FC3FA53BF84870F3F0F3354BF59
:10C288003B340F3F3B6B54BFDBE00E3F47A354BF2B
:10C29800658D0E3F31DB54BFDA390E3FFB1255BFB7
:10C2A80038E60D3FA44A55BF81920D3F2C8255BFF9
:10C2B800B33E0D3F93B955BFD0EA0C3FD9F055BFF7
:10C2C800D7960C3FFE2756BFC9420C3F025F56BFA8
:10C2D800A5EE0B3FE59556BF6B9A0B3FA7CC56BF13
:10C2E8001C460B3F480357BFB7F10A3FC73957BF32
:10C2F8003D9D0A3F267057BFAD480A3F63A657BF0A
:10C3080009F4093F7FDC57BF4E9F093F791258BF98
:10C318007F4A093F534858BF9BF5083F0B7E58BFDB
:10C32800A1A0083FA1B358BF924B083F17E958BFD7
:10C338006FF6073F6A1E59BF36A1073F9C5359BF86
:10C34800E84B073FAD8859BF86F6063F9CBD59BFED
:10C358000EA1063F6AF259BF824B063F16275ABF05
:10C36800E2F5053FA05B5ABF2CA0053F09905ABFD4
:10C37800624A053F50C45ABF84F4043F75F85ABF57
:10C38800919E043F792C5BBF8948043F5A605BBF8C
:10C398006DF2033F1A945BBF3D9C033FB8C75BBF78
:10C3A800F845033F34FB5BBF9FEF023F8E2E5CBF17
:10C3B8003299023FC7615CBFB142023FDD945CBF66
:10C3C8001CEC013FD1C75CBF7395013FA3FA5CBF6A
:10C3D800B53E013F532D5DBFE4E7003FE15F5DBF20
:10C3E800FF90003F4D925DBF063A003F97C45DBF86
:10C3F800F3C5FF3EBEF65DBFB217FF3EC3285EBF62
:10C408004A69FE3EA65A5EBFBBBAFD3E678C5EBF58
:10C41800040CFD3E05BE5EBF275DFC3E81EF5EBF9E
:10C4280022AEFB3EDB205FBFF7FEFA3E12525FBF33
:10C43800A54FFA3E27835FBF2DA0F93E19B45FBF11
:10C448008EF0F83EE9E45FBFC840F83E961560BF3D
:10C45800DC90F73E214660BFCBE0F63E897660BFB0
:10C468009330F63ECFA660BF3580F53EF2D660BF6A
:10C47800B1CFF43EF20661BF071FF43ED03661BF6C
:10C48800386EF33E8A6661BF43BDF23E229661BFB5
:10C49800290CF23E98C561BFEA5AF13EEAF461BF41
:10C4A80085A9F03E1A2462BFFBF7EF3E265362BF10
:10C4B8004C46EF3E108262BF7994EE3ED7B062BF21
:10C4C80080E2ED3E7BDF62BF6330ED3EFC0D63BF73
:10C4D800217EEC3E5A3C63BFBBCBEB3E956A63BF03
:10C4E8003019EB3EAC9863BF8166EA3EA1C663BFD4
:10C4F800AEB3E93E73F463BFB700E93E212264BFDF
:10C508009C4DE83EAC4F64BF5D9AE73E147D64BF26
:10C51800FBE6E63E59AA64BF7533E63E7BD764BFA7
:10C52800CB7FE53E790465BFFECBE43E543165BF61
:10C538000E18E43E0B5E65BFFA63E33EA08A65BF52
:10C54800C4AFE23E10B765BF6AFBE13E5EE365BF7C
:10C55800EE46E13E880F66BF4F92E03E8E3B66BFD7
:10C568008DDDDF3E716766BFA928DF3E309366BF69
:10C57800A273DE3ECCBE66BF79BEDD3E45EA66BF2D
:10C588002E09DD3E991567BFC153DC3ECA4067BF1F
:10C59800319EDB3ED86B67BF80E8DA3EC19667BF45
:10C5A800AD32DA3E87C167BFB97CD93E2AEC67BF96
:10C5B800A3C6D83EA81668BF6B10D83E034168BF13
:10C5C800135AD73E396B68BF99A3D63E4C9568BFBE
:10C5D800FDECD53E3CBF68BF4136D53E07E968BF94
:10C5E800647FD43EAE1269BF67C8D33E323C69BF90
:10C5F8004811D33E916569BF095AD23ECC8E69BFB6
:10C60800AAA2D13EE4B769BF2AEBD03ED7E069BF02
:10C618008A33D03EA7096ABFCA7BCF3E52326ABF6F
:10C62800EAC3CE3ED95A6ABFEA0BCE3E3C836ABF04
:10C63800CA53CD3E7BAB6ABF8B9BCC3E95D36ABFBA
:10C648002CE3CB3E8CFB6ABFAE2ACB3E5E236BBF8E
:10C658001072CA3E0C4B6BBF53B9C93E95726BBF83
:10C668007700C93EFB996BBF7C47C83E3BC16BBF97
:10C67800628EC73E58E86BBF29D5C63E500F6CBFC7
:10C68800D21BC63E24366CBF5C62C53ED45C6CBF10
:10C69800C8A8C43E5E836CBF15EFC33EC5A96CBF76
:10C6A8004435C33E07D06CBF557BC23E24F66CBFF1
:10C6B80048C1C13E1D1C6DBF1E07C13EF2416DBF82
:10C6C800D54CC03EA1676DBF6F92BF3E2D8D6DBF2B
:10C6D800EBD7BE3E93B26DBF4A1DBE3ED5D76DBFE8
:10C6E8008B62BD3EF2FC6DBFAFA7BC3EEB216EBFB7
:10C6F800B6ECBB3EBE466EBFA031BB3E6D6B6EBF97
:10C708006E76BA3EF88F6EBF1EBBB93E5DB46EBF83
:10C71800B2FFB83E9ED86EBF2A44B83EBAFC6EBF80
:10C728008488B73EB0206FBFC3CCB63E83446FBF8A
:10C73800E610B63E30686FBFEC54B53EB88B6FBF9D
:10C74800D698B43E1BAF6FBFA5DCB33E5AD26FBFBD
:10C758005820B33E73F56FBFEF63B23E671870BFE2
:10C768006BA7B13E373B70BFCBEAB03EE15D70BF0F
:10C77800102EB03E668070BF3A71AF3EC6A270BF41
:10C7880049B4AE3E02C570BF3CF7AD3E17E770BF77
:10C79800153AAD3E080971BFD47CAC3ED42A71BFAE
:10C7A80077BFAB3E7A4C71BF0102AB3EFB6D71BFE8
:10C7B8006F44AA3E578F71BFC486A93E8EB071BF21
:10C7C800FEC8A83E9FD171BF1F0BA83E8CF271BF57
:10C7D800254DA73E521372BF128FA63EF43372BF87
:10C7E800E5D0A53E705472BF9F12A53EC77472BFB4
:10C7F8003F54A43EF89472BFC595A33E04B572BFDA
:10C8080033D7A23EEBD472BF8718A23EACF472BFF6
:10C81800C259A13E471473BFE59AA03EBE3373BF09
:10C82800EEDB9F3E0E5373BFDF1C9F3E397273BF12
:10C83800B85D9E3E3F9173BF789E9D3E1FB073BF0B
:10C8480020DF9C3ED9CE73BFAF1F9C3E6EED73BFF9
:10C8580027609B3EDD0B74BF86A09A3E272A74BFD3
:10C86800CEE0993E4B4874BFFE20993E496674BF9E
:10C878001661983E228474BF17A1973ED5A174BF54
:10C8880000E1963E62BF74BFD220963EC9DC74BFF9
:10C898008D60953E0BFA74BF31A0943E271775BF83
:10C8A800BFDF933E1D3475BF351F933EED5075BFF6
:10C8B800945E923E976D75BFDD9D913E1C8A75BF53
:10C8C80010DD903E7BA675BF2C1C903EB3C275BF91
:10C8D800325B8F3EC6DE75BF229A8E3EB3FA75BFB5
:10C8E800FCD88D3E7A1676BFC0178D3E1B3276BFB8
:10C8F8006E568C3E974D76BF07958B3EEC6876BF9B
:10C908008AD38A3E1B8476BFF8118A3E249F76BF5D
:10C918005050893E07BA76BF938E883EC4D476BFFE
:10C92800C1CC873E5BEF76BFDA0A873ECC0977BF7A
:10C93800DF48863E172477BFCE86853E3C3E77BFCC
:10C94800AAC4843E3A5877BF7002843E137277BFF8
:10C958002240833EC58B77BFC07D823E51A577BFFD
:10C968004ABB813EB7BE77BFC0F8803EF7D777BFD6
:10C978002236803E10F177BFE1E67E3E040A78BF9A
:10C9880056617D3ED12278BFA4DB7B3E773B78BFE2
:10C99800CB557A3EF85378BFCCCF783E526C78BFEF
:10C9A800A649773E868478BF5AC3753E939C78BF64
:10C9B800E83C743E7BB478BF51B6723E3BCC78BF3E
:10C9C800942F713ED6E378BFB2A86F3E4AFB78BF7A
:10C9D800AB216E3E981279BF7F9A6C3EBF2979BF12
:10C9E8002F136B3EC04079BFBA8B693E9A5779BF07
:10C9F8002204683E4E6E79BF667C663EDC8479BF51
:10CA080086F4643E439B79BF836C633E83B179BFF0
:10CA18005CE4613E9DC779BF135C603E91DD79BFE0
:10CA2800A8D35E3E5EF379BF1A4B5D3E04097ABF18
:10CA38006AC25B3E841E7ABF97395A3EDD337ABF9D
:10CA4800A4B0583E10497ABF8F27573E1C5E7ABF64
:10CA5800589E553E02737ABF0115543EC1877ABF6E
:10CA6800898B523E599C7ABFF101513ECBB07ABFB7
:10CA780038784F3E16C57ABF60EE4D3E3AD97ABF38
:10CA880067644C3E37ED7ABF4FDA4A3E0E017BBFF2
:10CA98001850493EBE147BBFC2C5473E48287BBFDD
:10CAA8004D3B463EAB3B7BBFB9B0443EE74E7BBFF8
:10CAB8000726433EFC617BBF379B413EEA747BBF40
:10CAC8004910403EB2877BBF3E853E3E539A7BBFAE
:10CAD80015FA3C3ECDAC7BBFCF6E3B3E20BF7BBF43
:10CAE8006CE3393E4DD17BBFEC57383E53E37BBFF7
:10CAF80050CC363E31F57BBF9840353EE9067CBFC9
:10CB0800C4B4333E7A187CBFD428323EE5297CBFB2
:10CB1800C99C303E283B7CBFA2102F3E444C7CBFB2
:10CB280061842D3E3A5D7CBF04F82B3E086E7CBFC5
:10CB38008D6B2A3EB07E7CBFFCDE283E318F7CBFE9
:10CB48005152273E8A9F7CBF8CC5253EBDAF7CBF16
:10CB5800AD38243EC9BF7CBFB6AB223EAECF7CBF4A
:10CB6800A51E213E6CDF7CBF7B911F3E03EF7CBF7F
:10CB780038041E3E73FE7CBFDE761C3EBC0D7DBFB6
:10CB88006BE91A3EDD1C7DBFE05B193ED82B7DBFEB
:10CB98003DCE173EAC3A7DBF8340163E59497DBF16
:10CBA800B2B2143EDE577DBFCA24133E3D667DBF38
:10CBB800CC96113E74747DBFB708103E85827DBF48
:10CBC8008B7A0E3E6E907DBF4AEC0C3E309E7DBF48
:10CBD800F35D0B3ECCAB7DBF86CF093E40B97DBF30
:10CBE8000541083E8CC67DBF6EB2063EB2D37DBFFE
:10CBF800C223053EB1E07DBF0295033E88ED7DBFAF
:10CC08002E06023E38FA7DBF4577003EC2067EBF3B
:10CC180092D0FD3D24137EBF73B2FA3D5E1F7EBFE6
:10CC28002C94F73D722B7EBFC075F43D5E377EBFF6
:10CC38002E57F13D23437EBF7638EE3DC14E7EBF71
:10CC48009A19EB3D385A7EBF9AFAE73D88657EBF50
:10CC580076DBE43DB0707EBF2EBCE13DB17B7EBF8C
:10CC6800C49CDE3D8B867EBF377DDB3D3D917EBF1C
:10CC7800895DD83DC99B7EBFB93DD53D2DA67EBFF8
:10CC8800C81DD23D69B07EBFB7FDCE3D7FBA7EBF1D
:10CC980086DDCB3D6DC47EBF36BDC83D34CE7EBF7C
:10CCA800C69CC53DD4D77EBF397CC23D4CE17EBF12
:10CCB8008D5BBF3D9DEA7EBFC33ABC3DC7F37EBFD7
:10CCC800DD19B93DC9FC7EBFDAF8B53DA4057FBFC3
:10CCD800BBD7B23D580E7FBF80B6AF3DE4167FBFCD
:10CCE8002B95AC3D491F7FBFBA73A93D87277FBFEE
:10CCF8003052A63D9D2F7FBF8C30A33D8D377FBF1F
:10CD0800CF0EA03D543F7FBFF9EC9C3DF4467FBF5A
:10CD18000ACB993D6D4E7FBF05A9963DBF557FBF94
:10CD2800E786933DE95C7FBFB464903DEC637FBFC9
:10CD38006A428D3DC76A7FBF0A208A3D7B717FBFEB
:10CD480094FD863D08787FBF0ADB833D6D7E7FBFFB
:10CD58006CB8803DAB847FBF742B7B3DC28A7FBF9C
:10CD6800E9E5743DB1907FBF38A06E3D78967FBFEE
:10CD7800625A683D189C7FBF6814623D91A17FBFCD
:10CD88004CCE5B3DE3A67FBF0E88553D0DAC7FBF03
:10CD9800AF414F3D0FB17FBF2FFB483DEAB57FBF85
:10CDA80091B4423D9EBA7FBFD56D3C3D2ABF7FBF3F
:10CDB800FC26363D8FC37FBF07E02F3DCCC77FBF22
:10CDC800F698293DE2CB7FBFCC51233DD1CF7FBF21
:10CDD800880A1D3D98D37FBF2CC3163D37D77FBF28
:10CDE800B87B103DAFDA7FBF2F340A3D00DE7FBF2E
:10CDF80090EC033D29E17FBFB949FB3C2BE47FBFA1
:10CE08002DBAEE3C05E77FBF7B2AE23CB8E97FBF3D
:10CE1800A69AD53C43EC7FBFB00AC93CA7EE7FBFBA
:10CE28009B7ABC3CE3F07FBF69EAAF3CF8F27FBF76
:10CE38001C5AA33CE6F47FBFB6C9963CACF67FBF4C
:10CE480038398A3C4AF87FBF4B517B3CC1F97FBFD8
:10CE58000030623C11FB7FBF900E493C39FC7FBF1C
:10CE680002ED2F3C39FD7FBF59CB163C13FE7FBF27
:10CE78003053FB3BC4FE7FBF890FC93B4EFF7FBFCA
:10CE8800C1CB963BB1FF7FBFC70F493BECFF7FBFCC
:10CE9800D40FC93A000080BF00000000ECFF7FBF3C
:10CEA800D40FC9BAB1FF7FBFC70F49BB4EFF7FBFC1
:10CEB800C1CB96BBC4FE7FBF890FC9BB13FE7FBF22
:10CEC8003053FBBB39FD7FBF59CB16BC39FC7FBF44
:10CED80002ED2FBC11FB7FBF900E49BCC1F97FBF8B
:10CEE800003062BC4AF87FBF4B517BBCACF67FBFB9
:10CEF80038398ABCE6F47FBFB6C996BCF8F27FBF62
:10CF08001C5AA3BCE3F07FBF69EAAFBCA7EE7FBFA2
:10CF18009B7ABCBC43EC7FBFB00AC9BCB8E97FBFF1
:10CF2800A69AD5BC05E77FBF7B2AE2BC2BE47FBF6E
:10CF38002DBAEEBC29E17FBFB949FBBC00DE7FBF3B
:10CF480090EC03BDAFDA7FBF2F340ABD37D77FBF60
:10CF5800B87B10BD98D37FBF2CC316BDD1CF7FBF80
:10CF6800880A1DBDE2CB7FBFCC5123BDCCC77FBF94
:10CF7800F69829BD8FC37FBF07E02FBD2ABF7FBFAB
:10CF8800FC2636BD9EBA7FBFD56D3CBDEAB57FBFD6
:10CF980091B442BD0FB17FBF2FFB48BD0DAC7FBF21
:10CFA800AF414FBDE3A67FBF0E8855BD91A17FBF9E
:10CFB8004CCE5BBD189C7FBF681462BD78967FBF5E
:10CFC800625A68BDB1907FBF38A06EBDC28A7FBF6C
:10CFD800E9E574BDAB847FBF742B7BBD6D7E7FBFDD
:10CFE8006CB880BD08787FBF0ADB83BD7B717FBFCB
:10CFF80094FD86BDC76A7FBF0A208ABDEC637FBFE8
:10D008006A428DBDE95C7FBFB46490BDBF557FBFE8
:10D01800E78693BD6D4E7FBF05A996BDF4467FBFD9
:10D028000ACB99BD543F7FBFF9EC9CBD8D377FBFBC
:10D03800CF0EA0BD9D2F7FBF8C30A3BD87277FBF9C
:10D048003052A6BD491F7FBFBA73A9BDE4167FBF82
:10D058002B95ACBD580E7FBF80B6AFBDA4057FBF72
:10D06800BBD7B2BDC9FC7EBFDAF8B5BDC7F37EBF7A
:10D07800DD19B9BD9DEA7EBFC33ABCBD4CE17EBF98
:10D088008D5BBFBDD4D77EBF397CC2BD34CE7EBFD9
:10D09800C69CC5BD6DC47EBF36BDC8BD7FBA7EBF48
:10D0A80086DDCBBD69B07EBFB7FDCEBD2DA67EBFE8
:10D0B800C81DD2BDC99B7EBFB93DD5BD3D917EBFC0
:10D0C800895DD8BD8B867EBF377DDBBDB17B7EBFDA
:10D0D800C49CDEBDB0707EBF2EBCE1BD88657EBF3E
:10D0E80076DBE4BD385A7EBF9AFAE7BDC14E7EBFF3
:10D0F8009A19EBBD23437EBF7638EEBD5E377EBFFF
:10D108002E57F1BD722B7EBFC075F4BD5E1F7EBF6A
:10D118002C94F7BD24137EBF73B2FABDC2067EBF3E
:10D1280092D0FDBD38FA7DBF457700BE88ED7DBF42
:10D138002E0602BEB1E07DBF029503BEB2D37DBF0D
:10D14800C22305BE8CC67DBF6EB206BE40B97DBF88
:10D15800054108BECCAB7DBF86CF09BE309E7DBFE2
:10D16800F35D0BBE6E907DBF4AEC0CBE85827DBF21
:10D178008B7A0EBE74747DBFB70810BE3D667DBF46
:10D18800CC9611BEDE577DBFCA2413BE59497DBF58
:10D19800B2B214BEAC3A7DBF834016BED82B7DBF59
:10D1A8003DCE17BEDD1C7DBFE05B19BEBC0D7DBF4B
:10D1B8006BE91ABE73FE7CBFDE761CBE03EF7CBF34
:10D1C80038041EBE6CDF7CBF7B911FBEAECF7CBF18
:10D1D800A51E21BEC9BF7CBFB6AB22BEBDAF7CBFFA
:10D1E800AD3824BE8A9F7CBF8CC525BE318F7CBFDD
:10D1F800515227BEB07E7CBFFCDE28BE086E7CBFC5
:10D208008D6B2ABE3A5D7CBF04F82BBE444C7CBFB4
:10D2180061842DBE283B7CBFA2102FBEE5297CBFB0
:10D22800C99C30BE7A187CBFD42832BEE9067CBFC0
:10D23800C4B433BE31F57BBF984035BE53E37BBFE2
:10D2480050CC36BE4DD17BBFEC5738BE20BF7BBF1C
:10D258006CE339BECDAC7BBFCF6E3BBE539A7BBF70
:10D2680015FA3CBEB2877BBF3E853EBEEA747BBFE3
:10D27800491040BEFC617BBF379B41BEE74E7BBF78
:10D28800072643BEAB3B7BBFB9B044BE48287BBF33
:10D298004D3B46BEBE147BBFC2C547BE0E017BBF19
:10D2A800185049BE37ED7ABF4FDA4ABE3AD97ABF2D
:10D2B80067644CBE16C57ABF60EE4DBECBB07ABF70
:10D2C80038784FBE599C7ABFF10151BEC1877ABFE9
:10D2D800898B52BE02737ABF011554BE1C5E7ABF99
:10D2E800589E55BE10497ABF8F2757BEDD337ABF87
:10D2F800A4B058BE841E7ABF97395ABE04097ABFB3
:10D308006AC25BBE5EF379BF1A4B5DBE91DD79BF21
:10D31800A8D35EBE9DC779BF135C60BE83B179BFD9
:10D328005CE461BE439B79BF836C63BEDC8479BFD8
:10D3380086F464BE4E6E79BF667C66BE9A5779BF26
:10D34800220468BEC04079BFBA8B69BEBF2979BFC5
:10D358002F136BBE981279BF7F9A6CBE4AFB78BFB9
:10D36800AB216EBED6E378BFB2A86FBE3BCC78BF08
:10D37800942F71BE7BB478BF51B672BE939C78BFB0
:10D38800E83C74BE868478BF5AC375BE526C78BFB9
:10D39800A64977BEF85378BFCCCF78BE773B78BF25
:10D3A800CB557ABED12278BFA4DB7BBE040A78BFF6
:10D3B80056617DBE10F177BFE1E67EBEF7D777BF35
:10D3C800223680BEB7BE77BFC0F880BE51A577BFF2
:10D3D8004ABB81BEC58B77BFC07D82BE137277BF43
:10D3E800224083BE3A5877BF700284BE3C3E77BF66
:10D3F800AAC484BE172477BFCE8685BECC0977BF62
:10D40800DF4886BE5BEF76BFDA0A87BEC4D476BF34
:10D41800C1CC87BE07BA76BF938E88BE249F76BFDD
:10D42800505089BE1B8476BFF8118ABEEC6876BF5F
:10D438008AD38ABE974D76BF07958BBE1B3276BFBF
:10D448006E568CBE7A1676BFC0178DBEB3FA75BFFE
:10D45800FCD88DBEC6DE75BF229A8EBEB3C275BF1C
:10D46800325B8FBE7BA675BF2C1C90BE1C8A75BF15
:10D4780010DD90BE976D75BFDD9D91BEED5075BFF7
:10D48800945E92BE1D3475BF351F93BE271775BFB6
:10D49800BFDF93BE0BFA74BF31A094BEC9DC74BF62
:10D4A8008D6095BE62BF74BFD22096BED5A174BFF1
:10D4B80000E196BE228474BF17A197BE496674BF67
:10D4C800166198BE4B4874BFFE2099BE272A74BFC8
:10D4D800CEE099BEDD0B74BF86A09ABE6EED73BF19
:10D4E80027609BBED9CE73BFAF1F9CBE1FB073BF52
:10D4F80020DF9CBE3F9173BF789E9DBE397273BF7B
:10D50800B85D9EBE0E5373BFDF1C9FBEBE3373BF94
:10D51800EEDB9FBE471473BFE59AA0BEACF472BFA2
:10D52800C259A1BEEBD472BF8718A2BE04B572BFA0
:10D5380033D7A2BEF89472BFC595A3BEC77472BF95
:10D548003F54A4BE705472BF9F12A5BEF43372BF7D
:10D55800E5D0A5BE521372BF128FA6BE8CF271BF62
:10D56800254DA7BE9FD171BF1F0BA8BE8EB071BF3E
:10D57800FEC8A8BE578F71BFC486A9BEFB6D71BF18
:10D588006F44AABE7A4C71BF0102ABBED42A71BFE8
:10D5980077BFABBE080971BFD47CACBE17E770BFBC
:10D5A800153AADBE02C570BF3CF7ADBEC6A270BF8E
:10D5B80049B4AEBE668070BF3A71AFBEE15D70BF60
:10D5C800102EB0BE373B70BFCBEAB0BE671870BF35
:10D5D8006BA7B1BE73F56FBFEF63B2BE5AD26FBF10
:10D5E8005820B3BE1BAF6FBFA5DCB3BEB88B6FBFEF
:10D5F800D698B4BE30686FBFEC54B5BE83446FBFD5
:10D60800E610B6BEB0206FBFC3CCB6BEBAFC6EBFC4
:10D618008488B7BE9ED86EBF2A44B8BE5DB46EBFBC
:10D62800B2FFB8BEF88F6EBF1EBBB9BE6D6B6EBFC2
:10D638006E76BABEBE466EBFA031BBBEEB216EBFD2
:10D64800B6ECBBBEF2FC6DBFAFA7BCBED5D76DBFF5
:10D658008B62BDBE93B26DBF4A1DBEBE2D8D6DBF20
:10D66800EBD7BEBEA1676DBF6F92BFBEF2416DBF63
:10D67800D54CC0BE1D1C6DBF1E07C1BE24F66CBFB5
:10D6880048C1C1BE07D06CBF557BC2BEC5A96CBF1F
:10D698004435C3BE5E836CBF15EFC3BED45C6CBF9C
:10D6A800C8A8C4BE24366CBF5C62C5BE500F6CBF30
:10D6B800D21BC6BE58E86BBF29D5C6BE3BC16BBFDF
:10D6C800628EC7BEFB996BBF7C47C8BE95726BBFA5
:10D6D8007700C9BE0C4B6BBF53B9C9BE5E236BBF85
:10D6E8001072CABE8CFB6ABFAE2ACBBE95D36ABF86
:10D6F8002CE3CBBE7BAB6ABF8B9BCCBE3C836ABFA3
:10D70800CA53CDBED95A6ABFEA0BCEBE52326ABFDF
:10D71800EAC3CEBEA7096ABFCA7BCFBED7E069BF3E
:10D728008A33D0BEE4B769BF2AEBD0BECC8E69BFBE
:10D73800AAA2D1BE916569BF095AD2BE323C69BF5F
:10D748004811D3BEAE1269BF67C8D3BE07E968BF28
:10D75800647FD4BE3CBF68BF4136D5BE4C9568BF18
:10D76800FDECD5BE396B68BF99A3D6BE034168BF2F
:10D77800135AD7BEA81668BF6B10D8BE2AEC67BF6D
:10D78800A3C6D8BE87C167BFB97CD9BEC19667BFDB
:10D79800AD32DABED86B67BF80E8DABECA4067BF71
:10D7A800319EDBBE991567BFC153DCBE45EA66BF33
:10D7B8002E09DDBECCBE66BF79BEDDBE309366BF26
:10D7C800A273DEBE716766BFA928DFBE8E3B66BF47
:10D7D8008DDDDFBE880F66BF4F92E0BE5EE365BF9A
:10D7E800EE46E1BE10B765BF6AFBE1BEA08A65BF21
:10D7F800C4AFE2BE0B5E65BFFA63E3BE543165BFDA
:10D808000E18E4BE790465BFFECBE4BE7BD764BFC7
:10D81800CB7FE5BE59AA64BF7533E6BE147D64BFED
:10D82800FBE6E6BEAC4F64BF5D9AE7BE212264BF4B
:10D838009C4DE8BE73F463BFB700E9BEA1C663BFE1
:10D84800AEB3E9BEAC9863BF8166EABE956A63BFB2
:10D858003019EBBE5A3C63BFBBCBEBBEFC0D63BFBC
:10D86800217EECBE7BDF62BF6330EDBED7B062BF06
:10D8780080E2EDBE108262BF7994EEBE265362BF8D
:10D888004C46EFBE1A2462BFFBF7EFBEEAF461BF55
:10D8980085A9F0BE98C561BFEA5AF1BE229661BF5C
:10D8A800290CF2BE8A6661BF43BDF2BED03661BFA5
:10D8B800386EF3BEF20661BF071FF4BEF2D660BF32
:10D8C800B1CFF4BECFA660BF3580F5BE897660BF04
:10D8D8009330F6BE214660BFCBE0F6BE961560BF1A
:10D8E800DC90F7BEE9E45FBFC840F8BE19B45FBF7B
:10D8F8008EF0F8BE27835FBF2DA0F9BE12525FBF1E
:10D90800A54FFABEDB205FBFF7FEFABE81EF5EBF10
:10D9180022AEFBBE05BE5EBF275DFCBE678C5EBF48
:10D92800040CFDBEA65A5EBFBBBAFDBEC3285EBFCF
:10D938004A69FEBEBEF65DBFB217FFBE97C45DBFA3
:10D94800F3C5FFBE4D925DBF063A00BFE15F5DBF04
:10D95800FF9000BF532D5DBFE4E700BFA3FA5CBF93
:10D96800B53E01BFD1C75CBF739501BFDD945CBFF5
:10D978001CEC01BFC7615CBFB14202BF8E2E5CBF09
:10D98800329902BF34FB5BBF9FEF02BFB8C75BBFD2
:10D99800F84503BF1A945BBF3D9C03BF5A605BBF49
:10D9A8006DF203BF792C5BBF894804BF75F85ABF75
:10D9B800919E04BF50C45ABF84F404BF09905ABF53
:10D9C800624A05BFA05B5ABF2CA005BF16275ABFE5
:10D9D800E2F505BF6AF259BF824B06BF9CBD59BF2D
:10D9E8000EA106BFAD8859BF86F606BF9C5359BF26
:10D9F800E84B07BF6A1E59BF36A107BF17E958BFD2
:10DA08006FF607BFA1B358BF924B08BF0B7E58BF34
:10DA1800A1A008BF534858BF9BF508BF791258BF4B
:10DA28007F4A09BF7FDC57BF4E9F09BF63A657BF18
:10DA380009F409BF267057BFAD480ABFC73957BF99
:10DA48003D9D0ABF480357BFB7F10ABFA7CC56BFD1
:10DA58001C460BBFE59556BF6B9A0BBF025F56BFBE
:10DA6800A5EE0BBFFE2756BFC9420CBFD9F055BF64
:10DA7800D7960CBF93B955BFD0EA0CBF2C8255BFBF
:10DA8800B33E0DBFA44A55BF81920DBFFB1255BFCF
:10DA980038E60DBF31DB54BFDA390EBF47A354BF98
:10DAA800658D0EBF3B6B54BFDBE00EBF0F3354BF19
:10DAB8003B340FBFC3FA53BF84870FBF55C253BF50
:10DAC800B8DA0FBFC78953BFD52D10BF185153BF40
:10DAD800DC8010BF491853BFCDD310BF59DF52BFE8
:10DAE800A72611BF49A652BF6B7911BF186D52BF47
:10DAF80019CC11BFC63352BFB01E12BF54FA51BF62
:10DB0800307112BFC2C051BF9AC312BF108751BF34
:10DB1800EE1513BF3D4D51BF2A6813BF4A1351BFBD
:10DB280050BA13BF37D950BF5F0C14BF039F50BF03
:10DB3800585E14BFAF6450BF39B014BF3B2A50BF02
:10DB4800040215BFA8EF4FBFB75315BFF4B44FBFBA
:10DB580054A515BF1F7A4FBFD9F615BF2B3F4FBF2E
:10DB6800474816BF17044FBF9F9916BFE4C84EBF5A
:10DB7800DFEA16BF908D4EBF073C17BF1C524EBF41
:10DB8800188D17BF89164EBF12DE17BFD5DA4DBFE5
:10DB9800F52E18BF029F4DBFC07F18BF10634DBF41
:10DBA80073D018BFFD264DBF0F2119BFCBEA4CBF5C
:10DBB800947119BF79AE4CBF00C219BF08724CBF2F
:10DBC80055121ABF78354CBF93621ABFC7F84BBFBE
:10DBD800B8B21ABFF8BB4BBFC6021BBF097F4BBF09
:10DBE800BB521BBFFA414BBF99A21BBFCC044BBF12
:10DBF8005FF21BBF7FC74ABF0C421CBF138A4ABFD4
:10DC0800A2911CBF874C4ABF1FE11CBFDC0E4ABF54
:10DC180084301DBF12D149BFD17F1DBF299349BF91
:10DC280006CF1DBF215549BF221E1EBFFA1649BF88
:10DC3800266D1EBFB3D848BF12BC1EBF4E9A48BF40
:10DC4800E50A1FBFCA5B48BF9F591FBF271D48BFB2
:10DC580041A81FBF65DE47BFCBF61FBF849F47BFE4
:10DC68003B4520BF856047BF939320BF672147BFCF
:10DC7800D2E120BF2AE246BFF92F21BFCEA246BF7C
:10DC8800067E21BF546346BFFBCB21BFBB2346BFE3
:10DC9800D71922BF03E445BF996722BF2DA445BF0A
:10DCA80043B522BF396445BFD30223BF262445BFED
:10DCB8004B5023BFF5E344BFA99D23BFA5A344BF91
:10DCC800EEEA23BF376344BF1A3824BFAB2244BFF0
:10DCD8002C8524BF00E243BF25D224BF38A143BF0F
:10DCE800041F25BF516043BFCB6B25BF4C1F43BFEB
:10DCF80077B825BF29DE42BF0A0526BFE89C42BF88
:10DD0800845126BF895B42BFE39D26BF0B1A42BFE1
:10DD18002AEA26BF70D841BF563627BFB79641BFFB
:10DD2800688227BFE15441BF61CE27BFEC1241BFD3
:10DD3800401A28BFDAD040BF056628BFA98E40BF69
:10DD4800B0B128BF5C4C40BF41FD28BFF00940BFBF
:10DD5800B84829BF67C73FBF159429BFC0843FBFD4
:10DD680057DF29BFFC413FBF802A2ABF1BFF3EBFA8
:10DD78008E752ABF1BBC3EBF82C02ABFFF783EBF3C
:10DD88005B0B2BBFC5353EBF1B562BBF6EF23DBF8D
:10DD9800BFA02BBFF9AE3DBF4AEB2BBF676B3DBFA2
:10DDA800B9352CBFB8273DBF0F802CBFECE33CBF73
:10DDB80049CA2CBF03A03CBF69142DBFFC5B3CBF04
:10DDC8006F5E2DBFD9173CBF59A82DBF98D33BBF55
:10DDD80029F22DBF3B8F3BBFDE3B2EBFC14A3BBF65
:10DDE80078852EBF29063BBFF7CE2EBF75C13ABF37
:10DDF8005B182FBFA47C3ABFA5612FBFB7373ABFC6
:10DE0800D3AA2FBFACF239BFE6F32FBF85AD39BF18
:10DE1800DE3C30BF426839BFBB8530BFE12239BF25
:10DE28007CCE30BF65DD38BF221731BFCB9738BFF6
:10DE3800AD5F31BF165238BF1DA831BF430C38BF84
:10DE480071F031BF55C637BFAA3832BF4A8037BFD5
:10DE5800C78032BF233A37BFC9C832BFDFF336BFE6
:10DE6800AF1033BF7FAD36BF7A5833BF046736BFB4
:10DE780029A033BF6C2036BFBCE733BFB8D935BF44
:10DE8800342F34BFE79235BF8F7634BFFB4B35BF95
:10DE9800CFBD34BFF30435BFF30435BFCFBD34BFA6
:10DEA800FB4B35BF8F7634BFE79235BF342F34BF75
:10DEB800B8D935BFBCE733BF6C2036BF29A033BF04
:10DEC800046736BF7A5833BF7FAD36BFAF1033BF54
:10DED800DFF336BFC9C832BF233A37BFC78032BF66
:10DEE8004A8037BFAA3832BF55C637BF71F031BF35
:10DEF800430C38BF1DA831BF165238BFAD5F31BFC4
:10DF0800CB9738BF221731BF65DD38BF7CCE30BF15
:10DF1800E12239BFBB8530BF426839BFDE3C30BF24
:10DF280085AD39BFE6F32FBFACF239BFD3AA2FBFF7
:10DF3800B7373ABFA5612FBFA47C3ABF5B182FBF84
:10DF480075C13ABFF7CE2EBF29063BBF78852EBFD5
:10DF5800C14A3BBFDE3B2EBF3B8F3BBF29F22DBFE3
:10DF680098D33BBF59A82DBFD9173CBF6F5E2DBFB3
:10DF7800FC5B3CBF69142DBF03A03CBF49CA2CBF42
:10DF8800ECE33CBF0F802CBFB8273DBFB9352CBF91
:10DF9800676B3DBF4AEB2BBFF9AE3DBFBFA02BBFA0
:10DFA8006EF23DBF1B562BBFC5353EBF5B0B2BBF6B
:10DFB800FF783EBF82C02ABF1BBC3EBF8E752ABFFA
:10DFC8001BFF3EBF802A2ABFFC413FBF57DF29BF46
:10DFD800C0843FBF159429BF67C73FBFB84829BF52
:10DFE800F00940BF41FD28BF5C4C40BFB0B128BF1D
:10DFF800A98E40BF056628BFDAD040BF401A28BFA7
:10E00800EC1241BF61CE27BFE15441BF688227BFF0
:10E01800B79641BF563627BF70D841BF2AEA26BFF8
:10E028000B1A42BFE39D26BF895B42BF845126BFBE
:10E03800E89C42BF0A0526BF29DE42BF77B825BF44
:10E048004C1F43BFCB6B25BF516043BF041F25BF87
:10E0580038A143BF25D224BF00E243BF2C8524BF8B
:10E06800AB2244BF1A3824BF376344BFEEEA23BF4C
:10E07800A5A344BFA99D23BFF5E344BF4B5023BFCD
:10E08800262445BFD30223BF396445BF43B522BF09
:10E098002DA445BF996722BF03E445BFD71922BF06
:10E0A800BB2346BFFBCB21BF546346BF067E21BFBF
:10E0B800CEA246BFF92F21BF2AE246BFD2E120BF38
:10E0C800672147BF939320BF856047BF3B4520BF6B
:10E0D800849F47BFCBF61FBF65DE47BF41A81FBF60
:10E0E800271D48BF9F591FBFCA5B48BFE50A1FBF0E
:10E0F8004E9A48BF12BC1EBFB3D848BF266D1EBF7C
:10E10800FA1649BF221E1EBF215549BF06CF1DBFA3
:10E11800299349BFD17F1DBF12D149BF84301DBF8C
:10E12800DC0E4ABF1FE11CBF874C4ABFA2911CBF2F
:10E13800138A4ABF0C421CBF7FC74ABF5FF21BBF8E
:10E14800CC044BBF99A21BBFFA414BBFBB521BBFAC
:10E15800097F4BBFC6021BBFF8BB4BBFB8B21ABF83
:10E16800C7F84BBF93621ABF78354CBF55121ABF18
:10E1780008724CBF00C219BF79AE4CBF947119BF69
:10E18800CBEA4CBF0F2119BFFD264DBF73D018BF76
:10E1980010634DBFC07F18BF029F4DBFF52E18BF3B
:10E1A800D5DA4DBF12DE17BF89164EBF188D17BFBF
:10E1B8001C524EBF073C17BF908D4EBFDFEA16BFFB
:10E1C800E4C84EBF9F9916BF17044FBF474816BFF4
:10E1D8002B3F4FBFD9F615BF1F7A4FBF54A515BFA8
:10E1E800F4B44FBFB75315BFA8EF4FBF040215BF14
:10E1F8003B2A50BF39B014BFAF6450BF585E14BF3C
:10E20800039F50BF5F0C14BF37D950BF50BA13BF1C
:10E218004A1351BF2A6813BF3D4D51BFEE1513BFB6
:10E22800108751BF9AC312BFC2C051BF307112BF0D
:10E2380054FA51BFB01E12BFC63352BF19CC11BF1A
:10E24800186D52BF6B7911BF49A652BFA72611BFDF
:10E2580059DF52BFCDD310BF491853BFDC8010BF60
:10E26800185153BFD52D10BFC78953BFB8DA0FBF98
:10E2780055C253BF84870FBFC3FA53BF3B340FBF88
:10E288000F3354BFDBE00EBF3B6B54BF658D0EBF31
:10E2980047A354BFDA390EBF31DB54BF38E60DBF90
:10E2A800FB1255BF81920DBFA44A55BFB33E0DBFA7
:10E2B8002C8255BFD0EA0CBF93B955BFD7960CBF77
:10E2C800D9F055BFC9420CBFFE2756BFA5EE0BBFFC
:10E2D800025F56BF6B9A0BBFE59556BF1C460BBF36
:10E2E800A7CC56BFB7F10ABF480357BF3D9D0ABF29
:10E2F800C73957BFAD480ABF267057BF09F409BFD1
:10E3080063A657BF4E9F09BF7FDC57BF7F4A09BF2F
:10E31800791258BF9BF508BF534858BFA1A008BF42
:10E328000B7E58BF924B08BFA1B358BF6FF607BF0B
:10E3380017E958BF36A107BF6A1E59BFE84B07BF88
:10E348009C5359BF86F606BFAD8859BF0EA106BFBC
:10E358009CBD59BF824B06BF6AF259BFE2F505BFA3
:10E3680016275ABF2CA005BFA05B5ABF624A05BF3B
:10E3780009905ABF84F404BF50C45ABF919E04BF89
:10E3880075F85ABF894804BF792C5BBF6DF203BF8B
:10E398005A605BBF3D9C03BF1A945BBFF84503BF3F
:10E3A800B8C75BBF9FEF02BF34FB5BBF329902BFA8
:10E3B8008E2E5CBFB14202BFC7615CBF1CEC01BFBF
:10E3C800DD945CBF739501BFD1C75CBFB53E01BF8B
:10E3D800A3FA5CBFE4E700BF532D5DBFFF9000BF09
:10E3E800E15F5DBF063A00BF4D925DBFF3C5FFBE5A
:10E3F80097C45DBFB217FFBEBEF65DBF4A69FEBED9
:10E40800C3285EBFBBBAFDBEA65A5EBF040CFDBEE4
:10E41800678C5EBF275DFCBE05BE5EBF22AEFBBE3D
:10E4280081EF5EBFF7FEFABEDB205FBFA54FFABEE5
:10E4380012525FBF2DA0F9BE27835FBF8EF0F8BED2
:10E4480019B45FBFC840F8BEE9E45FBFDC90F7BE0F
:10E45800961560BFCBE0F6BE214660BF9330F6BE8E
:10E46800897660BF3580F5BECFA660BFB1CFF4BE58
:10E47800F2D660BF071FF4BEF20661BF386EF3BE66
:10E48800D03661BF43BDF2BE8A6661BF290CF2BEB9
:10E49800229661BFEA5AF1BE98C561BF85A9F0BE50
:10E4A800EAF461BFFBF7EFBE1A2462BF4C46EFBE29
:10E4B800265362BF7994EEBE108262BF80E2EDBE41
:10E4C800D7B062BF6330EDBE7BDF62BF217EECBE9A
:10E4D800FC0D63BFBBCBEBBE5A3C63BF3019EBBE30
:10E4E800956A63BF8166EABEAC9863BFAEB3E9BE06
:10E4F800A1C663BFB700E9BE73F463BF9C4DE8BE15
:10E50800212264BF5D9AE7BEAC4F64BFFBE6E6BE5E
:10E51800147D64BF7533E6BE59AA64BFCB7FE5BEE0
:10E528007BD764BFFECBE4BE790465BF0E18E4BE9A
:10E53800543165BFFA63E3BE0B5E65BFC4AFE2BE8C
:10E54800A08A65BF6AFBE1BE10B765BFEE46E1BEB3
:10E558005EE365BF4F92E0BE880F66BF8DDDDFBE0C
:10E568008E3B66BFA928DFBE716766BFA273DEBE99
:10E57800309366BF79BEDDBECCBE66BF2E09DDBE58
:10E5880045EA66BFC153DCBE991567BF319EDBBE45
:10E59800CA4067BF80E8DABED86B67BFAD32DABE63
:10E5A800C19667BFB97CD9BE87C167BFA3C6D8BEAD
:10E5B8002AEC67BF6B10D8BEA81668BF135AD7BE1F
:10E5C800034168BF99A3D6BE396B68BFFDECD5BEC1
:10E5D8004C9568BF4136D5BE3CBF68BF647FD4BE8A
:10E5E80007E968BF67C8D3BEAE1269BF4811D3BE7A
:10E5F800323C69BF095AD2BE916569BFAAA2D1BE91
:10E60800CC8E69BF2AEBD0BEE4B769BF8A33D0BECF
:10E61800D7E069BFCA7BCFBEA7096ABFEAC3CEBE2F
:10E6280052326ABFEA0BCEBED95A6ABFCA53CDBEB0
:10E638003C836ABF8B9BCCBE7BAB6ABF2CE3CBBE53
:10E6480095D36ABFAE2ACBBE8CFB6ABF1072CABE16
:10E658005E236BBF53B9C9BE0C4B6BBF7700C9BEF5
:10E6680095726BBF7C47C8BEFB996BBF628EC7BEF5
:10E678003BC16BBF29D5C6BE58E86BBFD21BC6BE0F
:10E68800500F6CBF5C62C5BE24366CBFC8A8C4BE40
:10E69800D45C6CBF15EFC3BE5E836CBF4435C3BE8C
:10E6A800C5A96CBF557BC2BE07D06CBF48C1C1BEEF
:10E6B80024F66CBF1E07C1BE1D1C6DBFD54CC0BE65
:10E6C800F2416DBF6F92BFBEA1676DBFEBD7BEBEF3
:10E6D8002D8D6DBF4A1DBEBE93B26DBF8B62BDBE90
:10E6E800D5D76DBFAFA7BCBEF2FC6DBFB6ECBBBE45
:10E6F800EB216EBFA031BBBEBE466EBF6E76BABE02
:10E708006D6B6EBF1EBBB9BEF88F6EBFB2FFB8BED1
:10E718005DB46EBF2A44B8BE9ED86EBF8488B7BEAB
:10E72800BAFC6EBFC3CCB6BEB0206FBFE610B6BE93
:10E7380083446FBFEC54B5BE30686FBFD698B4BE83
:10E74800B88B6FBFA5DCB3BE1BAF6FBF5820B3BE7D
:10E758005AD26FBFEF63B2BE73F56FBF6BA7B1BE7E
:10E76800671870BFCBEAB0BE373B70BF102EB0BE83
:10E77800E15D70BF3A71AFBE668070BF49B4AEBE8E
:10E78800C6A270BF3CF7ADBE02C570BF153AADBE9C
:10E7980017E770BFD47CACBE080971BF77BFABBEAA
:10E7A800D42A71BF0102ABBE7A4C71BF6F44AABEB6
:10E7B800FB6D71BFC486A9BE578F71BFFEC8A8BEC6
:10E7C8008EB071BF1F0BA8BE9FD171BF254DA7BECC
:10E7D8008CF271BF128FA6BE521372BFE5D0A5BED0
:10E7E800F43372BF9F12A5BE705472BF3F54A4BECB
:10E7F800C77472BFC595A3BEF89472BF33D7A2BEC3
:10E8080004B572BF8718A2BEEBD472BFC259A1BEAD
:10E81800ACF472BFE59AA0BE471473BFEEDB9FBE8F
:10E82800BE3373BFDF1C9FBE0E5373BFB85D9EBE61
:10E83800397273BF789E9DBE3F9173BF20DF9CBE27
:10E848001FB073BFAF1F9CBED9CE73BF27609BBEDE
:10E858006EED73BF86A09ABEDD0B74BFCEE099BE85
:10E86800272A74BFFE2099BE4B4874BF166198BE14
:10E87800496674BF17A197BE228474BF00E196BE93
:10E88800D5A174BFD22096BE62BF74BF8D6095BEFD
:10E89800C9DC74BF31A094BE0BFA74BFBFDF93BE4E
:10E8A800271775BF351F93BE1D3475BF945E92BE82
:10E8B800ED5075BFDD9D91BE976D75BF10DD90BEA3
:10E8C8001C8A75BF2C1C90BE7BA675BF325B8FBEA1
:10E8D800B3C275BF229A8EBEC6DE75BFFCD88DBE88
:10E8E800B3FA75BFC0178DBE7A1676BF6E568CBE4A
:10E8F8001B3276BF07958BBE974D76BF8AD38ABEEB
:10E90800EC6876BFF8118ABE1B8476BF505089BE6A
:10E91800249F76BF938E88BE07BA76BFC1CC87BEC8
:10E92800C4D476BFDA0A87BE5BEF76BFDF4886BEFF
:10E93800CC0977BFCE8685BE172477BFAAC484BE0C
:10E948003C3E77BF700284BE3A5877BF224083BEF0
:10E95800137277BFC07D82BEC58B77BF4ABB81BEAD
:10E9680051A577BFC0F880BEB7BE77BF223680BE3C
:10E97800F7D777BFE1E67EBE10F177BF56617DBE5F
:10E98800040A78BFA4DB7BBED12278BFCB557ABE00
:10E99800773B78BFCCCF78BEF85378BFA64977BE0F
:10E9A800526C78BF5AC375BE868478BFE83C74BE83
:10E9B800939C78BF51B672BE7BB478BF942F71BE5A
:10E9C8003BCC78BFB2A86FBED6E378BFAB216EBE92
:10E9D8004AFB78BF7F9A6CBE981279BF2F136BBE23
:10E9E800BF2979BFBA8B69BEC04079BF220468BE0F
:10E9F8009A5779BF667C66BE4E6E79BF86F464BE50
:10EA0800DC8479BF836C63BE439B79BF5CE461BEE1
:10EA180083B179BF135C60BE9DC779BFA8D35EBEC2
:10EA280091DD79BF1A4B5DBE5EF379BF6AC25BBEEA
:10EA380004097ABF97395ABE841E7ABFA4B058BE5B
:10EA4800DD337ABF8F2757BE10497ABF589E55BE0F
:10EA58001C5E7ABF011554BE02737ABF898B52BE01
:10EA6800C1877ABFF10151BE599C7ABF38784FBE31
:10EA7800CBB07ABF60EE4DBE16C57ABF67644CBE98
:10EA88003AD97ABF4FDA4ABE37ED7ABF185049BE35
:10EA98000E017BBFC2C547BEBE147BBF4D3B46BE01
:10EAA80048287BBFB9B044BEAB3B7BBF072643BEFB
:10EAB800E74E7BBF379B41BEFC617BBF491040BE20
:10EAC800EA747BBF3E853EBEB2877BBF15FA3CBE6B
:10EAD800539A7BBFCF6E3BBECDAC7BBF6CE339BED8
:10EAE80020BF7BBFEC5738BE4DD17BBF50CC36BE64
:10EAF80053E37BBF984035BE31F57BBFC4B433BE0A
:10EB0800E9067CBFD42832BE7A187CBFC99C30BEC7
:10EB1800E5297CBFA2102FBE283B7CBF61842DBE97
:10EB2800444C7CBF04F82BBE3A5D7CBF8D6B2ABE7B
:10EB3800086E7CBFFCDE28BEB07E7CBF515227BE6B
:10EB4800318F7CBF8CC525BE8A9F7CBFAD3824BE63
:10EB5800BDAF7CBFB6AB22BEC9BF7CBFA51E21BE60
:10EB6800AECF7CBF7B911FBE6CDF7CBF38041EBE5E
:10EB780003EF7CBFDE761CBE73FE7CBF6BE91ABE5A
:10EB8800BC0D7DBFE05B19BEDD1C7DBF3DCE17BE51
:10EB9800D82B7DBF834016BEAC3A7DBFB2B214BE3F
:10EBA80059497DBFCA2413BEDE577DBFCC9611BE1E
:10EBB8003D667DBFB70810BE74747DBF8B7A0EBEEC
:10EBC80085827DBF4AEC0CBE6E907DBFF35D0BBEA7
:10EBD800309E7DBF86CF09BECCAB7DBF054108BE48
:10EBE80040B97DBF6EB206BE8CC67DBFC22305BECE
:10EBF800B2D37DBF029503BEB1E07DBF2E0602BE33
:10EC080088ED7DBF457700BE38FA7DBF92D0FDBD47
:10EC1800C2067EBF73B2FABD24137EBF2C94F7BD23
:10EC28005E1F7EBFC075F4BD722B7EBF2E57F1BD2F
:10EC38005E377EBF7638EEBD23437EBF9A19EBBDA3
:10EC4800C14E7EBF9AFAE7BD385A7EBF76DBE4BD77
:10EC580088657EBF2EBCE1BDB0707EBFC49CDEBDA2
:10EC6800B17B7EBF377DDBBD8B867EBF895DD8BD1E
:10EC78003D917EBFB93DD5BDC99B7EBFC81DD2BDE4
:10EC88002DA67EBFB7FDCEBD69B07EBF86DDCBBDEC
:10EC98007FBA7EBF36BDC8BD6DC47EBFC69CC5BD2C
:10ECA80034CE7EBF397CC2BDD4D77EBF8D5BBFBD9D
:10ECB8004CE17EBFC33ABCBD9DEA7EBFDD19B9BD3C
:10ECC800C7F37EBFDAF8B5BDC9FC7EBFBBD7B2BDFE
:10ECD800A4057FBF80B6AFBD580E7FBF2B95ACBDD6
:10ECE800E4167FBFBA73A9BD491F7FBF3052A6BDC6
:10ECF80087277FBF8C30A3BD9D2F7FBFCF0EA0BDC0
:10ED08008D377FBFF9EC9CBD543F7FBF0ACB99BDBF
:10ED1800F4467FBF05A996BD6D4E7FBFE78693BDBC
:10ED2800BF557FBFB46490BDE95C7FBF6A428DBDAB
:10ED3800EC637FBF0A208ABDC76A7FBF94FD86BD8A
:10ED48007B717FBF0ADB83BD08787FBF6CB880BD4D
:10ED58006D7E7FBF742B7BBDAB847FBFE9E574BD3F
:10ED6800C28A7FBF38A06EBDB1907FBF625A68BDAE
:10ED780078967FBF681462BD189C7FBF4CCE5BBD80
:10ED880091A17FBF0E8855BDE3A67FBFAF414FBDA0
:10ED98000DAC7FBF2FFB48BD0FB17FBF91B442BD03
:10EDA800EAB57FBFD56D3CBD9EBA7FBFFC2636BD98
:10EDB8002ABF7FBF07E02FBD8FC37FBFF69829BD4D
:10EDC800CCC77FBFCC5123BDE2CB7FBF880A1DBD16
:10EDD800D1CF7FBF2CC316BD98D37FBFB87B10BDE2
:10EDE80037D77FBF2F340ABDAFDA7FBF90EC03BDA2
:10EDF80000DE7FBFB949FBBC29E17FBF2DBAEEBC5D
:10EE08002BE47FBF7B2AE2BC05E77FBFA69AD5BC6F
:10EE1800B8E97FBFB00AC9BC43EC7FBF9B7ABCBCD2
:10EE2800A7EE7FBF69EAAFBCE3F07FBF1C5AA3BC63
:10EE3800F8F27FBFB6C996BCE6F47FBF38398ABC02
:10EE4800ACF67FBF4B517BBC4AF87FBF003062BC39
:10EE5800C1F97FBF900E49BC11FB7FBF02ED2FBCEB
:10EE680039FC7FBF59CB16BC39FD7FBF3053FBBB84
:10EE780013FE7FBF890FC9BBC4FE7FBFC1CB96BB42
:10EE88004EFF7FBFC70F49BBB1FF7FBFD40FC9BAC1
:10EE9800ECFF7FBF00000080000080BFD40FC93A9C
:10EEA800ECFF7FBFC70F493BB1FF7FBFC1CB963B8C
:10EEB8004EFF7FBF890FC93BC4FE7FBF3053FB3B6A
:10EEC80013FE7FBF59CB163C39FD7FBF02ED2F3CA7
:10EED80039FC7FBF900E493C11FB7FBF0030623C7C
:10EEE800C1F97FBF4B517B3C4AF87FBF38398A3C18
:10EEF800ACF67FBFB6C9963CE6F47FBF1C5AA33C6C
:10EF0800F8F27FBF69EAAF3CE3F07FBF9B7ABC3C75
:10EF1800A7EE7FBFB00AC93C43EC7FBFA69AD53C99
:10EF2800B8E97FBF7B2AE23C05E77FBF2DBAEE3CFC
:10EF38002BE47FBFB949FB3C29E17FBF90EC033D3F
:10EF480000DE7FBF2F340A3DAFDA7FBFB87B103DAC
:10EF580037D77FBF2CC3163D98D37FBF880A1D3D86
:10EF6800D1CF7FBFCC51233DE2CB7FBFF698293D5F
:10EF7800CCC77FBF07E02F3D8FC37FBFFC26363D40
:10EF88002ABF7FBFD56D3C3D9EBA7FBF91B4423D3D
:10EF9800EAB57FBF2FFB483D0FB17FBFAF414F3D63
:10EFA8000DAC7FBF0E88553DE3A67FBF4CCE5B3DC1
:10EFB80091A17FBF6814623D189C7FBF625A683D6B
:10EFC80078967FBF38A06E3DB1907FBFE9E5743D6C
:10EFD800C28A7FBF742B7B3DAB847FBF6CB8803DFA
:10EFE8006D7E7FBF0ADB833D08787FBF94FD863D39
:10EFF8007B717FBF0A208A3DC76A7FBF6A428D3D09
:10F00800EC637FBFB464903DE95C7FBFE786933DC6
:10F01800BF557FBF05A9963D6D4E7FBF0ACB993D71
:10F02800F4467FBFF9EC9C3D543F7FBFCF0EA03D17
:10F038008D377FBF8C30A33D9D2F7FBF3052A63DBB
:10F0480087277FBFBA73A93D491F7FBF2B95AC3D6A
:10F05800E4167FBF80B6AF3D580E7FBFBBD7B23D29
:10F06800A4057FBFDAF8B53DC9FC7EBFDD19B93DFF
:10F07800C7F37EBFC33ABC3D9DEA7EBF8D5BBF3DF3
:10F088004CE17EBF397CC23DD4D77EBFC69CC53D0E
:10F0980034CE7EBF36BDC83D6DC47EBF86DDCB3D58
:10F0A8007FBA7EBFB7FDCE3D69B07EBFC81DD23DD9
:10F0B8002DA67EBFB93DD53DC99B7EBF895DD83D94
:10F0C8003D917EBF377DDB3D8B867EBFC49CDE3D98
:10F0D800B17B7EBF2EBCE13DB0707EBF76DBE43DE8
:10F0E80088657EBF9AFAE73D385A7EBF9A19EB3D8C
:10F0F800C14E7EBF7638EE3D23437EBF2E57F13D8D
:10F108005E377EBFC075F43D722B7EBF2C94F73DF1
:10F118005E1F7EBF73B2FA3D24137EBF92D0FD3DC1
:10F12800C2067EBF4577003E38FA7DBF2E06023EF6
:10F1380088ED7DBF0295033EB1E07DBFC223053E49
:10F14800B2D37DBF6EB2063E8CC67DBF0541083E78
:10F1580040B97DBF86CF093ECCAB7DBFF35D0B3E8A
:10F16800309E7DBF4AEC0C3E6E907DBF8B7A0E3E82
:10F1780085827DBFB708103E74747DBFCC96113E62
:10F188003D667DBFCA24133EDE577DBFB2B2143E32
:10F1980059497DBF8340163EAC3A7DBF3DCE173EF0
:10F1A800D82B7DBFE05B193EDD1C7DBF6BE91A3EA5
:10F1B800BC0D7DBFDE761C3E73FE7CBF38041E3E50
:10F1C80003EF7CBF7B911F3E6CDF7CBFA51E213EF9
:10F1D800AECF7CBFB6AB223EC9BF7CBFAD38243EA4
:10F1E800BDAF7CBF8CC5253E8A9F7CBF5152273E50
:10F1F800318F7CBFFCDE283EB07E7CBF8D6B2A3E03
:10F20800086E7CBF04F82B3E3A5D7CBF61842D3EBE
:10F21800444C7CBFA2102F3E283B7CBFC99C303E8B
:10F22800E5297CBFD428323E7A187CBFC4B4333E6B
:10F23800E9067CBF9840353E31F57BBF50CC363E61
:10F2480053E37BBFEC57383E4DD17BBF6CE3393E6F
:10F2580020BF7BBFCF6E3B3ECDAC7BBF15FA3C3E9B
:10F26800539A7BBF3E853E3EB2877BBF4910403EE6
:10F27800EA747BBF379B413EFC617BBF0726433E58
:10F28800E74E7BBFB9B0443EAB3B7BBF4D3B463EF0
:10F2980048287BBFC2C5473EBE147BBF1850493EB5
:10F2A8000E017BBF4FDA4A3E37ED7ABF67644C3EAA
:10F2B8003AD97ABF60EE4D3E16C57ABF38784F3ED0
:10F2C800CBB07ABFF101513E599C7ABF898B523E2F
:10F2D800C1877ABF0115543E02737ABF589E553EC6
:10F2E8001C5E7ABF8F27573E10497ABFA4B0583E9C
:10F2F800DD337ABF97395A3E841E7ABF6AC25B3EB5
:10F3080004097ABF1A4B5D3E5EF379BFA8D35E3E0F
:10F3180091DD79BF135C603E9DC779BF5CE4613EB7
:10F3280083B179BF836C633E439B79BF86F4643EA7
:10F33800DC8479BF667C663E4E6E79BF2204683EE7
:10F348009A5779BFBA8B693EC04079BF2F136B3E7D
:10F35800BF2979BF7F9A6C3E981279BFAB216E3E68
:10F368004AFB78BFB2A86F3ED6E378BF942F713EB0
:10F378003BCC78BF51B6723E7BB478BFE83C743E54
:10F38800939C78BF5AC3753E868478BFA649773E5A
:10F39800526C78BFCCCF783EF85378BFCB557A3EC5
:10F3A800773B78BFA4DB7B3ED12278BF56617D3E98
:10F3B800040A78BFE1E67E3E10F177BF2236803E30
:10F3C800F7D777BFC0F8803EB7BE77BF4ABB813E4C
:10F3D80051A577BFC07D823EC58B77BF2240833E53
:10F3E800137277BF7002843E3A5877BFAAC4843E2E
:10F3F8003C3E77BFCE86853E172477BFDF48863EE2
:10F40800CC0977BFDA0A873E5BEF76BFC1CC873E6F
:10F41800C4D476BF938E883E07BA76BF5050893ED3
:10F42800249F76BFF8118A3E1B8476BF8AD38A3E12
:10F43800EC6876BF07958B3E974D76BF6E568C3E2F
:10F448001B3276BFC0178D3E7A1676BFFCD88D3E2C
:10F45800B3FA75BF229A8E3EC6DE75BF325B8F3E09
:10F46800B3C275BF2C1C903E7BA675BF10DD903EC5
:10F478001C8A75BFDD9D913E976D75BF945E923E67
:10F48800ED5075BF351F933E1D3475BFBFDF933EEA
:10F49800271775BF31A0943E0BFA74BF8D60953E57
:10F4A800C9DC74BFD220963E62BF74BF00E1963EAD
:10F4B800D5A174BF17A1973E228474BF1661983EE8
:10F4C800496674BFFE20993E4B4874BFCEE0993E12
:10F4D800272A74BF86A09A3EDD0B74BF27609B3E27
:10F4E8006EED73BFAF1F9C3ED9CE73BF20DF9C3E2D
:10F4F8001FB073BF789E9D3E3F9173BFB85D9E3E1F
:10F50800397273BFDF1C9F3E0E5373BFEEDB9F3E05
:10F51800BE3373BFE59AA03E471473BFC259A13EDC
:10F52800ACF472BF8718A23EEBD472BF33D7A23EA9
:10F5380004B572BFC595A33EF89472BF3F54A43E6C
:10F54800C77472BF9F12A53E705472BFE5D0A53E26
:10F55800F43372BF128FA63E521372BF254DA73ED9
:10F568008CF271BF1F0BA83E9FD171BFFEC8A83E89
:10F578008EB071BFC486A93E578F71BF6F44AA3E33
:10F58800FB6D71BF0102AB3E7A4C71BF77BFAB3EDA
:10F59800D42A71BFD47CAC3E080971BF153AAD3E80
:10F5A80017E770BF3CF7AD3E02C570BF49B4AE3E29
:10F5B800C6A270BF3A71AF3E668070BF102EB03ED3
:10F5C800E15D70BFCBEAB03E373B70BF6BA7B13E81
:10F5D800671870BFEF63B23E73F56FBF5820B33E34
:10F5E8005AD26FBFA5DCB33E1BAF6FBFD698B43EEF
:10F5F800B88B6FBFEC54B53E30686FBFE610B63EAF
:10F6080083446FBFC3CCB63EB0206FBF8488B73E7B
:10F61800BAFC6EBF2A44B83E9ED86EBFB2FFB83E51
:10F628005DB46EBF1EBBB93EF88F6EBF6E76BA3E34
:10F638006D6B6EBFA031BB3EBE466EBFB6ECBB3E27
:10F64800EB216EBFAFA7BC3EF2FC6DBF8B62BD3E27
:10F65800D5D76DBF4A1DBE3E93B26DBFEBD7BE3E38
:10F668002D8D6DBF6F92BF3EA1676DBFD54CC03E5B
:10F67800F2416DBF1E07C13E1D1C6DBF48C1C13E92
:10F6880024F66CBF557BC23E07D06CBF4435C33EE1
:10F69800C5A96CBF15EFC33E5E836CBFC8A8C43E46
:10F6A800D45C6CBF5C62C53E24366CBFD21BC63EC0
:10F6B800500F6CBF29D5C63E58E86BBF628EC73E57
:10F6C8003BC16BBF7C47C83EFB996BBF7700C93E07
:10F6D80095726BBF53B9C93E0C4B6BBF1072CA3ED3
:10F6E8005E236BBFAE2ACB3E8CFB6ABF2CE3CB3EBE
:10F6F80095D36ABF8B9BCC3E7BAB6ABFCA53CD3ECA
:10F708003C836ABFEA0BCE3ED95A6ABFEAC3CE3EF3
:10F7180052326ABFCA7BCF3EA7096ABF8A33D03E3E
:10F72800D7E069BF2AEBD03EE4B769BFAAA2D13EB1
:10F73800CC8E69BF095AD23E916569BF4811D33E44
:10F74800323C69BF67C8D33EAE1269BF647FD43EFE
:10F7580007E968BF4136D53E3CBF68BFFDECD53EE2
:10F768004C9568BF99A3D63E396B68BF135AD73EEC
:10F77800034168BF6B10D83EA81668BFA3C6D83E21
:10F788002AEC67BFB97CD93E87C167BFAD32DA3E84
:10F79800C19667BF80E8DA3ED86B67BF319EDB3E13
:10F7A800CA4067BFC153DC3E991567BF2E09DD3ECD
:10F7B80045EA66BF79BEDD3ECCBE66BFA273DE3EBB
:10F7C800309366BFA928DF3E716766BF8DDDDF3ED7
:10F7D8008E3B66BF4F92E03E880F66BFEE46E13E25
:10F7E8005EE365BF6AFBE13E10B765BFC4AFE23EAA
:10F7F800A08A65BFFA63E33E0B5E65BF0E18E43E60
:10F80800543165BFFECBE43E790465BFCB7FE53E4E
:10F818007BD764BF7533E63E59AA64BFFBE6E63E74
:10F82800147D64BF5D9AE73EAC4F64BF9C4DE83ED3
:10F83800212264BFB700E93E73F463BFAEB3E93E6B
:10F84800A1C663BF8166EA3EAC9863BF3019EB3E40
:10F85800956A63BFBBCBEB3E5A3C63BF217EEC3E4F
:10F86800FC0D63BF6330ED3E7BDF62BF80E2ED3E9F
:10F87800D7B062BF7994EE3E108262BF4C46EF3E2D
:10F88800265362BFFBF7EF3E1A2462BF85A9F03EFC
:10F89800EAF461BFEA5AF13E98C561BF290CF23E0D
:10F8A800229661BF43BDF23E8A6661BF386EF33E61
:10F8B800D03661BF071FF43EF20661BFB1CFF43EF8
:10F8C800F2D660BF3580F53ECFA660BF9330F63ED6
:10F8D800897660BFCBE0F63E214660BFDC90F73EFC
:10F8E800961560BFC840F83EE9E45FBF8EF0F83E69
:10F8F80019B45FBF2DA0F93E27835FBFA54FFA3E1D
:10F9080012525FBFF7FEFA3EDB205FBF22AEFB3E1E
:10F9180081EF5EBF275DFC3E05BE5EBF040CFD3E69
:10F92800678C5EBFBBBAFD3EA65A5EBF4A69FE3E03
:10F93800C3285EBFB217FF3EBEF65DBFF3C5FF3EEC
:10F9480097C45DBF063A003F4D925DBFFF90003FF0
:10F95800E15F5DBFE4E7003F532D5DBFB53E013F6A
:10F96800A3FA5CBF7395013FD1C75CBF1CEC013F94
:10F97800DD945CBFB142023FC7615CBF3299023F70
:10F988008E2E5CBF9FEF023F34FB5BBFF845033F01
:10F99800B8C75BBF3D9C033F1A945BBF6DF2033F42
:10F9A8005A605BBF8948043F792C5BBF919E043F36
:10F9B80075F85ABF84F4043F50C45ABF624A053FE1
:10F9C80009905ABF2CA0053FA05B5ABFE2F5053F3E
:10F9D80016275ABF824B063F6AF259BF0EA1063F4F
:10F9E8009CBD59BF86F6063FAD8859BFE84B073F17
:10F9F8009C5359BF36A1073F6A1E59BF6FF6073F90
:10FA080017E958BF924B083FA1B358BFA1A0083FC0
:10FA18000B7E58BF9BF5083F534858BF7F4A093FA4
:10FA2800791258BF4E9F093F7FDC57BF09F4093F41
:10FA380063A657BFAD480A3F267057BF3D9D0A3F92
:10FA4800C73957BFB7F10A3F480357BF1C460B3F9A
:10FA5800A7CC56BF6B9A0B3FE59556BFA5EE0B3F5B
:10FA6800025F56BFC9420C3FFE2756BFD7960C3FD0
:10FA7800D9F055BFD0EA0C3F93B955BFB33E0D3FFF
:10FA88002C8255BF81920D3FA44A55BF38E60D3FE1
:10FA9800FB1255BFDA390E3F31DB54BF658D0E3F7F
:10FAA80047A354BFDBE00E3F3B6B54BF3B340F3FD3
:10FAB8000F3354BF84870F3FC3FA53BFB8DA0F3FE1
:10FAC80055C253BFD52D103FC78953BFDC80103FA7
:10FAD800185153BFCDD3103F491853BFA726113F24
:10FAE80059DF52BF6B79113F49A652BF19CC113F5C
:10FAF800186D52BFB01E123FC63352BF3071123F4D
:10FB080054FA51BF9AC3123FC2C051BFEE15133FFA
:10FB1800108751BF2A68133F3D4D51BF50BA133F5C
:10FB28004A1351BF5F0C143F37D950BF585E143F7A
:10FB3800039F50BF39B0143FAF6450BF0402153F54
:10FB48003B2A50BFB753153FA8EF4FBF54A5153FE9
:10FB5800F4B44FBFD9F6153F1F7A4FBF4748163F39
:10FB68002B3F4FBF9F99163F17044FBFDFEA163F41
:10FB7800E4C84EBF073C173F908D4EBF188D173F06
:10FB88001C524EBF12DE173F89164EBFF52E183F86
:10FB9800D5DA4DBFC07F183F029F4DBF73D0183FC5
:10FBA80010634DBF0F21193FFD264DBF9471193FBA
:10FBB800CBEA4CBF00C2193F79AE4CBF55121A3F71
:10FBC80008724CBF93621A3F78354CBFB8B21A3FDF
:10FBD800C7F84BBFC6021B3FF8BB4BBFBB521B3F0E
:10FBE800097F4BBF99A21B3FFA414BBF5FF21B3FF6
:10FBF800CC044BBF0C421C3F7FC74ABFA2911C3F9D
:10FC0800138A4ABF1FE11C3F874C4ABF84301D3FFF
:10FC1800DC0E4ABFD17F1D3F12D149BF06CF1D3F21
:10FC2800299349BF221E1E3F215549BF266D1E3FFD
:10FC3800FA1649BF12BC1E3FB3D848BFE50A1F3F9A
:10FC48004E9A48BF9F591F3FCA5B48BF41A81F3FF4
:10FC5800271D48BFCBF61F3F65DE47BF3B45203F0A
:10FC6800849F47BF9393203F856047BFD2E1203FE1
:10FC7800672147BFF92F213F2AE246BF067E213F71
:10FC8800CEA246BFFBCB213F546346BFD719223FC4
:10FC9800BB2346BF9967223F03E445BF43B5223FD4
:10FCA8002DA445BFD302233F396445BF4B50233FA2
:10FCB800262445BFA99D233FF5E344BFEEEA233F31
:10FCC800A5A344BF1A38243F376344BF2C85243F7B
:10FCD800AB2244BF25D2243F00E243BF041F253F87
:10FCE80038A143BFCB6B253F516043BF77B8253F51
:10FCF8004C1F43BF0A05263F29DE42BF8451263FD9
:10FD0800E89C42BFE39D263F895B42BF2AEA263F23
:10FD18000B1A42BF5636273F70D841BF6882273F2B
:10FD2800B79641BF61CE273FE15441BF401A283FF3
:10FD3800EC1241BF0566283FDAD040BFB0B1283F7A
:10FD4800A98E40BF41FD283F5C4C40BFB848293FC1
:10FD5800F00940BF1594293F67C73FBF57DF293FC8
:10FD6800C0843FBF802A2A3FFC413FBF8E752A3F8F
:10FD78001BFF3EBF82C02A3F1BBC3EBF5B0B2B3F15
:10FD8800FF783EBF1B562B3FC5353EBFBFA02B3F5C
:10FD98006EF23DBF4AEB2B3FF9AE3DBFB9352C3F64
:10FDA800676B3DBF0F802C3FB8273DBF49CA2C3F2A
:10FDB800ECE33CBF69142D3F03A03CBF6F5E2D3FB1
:10FDC800FC5B3CBF59A82D3FD9173CBF29F22D3FFA
:10FDD80098D33BBFDE3B2E3F3B8F3BBF78852E3F02
:10FDE800C14A3BBFF7CE2E3F29063BBF5B182F3FCA
:10FDF80075C13ABFA5612F3FA47C3ABFD3AA2F3F54
:10FE0800B7373ABFE6F32F3FACF239BFDE3C303F9D
:10FE180085AD39BFBB85303F426839BF7CCE303FA6
:10FE2800E12239BF2217313F65DD38BFAD5F313F71
:10FE3800CB9738BF1DA8313F165238BF71F0313FFC
:10FE4800430C38BFAA38323F55C637BFC780323F48
:10FE58004A8037BFC9C8323F233A37BFAF10333F54
:10FE6800DFF336BF7A58333F7FAD36BF29A0333F23
:10FE7800046736BFBCE7333F6C2036BF342F343FAE
:10FE8800B8D935BF8F76343FE79235BFCFBD343F01
:10FE9800FB4B35BFF304353FF30435BFFB4B353F10
:10FEA800CFBD34BFE792353F8F7634BFB8D9353FE1
:10FEB800342F34BF6C20363FBCE733BF0467363F6E
:10FEC80029A033BF7FAD363F7A5833BFDFF3363FC3
:10FED800AF1033BF233A373FC9C832BF4A80373FD4
:10FEE800C78032BF55C6373FAA3832BF430C383FA8
:10FEF80071F031BF1652383F1DA831BFCB97383F3C
:10FF0800AD5F31BF65DD383F221731BFE122393F90
:10FF18007CCE30BF4268393FBB8530BF85AD393FA5
:10FF2800DE3C30BFACF2393FE6F32FBFB7373A3F7C
:10FF3800D3AA2FBFA47C3A3FA5612FBF75C13A3F12
:10FF48005B182FBF29063B3FF7CE2EBFC14A3B3F68
:10FF580078852EBF3B8F3B3FDE3B2EBF98D33B3F80
:10FF680029F22DBFD9173C3F59A82DBFFC5B3C3F58
:10FF78006F5E2DBF03A03C3F69142DBFECE33C3FEF
:10FF880049CA2CBFB8273D3F0F802CBF676B3D3F48
:10FF9800B9352CBFF9AE3D3F4AEB2BBF6EF23D3F62
:10FFA800BFA02BBFC5353E3F1B562BBFFF783E3F3A
:10FFB8005B0B2BBF1BBC3E3F82C02ABF1BFF3E3FD3
:10FFC8008E752ABFFC413F3F802A2ABFC0843F3F2D
:10FFD80057DF29BF67C73F3F159429BFF009403F46
:10FFE800B84829BF5C4C403F41FD28BFA98E403F1F
:08FFF800B0B128BFDAD0403F90
:020000040801F1
:10000000056628BFEC12413F401A28BFE154413F2A
:1000100061CE27BFB796413F688227BF70D8413F66
:10002000563627BF0B1A423F2AEA26BF895B423F5A
:10003000E39D26BFE89C423F845126BF29DE423F14
:100040000A0526BF4C1F433F77B825BF5160433F89
:10005000CB6B25BF38A1433F041F25BF00E2433FC0
:1000600025D224BFAB22443F2C8524BF3763443FB5
:100070001A3824BFA5A3443FEEEA23BFF5E3443F6B
:10008000A99D23BF2624453F4B5023BF3964453FDC
:10009000D30223BF2DA4453F43B522BF03E4453F10
:1000A000996722BFBB23463FD71922BF5463463FFF
:1000B000FBCB21BFCEA2463F067E21BF2AE2463FB0
:1000C000F92F21BF6721473FD2E120BF8560473F1D
:1000D000939320BF849F473F3B4520BF65DE473F4A
:1000E000CBF61FBF271D483F41A81FBFCA5B483F33
:1000F0009F591FBF4E9A483FE50A1FBFB3D8483FDC
:1001000012BC1EBFFA16493F266D1EBF2155493F3E
:10011000221E1EBF2993493F06CF1DBF12D1493F62
:10012000D17F1DBFDC0E4A3F84301DBF874C4A3F44
:100130001FE11CBF138A4A3FA2911CBF7FC74A3FE1
:100140000C421CBFCC044B3F5FF21BBFFA414B3F3C
:1001500099A21BBF097F4B3FBB521BBFF8BB4B3F54
:10016000C6021BBFC7F84B3FB8B21ABF78354C3F29
:1001700093621ABF08724C3F55121ABF79AE4C3FBA
:1001800000C219BFCBEA4C3F947119BFFD264D3F09
:100190000F2119BF10634D3F73D018BF029F4D3F11
:1001A000C07F18BFD5DA4D3FF52E18BF89164E3FD8
:1001B00012DE17BF1C524E3F188D17BF908D4E3F59
:1001C000073C17BFE4C84E3FDFEA16BF17044F3F96
:1001D0009F9916BF2B3F4F3F474816BF1F7A4F3F8F
:1001E000D9F615BFF4B44F3F54A515BFA8EF4F3F44
:1001F000B75315BF3B2A503F040215BFAF64503FB1
:1002000039B014BF039F503F585E14BF37D9503FD9
:100210005F0C14BF4A13513F50BA13BF3D4D513FBD
:100220002A6813BF1087513FEE1513BFC2C0513F5C
:100230009AC312BF54FA513F307112BFC633523FB6
:10024000B01E12BF186D523F19CC11BF49A6523FC4
:100250006B7911BF59DF523FA72611BF4918533F91
:10026000CDD310BF1851533FDC8010BFC789533F17
:10027000D52D10BF55C2533FB8DA0FBFC3FA533F55
:1002800084870FBF0F33543F3B340FBF3B6B543F4A
:10029000DBE00EBF47A3543F658D0EBF31DB543FFB
:1002A000DA390EBFFB12553F38E60DBFA44A553F61
:1002B00081920DBF2C82553FB33E0DBF93B9553F80
:1002C000D0EA0CBFD9F0553FD7960CBFFE27563F5A
:1002D000C9420CBF025F563FA5EE0BBFE595563FE6
:1002E0006B9A0BBFA7CC563F1C460BBF4803573F2A
:1002F000B7F10ABFC739573F3D9D0ABF2670573F28
:10030000AD480ABF63A6573F09F409BF7FDC573FDA
:100310004E9F09BF7912583F7F4A09BF5348583F43
:100320009BF508BF0B7E583FA1A008BFA1B3583F63
:10033000924B08BF17E9583F6FF607BF6A1E593F37
:1003400036A107BF9C53593FE84B07BFAD88593FC3
:1003500086F606BF9CBD593F0EA106BF6AF2593F03
:10036000824B06BF16275A3FE2F505BFA05B5A3FF6
:100370002CA005BF09905A3F624A05BF50C45A3F9E
:1003800084F404BF75F85A3F919E04BF792C5B3FFB
:10039000894804BF5A605B3F6DF203BF1A945B3F0C
:1003A0003D9C03BFB8C75B3FF84503BF34FB5B3FD1
:1003B0009FEF02BF8E2E5C3F329902BFC7615C3F48
:1003C000B14202BFDD945C3F1CEC01BFD1C75C3F72
:1003D000739501BFA3FA5C3FB53E01BF532D5D3F4E
:1003E000E4E700BFE15F5D3FFF9000BF4D925D3FDE
:1003F000063A00BF97C45D3FF3C5FFBEBEF65D3F42
:10040000B217FFBEC3285E3F4A69FEBEA65A5E3FD2
:10041000BBBAFDBE678C5E3F040CFDBE05BE5E3FF1
:10042000275DFCBE81EF5E3F22AEFBBEDB205F3F5F
:10043000F7FEFABE12525F3FA54FFABE27835F3F19
:100440002DA0F9BE19B45F3F8EF0F8BEE9E45F3F1E
:10045000C840F8BE9615603FDC90F7BE2146603F6D
:10046000CBE0F6BE8976603F9330F6BECFA6603F04
:100470003580F5BEF2D6603FB1CFF4BEF206613FE3
:10048000071FF4BED036613F386EF3BE8A66613F07
:1004900043BDF2BE2296613F290CF2BE98C5613F72
:1004A000EA5AF1BEEAF4613F85A9F0BE1A24623F20
:1004B000FBF7EFBE2653623F4C46EFBE1082623F11
:1004C0007994EEBED7B0623F80E2EDBE7BDF623F43
:1004D0006330EDBEFC0D633F217EECBE5A3C633FB2
:1004E000BBCBEBBE956A633F3019EBBEAC98633F64
:1004F0008166EABEA1C6633FAEB3E9BE73F4633F53
:10050000B700E9BE2122643F9C4DE8BEAC4F643F7A
:100510005D9AE7BE147D643FFBE6E6BE59AA643FE0
:100520007533E6BE7BD7643FCB7FE5BE7904653F7C
:10053000FECBE4BE5431653F0E18E4BE0B5E653F52
:10054000FA63E3BEA08A653FC4AFE2BE10B7653F61
:100550006AFBE1BE5EE3653FEE46E1BE880F663FA3
:100560004F92E0BE8E3B663F8DDDDFBE7167663F1A
:10057000A928DFBE3093663FA273DEBECCBE663FC5
:1005800079BEDDBE45EA663F2E09DDBE9915673F9F
:10059000C153DCBECA40673F319EDBBED86B673FAC
:1005A00080E8DABEC196673FAD32DABE87C1673FE9
:1005B000B97CD9BE2AEC673FA3C6D8BEA816683F4F
:1005C0006B10D8BE0341683F135AD7BE396B683FE2
:1005D00099A3D6BE4C95683FFDECD5BE3CBF683FA5
:1005E0004136D5BE07E9683F647FD4BEAE12693F8D
:1005F00067C8D3BE323C693F4811D3BE9165693F9D
:10060000095AD2BECC8E693FAAA2D1BEE4B7693FD7
:100610002AEBD0BED7E0693F8A33D0BEA7096A3F34
:10062000CA7BCFBE52326A3FEAC3CEBED95A6A3FB6
:10063000EA0BCEBE3C836A3FCA53CDBE7BAB6A3F5A
:100640008B9BCCBE95D36A3F2CE3CBBE8CFB6A3F21
:10065000AE2ACBBE5E236B3F1072CABE0C4B6B3F03
:1006600053B9C9BE95726B3F7700C9BEFB996B3F0A
:100670007C47C8BE3BC16B3F628EC7BE58E86B3F2C
:1006800029D5C6BE500F6C3FD21BC6BE24366C3F68
:100690005C62C5BED45C6C3FC8A8C4BE5E836C3FC0
:1006A00015EFC3BEC5A96C3F4435C3BE07D06C3F30
:1006B000557BC2BE24F66C3F48C1C1BE1D1C6D3FB8
:1006C0001E07C1BEF2416D3FD54CC0BEA1676D3F54
:1006D0006F92BFBE2D8D6D3FEBD7BEBE93B26D3F07
:1006E0004A1DBEBED5D76D3F8B62BDBEF2FC6D3FCD
:1006F000AFA7BCBEEB216E3FB6ECBBBEBE466E3FA5
:10070000A031BBBE6D6B6E3F6E76BABEF88F6E3F8A
:100710001EBBB9BE5DB46E3FB2FFB8BE9ED86E3F81
:100720002A44B8BEBAFC6E3F8488B7BEB0206F3F83
:10073000C3CCB6BE83446F3FE610B6BE30686F3F91
:10074000EC54B5BEB88B6F3FD698B4BE1BAF6F3FAD
:10075000A5DCB3BE5AD26F3F5820B3BE73F56F3FCE
:10076000EF63B2BE6718703F6BA7B1BE373B703FF7
:10077000CBEAB0BEE15D703F102EB0BE6680703F28
:100780003A71AFBEC6A2703F49B4AEBE02C5703F5B
:100790003CF7ADBE17E7703F153AADBE0809713F93
:1007A000D47CACBED42A713F77BFABBE7A4C713FCC
:1007B0000102ABBEFB6D713F6F44AABE578F713F04
:1007C000C486A9BE8EB0713FFEC8A8BE9FD1713F3E
:1007D0001F0BA8BE8CF2713F254DA7BE5213723F6E
:1007E000128FA6BEF433723FE5D0A5BE7054723F9F
:1007F0009F12A5BEC774723F3F54A4BEF894723FC7
:10080000C595A3BE04B5723F33D7A2BEEBD4723FE9
:100810008718A2BEACF4723FC259A1BE4714733F01
:10082000E59AA0BEBE33733FEEDB9FBE0E53733F0F
:10083000DF1C9FBE3972733FB85D9EBE3F91733F10
:10084000789E9DBE1FB0733F20DF9CBED9CE733F04
:10085000AF1F9CBE6EED733F27609BBEDD0B743FE8
:1008600086A09ABE272A743FCEE099BE4B48743FBB
:10087000FE2099BE4966743F166198BE2284743F7B
:1008800017A197BED5A1743F00E196BE62BF743F29
:10089000D22096BEC9DC743F8D6095BE0BFA743FC2
:1008A00031A094BE2717753FBFDF93BE1D34753F3F
:1008B000351F93BEED50753F945E92BE976D753FA8
:1008C000DD9D91BE1C8A753F10DD90BE7BA6753FF5
:1008D0002C1C90BEB3C2753F325B8FBEC6DE753F27
:1008E000229A8EBEB3FA753FFCD88DBE7A16763F3B
:1008F000C0178DBE1B32763F6E568CBE974D763F2D
:1009000007958BBEEC68763F8AD38ABE1B84763F00
:10091000F8118ABE249F763F505089BE07BA763FB1
:10092000938E88BEC4D4763FC1CC87BE5BEF763F42
:10093000DA0A87BECC09773FDF4886BE1724773FA7
:10094000CE8685BE3C3E773FAAC484BE3A58773FE8
:10095000700284BE1372773F224083BEC58B773FFF
:10096000C07D82BE51A5773F4ABB81BEB7BE773FEF
:10097000C0F880BEF7D7773F223680BE10F1773FB0
:10098000E1E67EBE040A783F56617DBED122783F03
:10099000A4DB7BBE773B783FCB557ABEF853783FDC
:1009A000CCCF78BE526C783FA64977BE8684783F1C
:1009B0005AC375BE939C783FE83C74BE7BB4783FC5
:1009C00051B672BE3BCC783F942F71BED6E3783FD0
:1009D000B2A86FBE4AFB783FAB216EBE9812793F3A
:1009E0007F9A6CBEBF29793F2F136BBEC040793F01
:1009F000BA8B69BE9A57793F220468BE4E6E793F22
:100A0000667C66BEDC84793F86F464BE439B793F96
:100A1000836C63BE83B1793F5CE461BE9DC7793F5F
:100A2000135C60BE91DD793FA8D35EBE5EF3793F73
:100A30001A4B5DBE04097A3F6AC25BBE841E7A3FD0
:100A400097395ABEDD337A3FA4B058BE10497A3F79
:100A50008F2757BE1C5E7A3F589E55BE02737A3F61
:100A6000011554BEC1877A3F898B52BE599C7A3F8B
:100A7000F10151BECBB07A3F38784FBE16C57A3FF0
:100A800060EE4DBE3AD97A3F67644CBE37ED7A3F8F
:100A90004FDA4ABE0E017B3F185049BEBE147B3F61
:100AA000C2C547BE48287B3F4D3B46BEAB3B7B3F64
:100AB000B9B044BEE74E7B3F072643BEFC617B3F97
:100AC000379B41BEEA747B3F491040BEB2877B3FF3
:100AD0003E853EBE539A7B3F15FA3CBECDAC7B3F74
:100AE000CF6E3BBE20BF7B3F6CE339BE4DD17B3F19
:100AF000EC5738BE53E37B3F50CC36BE31F57B3FDD
:100B0000984035BEE9067C3FC4B433BE7A187C3FBA
:100B1000D42832BEE5297C3FC99C30BE283B7C3FAF
:100B2000A2102FBE444C7C3F61842DBE3A5D7C3FB9
:100B300004F82BBE086E7C3F8D6B2ABEB07E7C3FD6
:100B4000FCDE28BE318F7C3F515227BE8A9F7C3FFE
:100B50008CC525BEBDAF7C3FAD3824BEC9BF7C3F30
:100B6000B6AB22BEAECF7C3FA51E21BE6CDF7C3F64
:100B70007B911FBE03EF7C3F38041EBE73FE7C3F9B
:100B8000DE761CBEBC0D7D3F6BE91ABEDD1C7D3FD1
:100B9000E05B19BED82B7D3F3DCE17BEAC3A7D3F02
:100BA000834016BE59497D3FB2B214BEDE577D3F29
:100BB000CA2413BE3D667D3FCC9611BE74747D3F42
:100BC000B70810BE85827D3F8B7A0EBE6E907D3F4A
:100BD0004AEC0CBE309E7D3FF35D0BBECCAB7D3F3F
:100BE00086CF09BE40B97D3F054108BE8CC67D3F1A
:100BF0006EB206BEB2D37D3FC22305BEB1E07D3FDB
:100C0000029503BE88ED7D3F2E0602BE38FA7D3F79
:100C1000457700BEC2067E3F92D0FDBD24137E3FC5
:100C200073B2FABD5E1F7E3F2C94F7BD722B7E3FE0
:100C3000C075F4BD5E377E3F2E57F1BD23437E3F26
:100C40007638EEBDC14E7E3F9A19EBBD385A7E3FD5
:100C50009AFAE7BD88657E3F76DBE4BDB0707E3FE3
:100C60002EBCE1BDB17B7E3FC49CDEBD8B867E3F4A
:100C7000377DDBBD3D917E3F895DD8BDC99B7E3F01
:100C8000B93DD5BD2DA67E3FC81DD2BD69B07E3F02
:100C9000B7FDCEBD7FBA7E3F86DDCBBD6DC47E3F46
:100CA00036BDC8BD34CE7E3FC69CC5BDD4D77E3FC1
:100CB000397CC2BD4CE17E3F8D5BBFBD9DEA7E3F6E
:100CC000C33ABCBDC7F37E3FDD19B9BDC9FC7E3F49
:100CD000DAF8B5BDA4057F3FBBD7B2BD580E7F3F44
:100CE00080B6AFBDE4167F3F2B95ACBD491F7F3F5B
:100CF000BA73A9BD87277F3F3052A6BD9D2F7F3F86
:100D00008C30A3BD8D377F3FCF0EA0BD543F7F3FBA
:100D1000F9EC9CBDF4467F3F0ACB99BD6D4E7F3FF9
:100D200005A996BDBF557F3FE78693BDE95C7F3F30
:100D3000B46490BDEC637F3F6A428DBDC76A7F3F5C
:100D40000A208ABD7B717F3F94FD86BD08787F3F76
:100D50000ADB83BD6D7E7F3F6CB880BDAB847F3F77
:100D6000742B7BBDC28A7F3FE9E574BDB1907F3FA4
:100D700038A06EBD78967F3F625A68BD189C7F3F51
:100D8000681462BD91A17F3F4CCE5BBDE3A67F3F5F
:100D90000E8855BD0DAC7F3FAF414FBD0FB17F3FBA
:100DA0002FFB48BDEAB57F3F91B442BD9EBA7F3F5D
:100DB000D56D3CBD2ABF7F3FFC2636BD8FC37F3F2C
:100DC00007E02FBDCCC77F3FF69829BDE2CB7F3F20
:100DD000CC5123BDD1CF7F3F880A1DBD98D37F3F23
:100DE0002CC316BD37D77F3FB87B10BDAFDA7F3F2E
:100DF0002F340ABD00DE7F3F90EC03BD29E17F3F29
:100E0000B949FBBC2BE47F3F2DBAEEBC05E77F3F21
:100E10007B2AE2BCB8E97F3FA69AD5BC43EC7F3F72
:100E2000B00AC9BCA7EE7F3F9B7ABCBCE3F07F3F12
:100E300069EAAFBCF8F27F3F1C5AA3BCE6F47F3FDF
:100E4000B6C996BCACF67F3F38398ABC4AF87F3FBA
:100E50004B517BBCC1F97F3F003062BC11FB7F3F2F
:100E6000900E49BC39FC7F3F02ED2FBC39FD7F3F1E
:100E700059CB16BC13FE7F3F3053FBBBC4FE7F3FF4
:100E8000890FC9BB4EFF7F3FC1CB96BBB1FF7F3FF0
:100E9000C70F49BBECFF7F3FD40FC9BA737172749F
:100EA000660000004300232D302B2000686C4C00AE
:100EB000656667454647003031323334353637385A
:100EC00039414243444546003031323334353637B8
:090ED00038396162636465660053
:080EDC002866FF7F0100000001
:100EE40078563412541D0020000000000024F40041
:100EF40000F646A900000000000000010000020006
:100F04000003000004000005000006081D0700009F
:100F1400087000090F000A00000B00000C00000D0F
:100F240000000E00000F000010000011000012006D
:100F34000013000014000015000016000017000044
:100F44001800001900001A00001B70801C16FF1DF9
:100F540090FF1EB0FF1FC0FF20C0FF21CCFF22E383
:100F6400FF2300FF24061F25061F26061F27001F38
:100F74002863FF290C7F2A233F2B00002C00002D1F
:100F840000FF2E00FF2F143F302BFF3100FF32C231
:100F9400FF3327FF3410FF35D9FF3602FF3784FFB4
:100FA4003801FF3900FF3A00FF3BB7FF3C00FF3D2B
:100FB40000FF3E003F3F10FF4000FF4100FF4200A2
:100FC400FF4300FF4400FF4500FF4601FF4700FFC9
:100FD4004800FF49003F4A10FF4B38FF4CC3FF4D08
:100FE40020FF4E00FF4F00FF5000FF5109FF520049
:100FF400FF5300FF54003F5510FF5600FF5700FFFA
:101004005800FF5900FF5A00FF5B00FF5C00FF5DC2
:1010140000FF5E00FF5F003F601000619DFF6234CF
:10102400FF631CFF6400FF6500FF6600FF670DFFA0
:101034006800FF6900FF6A80BF6B00FF6C00FF6DF2
:1010440000FF6E40FF6F00FF7000FF7100FF7240F1
:10105400FF7300FF7480FF7500FF7640FF7700FF89
:101064007800FF7900FF7A40FF7B00FF7C00FF7D62
:1010740000FF7E00FF7F00FF8000FF81000F8200E1
:101084000F8300FF8400FF8500FF8600FF8700FFB9
:101094008800FF8900FF8A00FF8B00FF8C00FF8D12
:1010A40000FF8E00FF8F00FF9000FF91000092FF71
:1010B4000093000094000095000096000097000043
:1010C4009800FF9900FF9A00FF9B00FF9C00FF9D82
:1010D40000FF9E000F9F000FA000FFA100FFA200D1
:1010E400FFA300FFA400FFA500FFA600FFA700FFC9
:1010F400A800FFA900FFAA00FFAB00FFAC00FFADF2
:1011040000FFAE00FFAF00FFB000FFB100FFB20070
:10111400FFB300FFB400FFB5000FB600FFB700FF38
:10112400B800FFB900FFBA00FFBB00FFBC00FFBD61
:1011340000FFBE00FFBF00FFC000FFC100FFC200F0
:10114400FFC300FFC400FFC500FFC600FFC700FFC8
:10115400C800FFC900FFCA00FFCB000FCC00FFCDC1
:1011640000FFCE00FFCF00FFD000FFD100FFD20070
:10117400FFD300FFD400FFD500FFD600FFD700FF48
:10118400D800FFD900FFDA0000DB0000DC0000DD3E
:101194000D00DE0000DF0000E0F400E1F000E200FA
:1011A40000E30000E40000E50000E70000E80000C0
:1011B400E90000EA0000EB0000EC0000ED0000EEA6
:1011C4001400EF0000F00000F20002F3F000F4005D
:1011D40000F50000F70000F80000F9A800FA00008C
:1011E400FB8400FC0000FD0000FE0000FF01FF0086
:1011F40000000100000200000300000400000500DC
:10120400000600000700000800000900000A0000B2
:101214000B00000C00000D00000E00000F00001079
:101224000000110100120000130000149000153199
:10123400001600001700001801001900001A000031
:101244001B00001C00001D00001E00001F00FF20EA
:1012540000FF2101FF2200FF2300FF2490FF25311E
:10126400FF2600FF2700FF2801FF2900FF2A00FFB7
:101274002B000F2C00002D00002E00002F00FF304B
:1012840000FF3101FF3200FF3300FF3490FF35319E
:10129400FF3600FF3700FF3801FF3900FF3A00FF37
:1012A4003B000F3C00003D00003E00003F00FF40BB
:1012B40000FF4101FF4200FF4300FF4490FF45311E
:1012C400FF4600FF4700FF4801FF4900FF4A00FFB7
:1012D4004B000F4C00004D00004E00004F00FF502B
:1012E40000FF5100FF5200FF5300FF5490FF55319F
:1012F400FF5600FF5700FF5801FF5900FF5A00FF37
:101304005B000F5C00005D00005E0000FF00FF005A
:1013140000000000000000000000000000009B3CF2
:10132400D2FE0038000000000000000000000000B1
:10133400000000000000000000000C00FFB7FFFFE9
:10134400FFFFD2FE00380000000000000000000093
:1013540000000000000000009B3CFFFFFFFFFFFFB8
:1013640020B30000000000000000000000000000A6
:1013740000000000D201FFDFFFFFFFFFD2FE0038B4
:101384000000000000000000000000000000000059
:101394000000BF65FFFFFFFFFFFF20B30000000058
:1013A4000000000000000000000000000000D20166
:1013B400FFDFFFFFFFFFD2FE003800000000000047
:1013C400000000000000000000000000BF65FFFFF7
:1013D400FFFFFFFF20B3000000000000000000003A
:1013E4000000000000000000D201FFDFFFFFFFFF4C
:1013F400ACFD000000000000000000000000000040
:10140400000000000000BF65FFFFFFFFFFFFFFFFBC
:10141400FFFFF6FF00600000000000000000000075
:1014240000003603FFFFFFFFFFFFFFFFFFFFFFFF8B
:10143400FFFFFFFF87DC0000000000000000070042
:10144400DF96FFFFFFFFFFFFFFFFFFFFFFFFFFFF31
:10145400FFFFFFFF87DC0000000000003603FFFFF2
:10146400FFFFFFFFD2FE00380000D201FFDFFFFFC5
:10147400FFFFF6FF006000000000BF65FFFFFFFFF5
:10148400F6FF00600000000000003603FFFFFFFFCE
:10149400FFFF20B300000000BF65FFFFFFFFD2FE87
:1014A4000038000000000000D201FFDFFFFFFFFF53
:1014B40020B300000000BF65FFFFFFFFFBFFC091EA
:1014C4000000000000003603FFFFFFFFFFFF20B312
:1014D400000000003603FFFFFFFFFFFFD2FE0038CD
:1014E4000000D201FFDFFFFFFFFFF6FF00600000F6
:1014F40000000000BF65FFFFFFFFFFFFFFFFFFFFCE
:10150400FFFFFFFFFFFFFFFF87DC0000000000007C
:1015140000000700DF96FFFFFFFFFFFFFFFFFFFF55
:10152400FFFFFFFF87DC0000000000000000000058
:1015340000000000D201FFDFFFFFFFFFFFFFF6FF07
:101544000060000000000000000000000000000037
:1015540000000000D201FFDFFFFFFFFFFFFFFBFFE2
:10156400C091000000000000000000000000000026
:10157400BF65FFFFFFFFFFFFFFFFFFFFFFFFFFFF51
:10158400ACFD00000000000000000000BF65FFFF8C
:10159400FFFFFFFFFFFFFFFFFFFFFFFFFFFFFFFF57
:1015A400ACFD000000000000D201FFDFFFFFFFFFE1
:1015B400F6FF006000000C00FFB7FFFFFFFFFBFF1A
:1015C400C091000000009B3CFFFFFFFFFBFFC091A8
:1015D400000000000000D201FFDFFFFFFFFFACFDB1
:1015E40000000700DF96FFFFFFFFD2FE0038000077
:1015F400000000000700DF96FFFFFFFFD2FE003867
:101604000C00FFB7FFFFFFFFACFD0000000000006F
:1016140000000000BF65FFFFFFFFF6FF0060D2017E
:10162400FFDFFFFFFFFF87DC000000000000000079
:1016340000009B3CFFFFFFFFFBFFC091D201FFDFD7
:10164400FFFFFFFF87DC0000000000000000000037
:101654009B3CFFFFFFFFFBFFC091D201FFDFFFFFB9
:10166400FFFF87DC000000000000000000009B3C3E
:10167400FFFFFFFFFBFFC091D201FFDFFFFFFFFF72
:1016840087DC000000000000000000009B3CFFFF1E
:10169400FFFFFBFFC091D201FFDFFFFFFFFF87DCED
:1016A400000000000000000000009B3CFFFFFFFF63
:1016B400FBFFC0910C00FFB7FFFFFFFFACFD000074
:1016C4000000000000000000BF65FFFFFFFFF6FF01
:1016D40000600700DF96FFFFFFFFD2FE0038000026
:1016E400000000000700DF96FFFFFFFFD2FE003876
:1016F4000000BF65FFFFFFFFFBFFC091000000007B
:1017040000003603FFFFFFFFFFFFACFD00000000F9
:10171400D201FFDFFFFFFFFFF6FF006000000C00B7
:10172400FFB7FFFFFFFFFBFFC091000000000000B8
:10173400BF65FFFFFFFFFFFFFFFFFFFFFFFFFFFF8F
:10174400FFFFFFFFACFD00000000000000000700E9
:10175400DF96FFFFFFFFFFFFFFFFFFFFFFFFFFFF1E
:10176400D2FE00380000000000000000000000006D
:10177400D201FFDFFFFFFFFFFFFFFFFF20B30000E9
:101784000000000000000000000000000000000055
:101794000C00FFB7FFFFFFFFFFFFFFFF20B30000B8
:1017A4000000000000000000000000009B3CFFFF60
:1017B400FFFFFFFFFFFFFFFFFFFFFFFFD2FE003829
:1017C40000000000000000003603FFFFFFFFFFFFE2
:1017D400FFFFFFFFFFFFFFFFFFFFFFFFACFD000068
:1017E400000000000700DF96FFFFFFFFFFFF20B3AC
:1017F40000000700DF96FFFFFFFFFBFFC091000022
:101804000000D201FFDFFFFFFFFF87DC00000000C4
:1018140000003603FFFFFFFFFFFF20B300000000BE
:1018240000000000000000000000000000000000B4
:101834009B3CFFFFFFFFFBFFC09100000000000086
:10184400000000000000000000000000BF65FFFF72
:10185400FFFFFFFFD2FE0038000000000000000080
:10186400000000000C00FFB7FFFFFFFFFFFFFFFFBA
:10187400D2FE00380000000000000000000000005C
:1018840000000C00FFB7FFFFFFFFFFFFF6FF006043
:101894000000000000000000000000000000000044
:1018A4000C00FFB7FFFFFFFFFFFFFFFFFFFFACFDD3
:1018B4000000000000000000000000000000000024
:1018C400000000003603FFFFFFFFFFFFFFFF87DC80
:1018D4000000000000000000000000000000000004
:1018E400000000000C00FFB7FFFFFFFFF6FF0060E1
:1018F40000000000000000000000000000000000E4
:10190400000000009B3CFFFFFFFFFBFFC091D201E2
:10191400FFDFFFFFFFFF87DC000000000000000086
:1019240000009B3CFFFFFFFFFBFFC0910C00FFB7D3
:10193400FFFFFFFFD2FE0038000000000000070098
:10194400DF96FFFFFFFFF6FF00600000BF65FFFFAB
:10195400FFFFFFFFD2FE003800000000BF65FFFF5D
:10196400FFFFFFFFACFD000000000C00FFB7FFFF0E
:10197400FFFFFFFFFFFFFFFFFFFFFFFFFFFFFFFF73
:10198400F6FF0060000000000000D201FFDFFFFF4F
:10199400FFFFFFFFFFFFFFFFFFFFFFFFF6FF0060FA
:1019A4000000000000000000000000009B3CFFFF5E
:1019B400FFFFFFFFFFFFFFFF20B300000000000058
:1019C400000000000000000000000000D201FFDF62
:1019D400FFFFFFFFFFFFFBFFC091000000000000BE
:1019E4000000000000000700DF96FFFFFFFFFFFF7D
:1019F400FFFFFFFFFFFFFFFFACFD00000000000042
:101A040000000700DF96FFFFFFFFFFFFFFFFFFFF60
:101A1400FFFFFFFFFFFFFFFF87DC00000000000067
:101A24003603FFFFFFFFFFFFD2FE003800000C006B
:101A3400FFB7FFFFFFFFFBFFC09100000000BF6581
:101A4400FFFFFFFFF6FF0060000000000000360308
:101A5400FFFFFFFFFFFF20B300000700DF96FFFF3B
:101A6400FFFFD2FE0038000000000000D201FFDFBB
:101A7400FFFFFFFF87DC0000000000000000000003
:101A840000000000000000000000D201FFDFFFFFA3
:101A9400FFFF87DC000000000000000000000000E1
:101AA4000000000000000000BF65FFFFFFFFFBFF18
:101AB400C0910000000000000000000000000000D1
:101AC40000000000D201FFDFFFFFFFFFD2FE00385D
:101AD4000000000000000000000000000000000002
:101AE4000C00FFB7FFFFFFFFFFFF20B30000000063
:101AF4000000000000000000000000000700DF9666
:101B0400FFFFFFFFFFFFD2FE0038000000000000CF
:101B140000000000000000000700DF96FFFFFFFF49
:101B2400FFFFF6FF0060000000000000000000005E
:101B3400000000000700DF96FFFFFFFFFFFFFBFF31
:101B4400C091000000000000000000000000000040
:101B54000700DF96FFFFFFFFFFFFFFFF20B300003A
:101B64000000000000000000000000000000BF654D
:101B7400FFFFFFFFFFFFFFFF20B300000000000096
:101B840000000000000000000000BF65FFFFFFFF31
:101B9400FFFFFFFF20B30000000000000000000072
:101BA400000000000000BF65FFFFFFFFFFFFFFFF15
:101BB400FFFFFFFFFFFFFFFFFFFFFFFFFFFFACFD86
:101BC40000009B3CFFFFFFFFFFFFFFFFFFFFFFFF46
:101BD400FFFFFFFFFFFFFFFFFFFFFFFFACFD000064
:101BE4009B3CFFFFFFFFFFFFFFFFFFFFFFFFFFFF28
:101BF400FFFFFFFFFFFFFFFFFFFFACFD0000000042
